:100000000C946C370C949D370C949D370C949D3751
:100010000C949D370C949D370C949D370C949D3710
:100020000C949D370C949D370C949D370C949D3700
:100030000C949D370D945AA30C949D370C949D37C6
:100040000C949D370C94E7E50C949D370C949D37E8
:100050000C949D370C949D370C94AEE20D9410A334
:100060000C949D370D94FF7C0D94F57C0C949D377A
:100070000C949D370C949D370C949D370C949D37B0
:100080000D9469450C949D370C949D370C949D37C5
:100090000C949D370C949D370C949D370C949D3790
:1000A0000C949D370C949D370D943B450C949D37D3
:1000B0000C949D370C949D370C949D370C949D3770
:1000C0000C949D370C949D370C949D370C949D3760
:1000D0000C949D370C949D370C949D370C949D3750
:1000E0000C949D37084AD73B3BCE016E84BCBFFDC4
:1000F000C12F3D6C74319ABD56833DDA3D00C77FF8
:1001000011BED9E4BB4C3E916BAAAABE0000008090
:100110003F05A84CCDB2D44EB93836A9020C50B91F
:10012000918688083CA6AAAA2ABE000000803F0744
:10013000634236B79BD8A71A39685618AEBAAB5582
:100140008C1D3CB7CC5763BD6DEDFD753EF6177247
:1001500031BF000000803F08000000BE9224491219
:100160003EABAAAA2ABECDCCCC4C3E00000080BE3D
:10017000ABAAAAAA3E00000000BF000000803F001A
:1001800000000000084178D3BB4387D1133D190E0E
:100190003CC3BD4282AD2B3E68EC8276BED98FE176
:1001A000A93E4C80EFFFBE01C4FF7F3F000000006E
:1001B00000000C941B490C940C380C945FD20C94E6
:1001C0001ED70D943D2D0D94E89D0D9452310C9445
:1001D00071400C94B09B0C946A8C0D94109E0D94FD
:1001E0006C7D0C94EA630C9467770D942B9D0C94B2
:1001F00029400D94E89C0C94E1D50C9499820C94C0
:10020000244F0C9492560C940A4C0C94E94B0D9488
:10021000399D0D947A7E0C9493820C94668C0C9488
:100220005F520C949C820C94F3840C941E4C0C949E
:10023000BF580C94DB4C0C94BF3A0C94E2630D94C1
:10024000979D0D94099D0C9467560C94988D0D9470
:10025000FC9D0D94A37F0C945E3C0C945F890C94E0
:10026000B0450C94C0510C94144C0D943F7B0C94ED
:10027000F1570C9412410D94A17D0D94029D0C94A4
:10028000A4820C9435D40D94B7400C945F400C9428
:10029000B3560C944D400C946B560C9488740C948B
:1002A00035400D944F7B0C94773C0C94F8520D9490
:1002B000BB7D0C94C84F0C94CD370C94458F0C9497
:1002C000203F0C94EB3A0D940E7A0D94A97D0D9479
:1002D000957D0C9496820C9427800D94CB780D9488
:1002E000B07D0C94E8630C949F820D94BB460C94F3
:1002F0002E380C94C5640C94B77A0C9402710D944A
:1003000016790D947E9D0C94F6840D947B7D0C944F
:100310003F640C94C48E0C94823C0C9441400D9428
:10032000E39C0C9478450C9419590C942F400D942F
:100330001D9D0C9461D60D94A99D0D943D7D0C944A
:100340002A5B0C9498480C9437430C9410590C94E5
:10035000493D0C94653E0C9465400C94FD460C940C
:10036000653B0C946A6A0C94DF3B0D9405450D9433
:10037000487B0C9490820C94C1890C9469D50C94A0
:10038000628C0C94E2840D94F29D0C942C3C0C94A1
:10039000A43A0C9446D60C94F6500D944D7E0C94D1
:1003A000E2D20C94543A0C94E6630C94E7570C9404
:1003B00002D60D9400AF0C944A6D0C94EE630D942C
:1003C000917D0D948A7D0C9473560C94E4820C9468
:1003D0007E3B0C9409580C9437990D94FE9C0C9418
:1003E0002E490C944CD50D948D9D0C94A9820C949F
:1003F000F3460D94B4320C94977B0D94219D0C948C
:1004000095560C94008F0C94E4630D94FA9C0D9413
:10041000A19D0C94953B0C94217D0C947B560D94DE
:10042000E2460D94CF440C94D14A0C94E8D70D9435
:10043000BB9D0C945A860C9423400D94C37D0C9460
:10044000E0630C947B6B0D94997D0C9420830C9449
:1004500077560D94069D0D949D7D0C94BC640D946F
:10046000C59D0C943D4C0C94D94A0C9458590C944D
:10047000303B0C948B560C94216F0D94E2AE0C948F
:10048000133C0D940F9D0C94664F0D948FAE0C94FD
:10049000D14F0D94DE9D0C9498560C94FE3A0C941A
:1004A000B83B0C946F560C94E1D20C948A820C9455
:1004B00001510C941E440C946B400C9486850C9452
:1004C0003B400C945A5F0C94D73B0C9447480C94D7
:1004D000CB840C9485580D94199D0C947F560C94E4
:1004E00054440C9487560D94359D0C943F3B0C94CA
:1004F0003B3A0C94C9990C94294F0C94CF4A0C9414
:10050000BB660C94173B0C948F560C944E6E0C9457
:10051000109E0C94F1630C944F8D0C940F4C0C9422
:10052000D5720C94CDD40C94523B0C94F1D60C940F
:10053000917F0C942E4F0C94754F0C94295E0C9463
:100540008D820C94DFD60C94953A0C94A6820C9470
:1005500053400C94D83A0D94069E0C9401590C9477
:10056000194C0C94453C0C94BC4C0C942F830C946B
:100570005C4C0C946D3A0C9483560C9459400D9439
:1005800020450C94B4840C94DE630D94CF9D0C94A0
:10059000F8460D94AC7E0C94DE4A0C944D480C94B5
:1005A000FB680C9447400C94AC3B0C947F820C94F9
:1005B000D4400D94EA440C94D5530D94279D0C948B
:1005C0009D4C0C9415380C94EC630C94C2370D942C
:1005D000C4780C9406430D94139D0C94A4750C944C
:1005E0009F370C947C3A0C94D34A0D942F9D0D9414
:1005F000769D0D94A57D0D94B19D0D94839D0C94D5
:100600004B640D9427360C9436894E414E494E4921
:100610005459494E46CDCCCC3D0AD7233C17B7D1CF
:100620003877CC2B329595E6241FB14F0A00002075
:10063000410000C84200401C4620BCBE4CCA1B0EF4
:100640005AAEC59D7400407A10F35A00A0724E183D
:10065000090010A5D4E80000E87648170000E40B74
:1006600054020000CA9A3B000000E1F5050000803A
:10067000969800000040420F000000A08601000094
:1006800000102700000000E80300000000640000E4
:100690000000000A00000000000100000000002C23
:1006A00076D888DC674F0823DFC1DFAE59E1B1B7E8
:1006B00096E5E3E453C63AE651997696E8E6C284B5
:1006C00026EB898C9B62ED407C6FFCEFBC9C9F40CD
:1006D000F2BAA56FA5F490055A2AF75C936B6CF9F2
:1006E000676DC11BFCE0E40D47FEF520E6B500D0C8
:1006F000ED902E0300943577050080841E080000DD
:10070000204E0A000000C80C333333330F986E12AA
:10071000831141EF8D2114893BE65516CFFEE6DBB0
:1007200018D1844B381BF77C1D901DA4BBE42420FA
:100730003284725E228100C9F124ECA1E53D275587
:100740004E4C4F41442046494C414D454E54004C7F
:100750004F41442046494C414D454E540046494C7A
:10076000414D454E54204348414E47450050494471
:10077000204175746F74756E65202A005049442DB0
:1007800044202A005049442D49202A005049442D34
:1007900050202A0020082046616374002008204D64
:1007A0006178002008204D696E004F6666004F6E2C
:1007B000004175746F74656D7000565472617620D7
:1007C0004D696E00566D696E00566D61782045006A
:1007D000566D6178205A00566D6178205900566D2B
:1007E0006178205800416D6178204500416D617845
:1007F000205A00416D6178205900416D6178205880
:1008000000412D54726176656C00412D5265747201
:1008100061637400416363656C0056652D4A6572BF
:100820006B00565A2D4A65726B0056592D4A6572F7
:100830006B0056582D4A65726B0050726F626520CE
:100840005A204F66667365740050726F6265205956
:10085000204F66667365740050726F626520582081
:100860004F666673657400452073746570732F6DF1
:100870006D005A2053746570732F6D6D00592053AD
:10088000746570732F6D6D00582053746570732FED
:100890006D6D00416476616E6365642053657474A8
:1008A000696E6773003F0043616E63656C00496E5B
:1008B0006974004D34323800496E697469616C693D
:1008C0007A6520454550524F4D0046696C616D6513
:1008D0006E740054656D7065726174757265005355
:1008E000746570732F6D6D0050726F6265204F6676
:1008F0006673657473004A65726B00416363656C6F
:1009000065726174696F6E0056656C6F63697479A6
:100910000053657420486F6D65204F66667365747B
:100920007300436F6E66696775726174696F6E00FC
:100930003F004E65787420506F696E7400446F6E8E
:1009400065004E657874003F0043616E63656C20FE
:100950004F626A656374004E4F005945530043610E
:100960006E63656C204F626A656374203D004D6163
:10097000696E0053746F77004465706C6F79005333
:10098000572D4D6F64650053656C662D5465737407
:1009900000526573657400426564004E6F7A7A6C2C
:1009A000650046616E20537065656400436F6E6636
:1009B000696775726174696F6E00526573746F72E6
:1009C000652044656661756C7473004C6F616420CA
:1009D00053657474696E67730053746F7265205346
:1009E000657474696E677300507265686561742020
:1009F0002420436F6E6600506F776572204F7574C8
:100A0000616765004F6666004F6E0052756E6F75C8
:100A1000742053656E736F7200424C546F75636837
:100A20000050726F6265205A204F666673657400CD
:100A3000416476616E6365642053657474696E67A2
:100A400073004D61696E004D3730322054256400CB
:100A50004D36303020423020542564004D3730323E
:100A6000203B2564004D37303120542564004D373C
:100A70003032004D373031004D36303020423000BA
:100A80004D61696E00436F6E74696E7565004F66E7
:100A900066004F6E0052756E6F75742053656E73ED
:100AA0006F72005075726765206D6F7265005245F8
:100AB00053554D45204F5054494F4E533A005052D4
:100AC000494E54205041555345440020204E6F7AE2
:100AD0007A6C653A20005061726B696E672E2E2E1B
:100AE0000000005761697420666F720066696C616E
:100AF0006D656E74206368616E676500746F207346
:100B000074617274005761697420666F720066695F
:100B10006C616D656E7420756E6C6F616400004E63
:100B20006F7A7A6C652068656174696E6700506CD5
:100B30006561736520776169742E2E2E00005072F6
:100B400065737320627574746F6E00746F206865CE
:100B50006174206E6F7A7A6C650000496E736572FD
:100B6000742066696C616D656E7400616E642070DE
:100B70007265737320627574746F6E00746F206396
:100B80006F6E74696E7565005761697420666F7267
:100B90000066696C616D656E74206C6F6164000045
:100BA000507265737320427574746F6E00746F2099
:100BB000726573756D65207072696E74000057619F
:100BC000697420666F72207072696E7400746F2091
:100BD000726573756D652E2E2E0000576169742045
:100BE000666F720066696C616D656E7420707572F7
:100BF000676500003E2000256C642E25696D004568
:100C00007874727564656420546F74616C003E2062
:100C1000004C6F6E67657374204A6F622054696D73
:100C200065003E2000546F74616C205072696E74D0
:100C30002054696D6500436F6D706C657465640068
:100C40003A20005072696E7420436F756E74003ADA
:100C500020003135300035004245443A20415443AC
:100C60002031303447542D320052756E61776179EE
:100C70002057617463683A204F4E004D61782054CC
:100C8000656D7000333135004D696E2054656D70AF
:100C900000350045313A204550434F532031303024
:100CA0004B005053550047656E6572696300507282
:100CB0006F746F636F6C00312E3000426175640099
:100CC00032353030303000437265616C697479338D
:100CD000442052414D505300556E69666965642049
:100CE000426564204C6576656C696E670045787472
:100CF00072756465727300310074696E796D616339
:100D000068696E657333642E636F6D00544D3344B0
:100D10002043523130563200323032312D30342DB2
:100D2000313800322E302E375F4457372E33004D86
:100D300061726C696E005072696E746572205374D2
:100D400061747300546865726D6973746F727300B7
:100D5000426F61726420496E666F005072696E74F2
:100D6000657220496E666F004D61696E004D3130CD
:100D700030300053746F70205072696E7400526589
:100D800073756D65205072696E7400506F7765726F
:100D9000204F7574616765004D3139305335350A20
:100DA0004732380A47323950310A47323950330A0C
:100DB00047323953310A47323953300A47323946BC
:100DC000302E300A473239410A4D313034533231F6
:100DD000350A4732380A4D313039533231350A47F6
:100DE00031583135305931353046353030300A4799
:100DF000315A300A4D3530300A4D3430300A4D31D9
:100E0000313720536574205A204F6666736574002D
:100E10004D313036533132380A4D33303343385345
:100E20003231354530550A4D3530300A4D31313784
:100E3000205049442054756E6520446F6E65004D06
:100E40003139305335350A4D313034533231350A6A
:100E50004732380A4732394C310A4731205831304D
:100E6000305931303046353030300A47315A300051
:100E70004D3530300A4D3131372053657474696E09
:100E800067732053746F72656400507265702066DA
:100E90006F72205A2041646A75737400504944206F
:100EA00054756E650053746F726520536574746970
:100EB0006E6773005365747570004D61696E003F15
:100EC000004261636B0053746F70005072696E74FE
:100ED0002066726F6D204D65646961004368616EC4
:100EE0006765204D65646961004D32310041626F74
:100EF0007574205072696E746572004368616E6724
:100F0000652046696C616D656E74004C6576656C34
:100F1000696E6720546F6F6C7300436F6E6669670C
:100F200075726174696F6E0054656D70657261747D
:100F3000757265004D6F74696F6E00486F73742031
:100F40005374617274004E6F204D65646961005284
:100F50006573756D65205072696E740043616E63D0
:100F6000656C204F626A6563740054756E6500534A
:100F7000746F70205072696E7400506175736520D3
:100F80005072696E7400496E666F205363726565B6
:100F90006E003F005374617274205072696E740069
:100FA00043616E63656C005072696E740043616EDC
:100FB0006E6F7420656E74657220737562646972F9
:100FC0003A2000022E2E004D61696E002100486F0C
:100FD00074656E6420746F6F20636F6C640042618F
:100FE000636B0050726F63656564004F6666004F07
:100FF0006E00536F667420456E6473746F70730077
:101000004D6F74696F6E0044697361626C65205343
:1010100074657070657273004D3834004D3438203B
:1010200050726F62652054657374004732384F0AFE
:101030004D343820503130004C6576656C20436F5C
:10104000726E65727300556E6966696564204265EB
:1010500064204C6576656C696E6700486F6D65202D
:101060005A004732385A00486F6D652059004732A0
:10107000385900486F6D6520580047323858004194
:1010800075746F20486F6D65004D61696E00507218
:101090006568656174202420456E6400507265683F
:1010A0006561742024204265640054656D7065722A
:1010B000617475726500436F6F6C646F776E00507A
:1010C00072656865617420240046616E2053706506
:1010D0006564207E00426564004E6F7A7A6C65001C
:1010E0004D61696E0050726F6265205A204F6666CE
:1010F00073657400466C6F770046616E20537065AF
:101100006564207E00426564004E6F7A7A6C6500EB
:101110005370656564004D61696E005A2056616CBC
:101120007565004732380A4D313930205325690A38
:101130004D313039205325690A473239205031006A
:101140004265642054656D7000486F74656E64205C
:1011500054656D70002E2569004732395036432D95
:101160000048656967687420416D6F756E74004151
:10117000646A757374204D65736820486569676893
:10118000740046696E652054756E6520436C6F73FC
:10119000657374004732395034540046696E6520D7
:1011A00054756E6520416C6C0047323950345239A9
:1011B000393954004732380A473236435048256996
:1011C0004225690056616C696461746520437573DA
:1011D000746F6D204D657368004732380A473236A8
:1011E000435049310056616C6964617465204D65F6
:1011F000736820282429004732380A473236435082
:101200004930004732394A2569004C6576656C20C3
:101210004D657368005369646520506F696E74731F
:101220000047726964204D657368204C6576656C73
:10123000696E6700332D506F696E74204C6576655A
:101240006C696E67004732394A3000473239503393
:1012500052432E2569004D616E75616C2046696CA4
:101260006C2D696E00473239503242543000536D54
:101270006172742046696C6C2D696E00473239507A
:101280003354300046696C6C2D696E20416D6F756A
:101290006E74004D65736820696E76616C69646177
:1012A0007465642E0A00496E666F2053637265652B
:1012B0006E00496E76616C696461746520436C6F81
:1012C00073657374004732394900496E76616C6901
:1012D0006461746520416C6C00436F6E74696E7557
:1012E0006520426564204D6573680047323950318E
:1012F000430046696C6C2D696E204D657368004231
:1013000075696C6420436F6C64204D657368004799
:1013100032394E5031004275696C642043757374E4
:101320006F6D204D657368004732380A4D31393092
:1013300049310A4D31303949310A47323950310A81
:101340004D31303453300A4D313430533000427512
:10135000696C64204D657368202824290047323861
:101360000A4D31393049300A4D31303949300A4758
:10137000323950310A4D31303453300A4D31343026
:10138000533000473239256325690A4D3131372002
:10139000004D657368202569204C6F6164656400A9
:1013A0004D6573682025692053617665640053613B
:1013B000766520426564204D657368004C6F6164FA
:1013C00020426564204D657368004D656D6F7279CC
:1013D00020536C6F74004E6F2053746F7261676599
:1013E0000047323950345825735925735225690006
:1013F000202D2D2D2D2D005A3A00593A00486F6DA1
:10140000696E672058595A00473238004F66662087
:101410005072696E746572204261636B757000472B
:101420003239532D31004F757470757420666F72A8
:1014300020435356004732395431004F757470754C
:101440007420666F7220486F7374004732395430CD
:10145000004D657368204C6576656C696E67004564
:10146000646974204D6573680056616C69646174C9
:1014700065204D657368004D616E75616C6C7920F7
:101480004275696C64204D6573680047323949398B
:1014900039390A4732395032425430004275696C4A
:1014A00064204D65736800372E20536176652042B5
:1014B0006564204D65736800362E2046696E652090
:1014C00054756E6520416C6C004732395034523986
:1014D00039395400352E2056616C69646174652079
:1014E0004D65736800342E2046696E652054756E14
:1014F0006520416C6C0047323950345239393954C7
:1015000000332E2056616C6964617465204D6573EB
:101510006800322E20536D6172742046696C6C2D08
:10152000696E004732395033543000312E204275F5
:10153000696C6420436F6C64204D657368004732AA
:10154000394E503100556E696669656420426564A4
:10155000204C6576656C696E67004661646520485D
:101560006569676874004F75747075742055424CD6
:1015700020496E666F00473239570055424C20545F
:101580006F6F6C73004F7574707574204D65736860
:10159000204D6170004D6573682053746F726167F0
:1015A00065004D6573682045646974005374657007
:1015B0002D42792D537465702055424C004163745F
:1015C00069766174652055424C00473239410044C8
:1015D0006561637469766174652055424C004732D9
:1015E0003944004D6F74696F6E00434F4D4D554E39
:1015F00049434154494F4E0044525952554E0045BB
:1016000052524F525300494E464F004543484F00F7
:101610004F46460A004661646520486569676874FC
:101620002000426564204C6576656C696E67200019
:101630004661696C656420746F20656E61626C65DB
:1016400020426564204C6576656C696E670A0049C6
:101650006E76616C6964206D6573682E0A00766130
:101660006C69640A53746F7261676520736C6F7480
:101670003A2000696E004D65736820697320003F51
:10168000557365203020746F20003F496E76616C81
:1016900069642073746F7261676520736C6F742E58
:1016A0000A003F454550524F4D2073746F72616779
:1016B00065206E6F7420617661696C61626C652E65
:1016C0000A004D65736820706F696E74206F7574C1
:1016D000206F662072616E67650A004D34323120DA
:1016E000696E636F727265637420706172616D659B
:1016F0007465722075736167650A00446576696177
:1017000074696F6E0025533A2025730046696E692F
:1017100073686564210A003A207A3A2000206F66D7
:101720002000476F696E6720746F3A205800435756
:101730000A00206469723A0020616E676C653A00A5
:101740005374617274207261646975733A004D3428
:101750003820506F696E740025533A2025642F2578
:101760006400506F736974696F6E696E6720746886
:10177000652070726F62652E2E2E0A003F4C6567E1
:1017800073206F66206D6F76656D656E7420696D70
:10179000706C61757369626C652028302D31352954
:1017A0002E0A003F2028582C5929206F7574206F6D
:1017B0006620626F756E64732E0A0050726F6265E8
:1017C000206F7574206F6620626F756E6473003FC2
:1017D00053616D706C652073697A65206E6F74203B
:1017E000706C61757369626C652028342D35302901
:1017F0002E0A004D3438205A2D50726F62652052E7
:1018000065706561746162696C697479205465738F
:10181000740A003F2856296572626F7365206C65F3
:1018200076656C20696D706C61757369626C65209A
:1018300028302D34292E0A005374616E646172645D
:1018400020446576696174696F6E3A2000205261A8
:101850006E67653A2000204D61783A2000204D697E
:101860006E3A2000205369676D613A20004D656132
:101870006E3A20005741524E494E4721204C6F7717
:10188000205A204A65726B206D6179206C65616415
:1018900020746F20756E77616E7465642070617559
:1018A0007365732E0A004F4646004F4E0020204DB0
:1018B00061783A2000200020204D696E3A200053C4
:1018C0006F667420656E6473746F70733A20004D98
:1018D00032342053256C642054256C64004739321F
:1018E0002E392045257300473120462564004739AD
:1018F000322E39205A2573004731205A3020463283
:101900003030004731205825732059257320463345
:10191000303030004D34323020532569205A257341
:10192000004D3130362050256920532569004D3255
:101930003030204425730047323852305859004720
:1019400039322E39204530205A300A47315A257312
:10195000004D31303920532569004D313930205345
:101960002569004D343230205330205A3000204950
:101970006E76616C69642065787472756465722036
:101980000047322F47332062616420706172616DBD
:1019900065746572730A00536C6565702E2E2E0097
:1019A0005A2050726F6265205061737420426564E2
:1019B0000A005A2050726F62652050617374204291
:1019C000656400205A3A200020593A20004265649C
:1019D00020583A20004D65736820706F696E74203E
:1019E0006F7574206F662072616E67650A004D30F6
:1019F0002053746F70004D312053746F7000436C2E
:101A000069636B20746F20526573756D652E2E2E81
:101A1000004E6F204D6F76652E00456E642066691E
:101A20006C65206C6973740A00426567696E206694
:101A3000696C65206C6973740A004E6F206D656473
:101A400069610A00526573756D696E6720534400C1
:101A5000286E6F2066696C65290043757272656E29
:101A6000742066696C653A20005072696E74207447
:101A7000696D653A20000A53746174733A204669AF
:101A80006C616D656E7420757365643A20002C205E
:101A90004C6F6E67657374206A6F623A2000546FF2
:101AA00074616C2074696D653A20005374617473BD
:101AB0003A20002C204661696C65643A20002C2095
:101AC00046696E69736865643A20005072696E7485
:101AD000733A200053746174733A2000436F6F6C43
:101AE000696E672E2E2E0048656174696E672E2E12
:101AF0002E0045202553006F6B006F6666000B16A5
:101B00000616FF15F815EA1544454255473A004DAB
:101B100031313320530042656420436F6F6C696E2E
:101B2000672E2E2E004265642048656174696E67D9
:101B30002E2E2E00544D3344204352313056322045
:101B40004F46462E002F2F004D31343520533C692F
:101B50006E6465783E206F7574206F662072616ECA
:101B600067652028302D31290A0020520041636327
:101B7000656C65726174696F6E3A2050004D323049
:101B80003620580046523A0020466C6F773A2000C3
:101B90003A200020536572766F2000206F75742004
:101BA0006F662072616E67650A00536572766F20FA
:101BB0000020643A0020693A0020703A00496E76AD
:101BC000616C69642065787472756465720A0020BE
:101BD000643A0020693A0020703A00646973006535
:101BE0006E0043290A0061626C656420286D696E8D
:101BF0002074656D702000436F6C6420657874728A
:101C00007564657320617265200046696C616D655D
:101C10006E742072756E6F75742064697374616E72
:101C2000636520286D6D293A200046696C616D65F9
:101C30006E742072756E6F757420004F66667365E2
:101C40007473204170706C696564004572723A204B
:101C5000546F6F206661722100546F6F206661724D
:101C60002066726F6D207265666572656E636520B1
:101C7000706F696E740A00454550524F4D204F4BAE
:101C80000A00506F7765722D6C6F737320726563F5
:101C90006F7665727920004D383400446F6E652090
:101CA0007072696E74696E672066696C650A004DB2
:101CB0003737004D3331004361703A004D45415490
:101CC0005041434B00434F4F4C45525F54454D509C
:101CD00045524154555245004348414D4245525F9B
:101CE00054454D5045524154555245004241425988
:101CF0005354455050494E470041524353004D4FB5
:101D000054494F4E5F4D4F44455300544845524D42
:101D1000414C5F50524F54454354494F4E004C4F35
:101D20004E475F46494C454E414D45004155544F45
:101D30005245504F52545F53445F5354415455538E
:101D40000053445F57524954450052455045415451
:101D5000005344434152440050524F4D50545F533E
:101D60005550504F525400454D455247454E4359EA
:101D70005F50415253455200434153455F4C4947E0
:101D800048545F4252494748544E45535300544FBC
:101D900047474C455F4C494748545300534F4654BE
:101DA000574152455F504F574552004255494C44A8
:101DB0005F50455243454E54004C4556454C494EA4
:101DC000475F44415441005A5F50524F42450052D0
:101DD000554E4F5554004155544F4C4556454C00B7
:101DE0005052494E545F4A4F420050524F4752455D
:101DF0005353004155544F5245504F52545F544530
:101E00004D5000564F4C554D4554524943004545A1
:101E100050524F4D0042494E4152595F46494C4540
:101E20005F5452414E534645520053455249414C2E
:101E30005F584F4E5F584F4646004649524D5741F6
:101E400052455F4E414D453A4D61726C696E20328C
:101E50002E302E375F4457372E3320544D334420D5
:101E600053534D4442552028417072203234203261
:101E70003032312032303A30373A34332920534F20
:101E8000555243455F434F44455F55524C3A687441
:101E90007470733A2F2F6769746875622E636F6D63
:101EA0002F496E73616E6974794175746F6D6174D9
:101EB000696F6E2F4D61726C696E2F747265652F3C
:101EC000437265616C6974794477696E5F322E3054
:101ED0002050524F544F434F4C5F56455253494F39
:101EE0004E3A312E30204D414348494E455F5459BA
:101EF00050453A544D3344204352313056322045F8
:101F0000585452554445525F434F554E543A312030
:101F1000555549443A63656465326132662D343102
:101F200061322D343734382D396231322D633535F5
:101F30006336326633363766660A0050726F626502
:101F4000204F6666736574205A0050726F62652078
:101F50004F6666736574205A00290A0020746F204A
:101F6000003F5A206F7574206F662072616E67653E
:101F7000202800290A0020746F20003F59206F7527
:101F800074206F662072616E676520282D00290A13
:101F90000020746F20003F58206F7574206F6620FA
:101FA00072616E676520282D0050726F6265204F48
:101FB000666673657420580043616E6E6F74206F9F
:101FC00070656E2073756264697220002569730004
:101FD00025696D20256973002569682025696D20B4
:101FE00025697300256964202569682025696D20AD
:101FF0002569730025697920256964202569682091
:1020000025696D202569730023646566696E652006
:1020100044454641554C545F00626564004B642062
:10202000004B6920004B70200050494420417574DA
:102030006F74756E652066696E69736865642120CA
:1020400050757420746865206C617374204B702C1B
:10205000204B6920616E64204B6420636F6E737443
:10206000616E74732066726F6D2062656C6F77208D
:10207000696E746F20436F6E66696775726174690B
:102080006F6E2E680A00504944204175746F747554
:102090006E65206661696C6564212074696D656F89
:1020A00075740A00504944204175746F74756E65EB
:1020B000206661696C6564212054656D706572618C
:1020C0007475726520746F6F20686967680A0020F4
:1020D0004B643A2000204B693A2000204B703A2094
:1020E0000020436C617373696320504944200A00E7
:1020F000204E6F206F76657273686F6F740A0020D0
:1021000054753A2000204B753A2000206D61783AD2
:102110002000206D696E3A200020643A2000206281
:102120006961733A2000504944204175746F747599
:102130006E652073746172740A00504944204175C1
:10214000746F74756E65206661696C6564212054D6
:10215000656D706572617475726520746F6F20684B
:102160006967680A00504944204175746F74756E40
:102170006500504944204175746F74756E65206622
:1021800061696C65642120426164206865617465E1
:10219000722069640A004572723A207574663820AC
:1021A000666F6E74206E6F7420696E697469616CFD
:1021B000697A65642E004572723A2075746638201B
:1021C000666F6E74206E6F7420696E697469616CDD
:1021D000697A65642E004572723A207574663820FB
:1021E000666F6E74206E6F7420696E697469616CBD
:1021F000697A65642E0000FE0003FF8007C7C007F0
:1022000001E00000E00000F00000700400700E002B
:10221000701F00703F80F00E00E00F01E007C7C0A4
:1022200003FF8000FE0000FE0003FF8007C7C00F11
:1022300001E00E00E03F80F01F00700E007004000F
:10224000700000700000F00000E00701E007C7C068
:1022500003FF8000FE000E000E000E000E000E00B8
:102260000E000E000E007FC03F801F000E00040015
:1022700004000E001F003F807FC00E000E000E0005
:102280000E000E000E000E000E00FFFFFF7F80FF0D
:10229000C0FFC0FFC07F807F80FFC0FFC0FFC03F86
:1022A000001E000C0042656400456E636C6F737520
:1022B0007265002568753A25303268750025303220
:1022C00068753A25303268750020202020202020B3
:1022D0000020202020001FE02010201020101020BF
:1022E00010202010201030300840048003001FE030
:1022F0003FF03FF03FF01FE01FE03FF03FF03FF0C6
:102300000FC0078003003FFFF038007030FC302022
:10231000FC102078102030102C00D02E31D02F7BD4
:10232000D02F7BD02E31D02C00D020301020781030
:1023300020FC1030FC303800703FFFF03FFFF038D9
:1023400000703186302387102787902F87D02F0386
:10235000D02030102078102078102030102F03D09B
:102360002F87D02787902387103186303800703F21
:10237000FFF01FFFF81FFFF80410400208200208BA
:1023800020041040082080104100104100082080E7
:102390000410400000001FFFF81FFFF8FFFFFF8040
:1023A00000018E00E19F01F19381399F81F99F81A6
:1023B000F99FB9F98F28F18038018000019FFFF95A
:1023C0009174999B06A99B54A99B56A99B54999FCC
:1023D000FFF9FFFFFF544D33442043523130563252
:1023E0002052656164792E005072696E74696E675F
:1023F0002E2E2E006E6F74696669636174696F6E4C
:10240000200063616E63656C005072696E742041D8
:10241000626F72746564004469736D69737300550B
:10242000492041626F72746564004D323520500A54
:102430004D3234005072696E74205061757365645A
:1024400000526573756D650055492050617573655F
:102450000050617573696E672E2E2E00726573755C
:102460006D65004D32340050726F6265205A204F06
:1024700066667365740052756E6F75742044697377
:1024800074206D6D004C6F6164206D6D00556E6C35
:102490006F6164206D6D0046696C2E204469612E69
:1024A000004520696E206D6D5E33004D3330332062
:1024B0005531204525692053256900000C0F00FE89
:1024C00007022503BB017FFE08FE08FE050808067B
:1024D000000040F0C88888987810050808060000B9
:1024E000C0F88888888888F805050506000120302E
:1024F000F830200508080600002070F82020202071
:10250000E00509090600FF2070A8A8B88888702097
:10251000070505070001D86C366CD80509090600C7
:10252000FFF8A88888888888A8F8050A0A0600FEA7
:10253000205050505088A8A8887003030306000359
:1025400040A040FFFFFFFFFFFFFFFFFFFFFFFFFF78
:10255000FFFFFFFFFFFFFFFFFF0000000605FF0179
:102560000707060200808080808000800303030646
:102570000105A0A0A005060606000050F85050F87E
:10258000500509090600FF2070A8A07028A8702037
:10259000050707060000C8C81020409898050707DF
:1025A00006000040A0A040A89068010303060205B1
:1025B0008080800309090601FF2040408080804020
:1025C00040200309090601FF8040402020204040B0
:1025D0008005070706000020A8702070A8200505C8
:1025E000050600012020F820200203030601FFC099
:1025F0004080050101060003F8020202060100C046
:10260000C00507070600000810102040408005079D
:1026100007060000708898A8C8887003070706019D
:102620000040C040404040E00507070600007088B9
:1026300008102040F8050707060000F808103008C9
:10264000887005070706000010305090F81010053C
:102650000707060000F880F00808887005070706DD
:102660000000304080F0888870050707060000F8F9
:1026700008101020202005070706000070888870C9
:102680008888700507070600007088887808106041
:10269000020505060100C0C000C0C0020606060112
:1026A000FFC0C000C0408003050506010120408036
:1026B0004020050303060002F800F80305050601A3
:1026C0000180402040800507070600007088102028
:1026D0002000200507070600007088B8A8B88070A1
:1026E000050707060000708888F8888888050707AE
:1026F000060000F04848704848F00507070600004B
:1027000070888080808870050707060000F04848C0
:10271000484848F0050707060000F88080F08080F0
:10272000F8050707060000F88080F0808080050724
:1027300007060000708880809888700507070600EB
:1027400000888888F8888888030707060100E04029
:1027500040404040E0050707060000381010101008
:1027600090600507070600008890A0C0A09088052B
:102770000707060000808080808080F80507070634
:10278000000088D8A8888888880507070600008880
:1027900088C8A89888880507070600007088888878
:1027A000888870050707060000F08888F080808020
:1027B00005070706000070888888A8906805070745
:1027C000060000F08888F0A0908805070706000042
:1027D00070888070088870050707060000F82020C0
:1027E0002020202005070706000088888888888820
:1027F0007005070706000088888888505020050764
:102800000706000088888888A8A8500507070600E2
:1028100000888850205088880507070600008888AF
:102820005020202020050707060000F8081020404F
:1028300080F80309090601FFE080808080808080A5
:10284000E00507070600008040402010100803093B
:10285000090601FFE020202020202020E0050303BE
:102860000600052050880501010600FEF803030359
:1028700006010580402005050506000070087888DF
:10288000780507070600008080F0888888F0050535
:1028900005060000708080887005070706000008A4
:1028A0000878888888780505050600007088F0801B
:1028B00070050707060000304840E040404005072B
:1028C000070600FE708888887808700507070600EC
:1028D000008080F088888888030707060100400090
:1028E000C0404040E00409090601FE10003010100D
:1028F0001010906005070706000080808890E09027
:1029000088030707060100C04040404040E005053D
:1029100005060000D0A8A8A8A8050505060000B077
:10292000C8888888050505060000708888887005B5
:1029300007070600FEF0888888F0808005070706F4
:1029400000FE78888888780808050505060000B02C
:10295000C880808005050506000078807008F005B5
:1029600007070600002020F820202018050505068E
:102970000000888888986805050506000088888812
:1029800050200505050600008888A8A85005050503
:1029900006000088502050880507070600FE88883A
:1029A0008850204080050505060000F8102040F8FA
:1029B0000309090601FF20404040804040402001BB
:1029C00009090602FF808080808080808080030962
:1029D000090601FF8040404020404040800503033D
:1029E00006000248A890FF486F6D696E6720466137
:1029F000696C6564006F70656E00545249474745C5
:102A0000524544003A200066696C616D656E740041
:102A10007A5F6D696E00795F6D696E00785F6D69D0
:102A20006E005265706F7274696E6720656E6473B4
:102A3000746F70207374617475730A0020746F6F03
:102A4000206C6F6E6720657874727573696F6E2085
:102A500070726576656E7465640A0020636F6C64DD
:102A600020657874727573696F6E20707265766513
:102A70006E7465640A00486F6D65202573257325A3
:102A800073204669727374005761726E696E673A9B
:102A900020486F6D696E672042756D7020446976BD
:102AA00069736F72203C20310A00020204000000AA
:102AB00000000000000000000000809D4300009B1B
:102AC000430000C843000000410000004100000036
:102AD00040FFFFFF00000001000000010000800037
:102AE000555555000000400033333300AAAA2A0090
:102AF0004992240000002000C7711C009999190018
:102B0000D1451700555515003BB11300244912005B
:102B100011111100000010000F0F0F00E3380E001C
:102B200043790D00CCCC0C00C3300C00E8A20B00A4
:102B300064210B00AAAA0A00703D0A009DD8090072
:102B4000427B090092240900DCD308008888080031
:102B50001042080000000800F0C107008787070046
:102B600075500700711C07003EEB0600A1BC060073
:102B70006990060066660600703E06006118060051
:102B800017F4050074D105005BB00500B290050094
:102B9000627205005555050078390500B81E05001C
:102BA000050505004EEC040087D40400A1BD040017
:102BB00090A7040049920400C17D0400EE6904005E
:102BC000C7560400444404005C3204000821040099
:102BD00041100400000004003FF00300F8E003008F
:102BE00026D20300C3C30300CCB503003AA80300F8
:102BF0000A9B0300388E0300C08103009F75030009
:102C0000D0690300505E03001D53030034480300E5
:102C1000913D03003333030016290300381F0300DE
:102C200097150300300C0300030303000BFA0200A6
:102C300049F10200BAE802005CE002002DD802006F
:102C40002DD0020059C80200B0C0020031B9020004
:102C5000DAB10200AAAA0200A0A30200BC9C0200F2
:102C6000FA9502005C8F0200DF8802008282020077
:102C7000457C02002776020027700200436A0200AA
:102C80007C640200D05E02003F590200C85302007B
:102C9000FFFDFCFAF8F6F4F2F0EEECEAE9E7E5E322
:102CA000E1E0DEDCDAD9D7D5D4D2D0CFCDCBCAC8DB
:102CB000C7C5C3C2C0BFBDBCBAB9B7B6B4B3B2B062
:102CC000AFADACAAA9A8A6A5A4A2A1A09E9D9C9ABE
:102CD00099989795949392908F8E8D8B8A898887F7
:102CE0008684838281807F7E7D7B7A797877767512
:102CF00074737271706F6E6D6C6B6A69686766650C
:102D000064636261605F5E5D5C5B5A5958585756F8
:102D1000555453525150504F4E4D4C4B4A4A4948CE
:102D2000474646454443424241403F3E3E3D3C3B90
:102D30003B3A393838373635353433323231303042
:102D40002F2E2E2D2C2B2B2A2929282727262525E7
:102D500024232322212120201F1E1E1D1C1C1B1B7F
:102D60001A1919181817161615151413131212110B
:102D700011100F0F0E0E0D0D0C0C0B0A0A0909088D
:102D80000807070606050504040303020201000004
:102D900000809D4300009B430000C84300000000EA
:102DA000000000000000000053657474696E6773D2
:102DB0002053746F72656400454550524F4D204951
:102DC0006E697469616C697A65640A003F556E6169
:102DD000626C6520746F2073617665206D65736821
:102DE00020646174612E0A003F556E61626C65203B
:102DF000746F206C6F6164206D657368206461740A
:102E0000612E0A00556E696669656420426564201A
:102E10004C6576656C696E67003B20003A0A0020BD
:102E2000204D363033200020440020204D343132F4
:102E300020530046696C616D656E742072756E6F0B
:102E400075742073656E736F723A002055004C00E4
:102E500046696C616D656E74206C6F61642F756E70
:102E60006C6F6164206C656E677468733A00202033
:102E70004D3835312058005A2D50726F6265204F01
:102E800066667365740020204D3431332053005042
:102E90006F7765722D4C6F7373205265636F766523
:102EA00072793A0020440020490020204D3330340C
:102EB00020500020440020490020204D3330312094
:102EC00050005049442073657474696E67733A000A
:102ED00020460020480020204D3134352053004D3D
:102EE0006174657269616C206865617475702070C9
:102EF0006172616D65746572733A00206D65736807
:102F000065732E0A0A00454550524F4D2063616E8D
:102F100020686F6C642000416374697665204D659C
:102F2000736820536C6F743A200020204D34323087
:102F300020530020204D323036205800486F6D65F8
:102F4000206F66667365743A002058002053002095
:102F5000204D323035204200416476616E636564F5
:102F60003A20423C6D696E5F7365676D656E745F94
:102F700074696D655F75733E20533C6D696E5F6665
:102F8000656564726174653E20543C6D696E5F7462
:102F9000726176656C5F66656564726174653E201A
:102FA000583C6D61785F785F6A65726B3E20593C72
:102FB0006D61785F795F6A65726B3E205A3C6D6126
:102FC000785F7A5F6A65726B3E20453C6D61785F21
:102FD000655F6A65726B3E0020540020520020201D
:102FE0004D323034205000416363656C657261740A
:102FF000696F6E2028756E6974732F7332293A20B9
:10300000503C7072696E745F616363656C3E205200
:103010003C726574726163745F616363656C3E20CA
:10302000543C74726176656C5F616363656C3E00ED
:1030300020204D3230312058004D6178696D756D1A
:1030400020416363656C65726174696F6E202875D9
:103050006E6974732F7332293A0020204D32303359
:103060002058004D6178696D756D206665656472E4
:10307000617465732028756E6974732F73293A0023
:1030800053746570732070657220756E69743A00B0
:1030900020440020204D32303020530020446973FA
:1030A00061626C65640A0046696C616D656E7420CE
:1030B00073657474696E67733A0020204D3134393A
:1030C0002043203B20556E69747320696E20436550
:1030D0006C736975730A0020286D6D2900202047E4
:1030E0003231202020203B20556E69747320696E98
:1030F000206D6D003F4D65736820746F6F206269AD
:103100006720666F7220454550524F4D2E0A0000D1
:1031100000FA430000FA43000020410000964200FC
:1031200000A0420000A0420000C8430000BA42DCF8
:10313000050000DC050000640000004B00000024D6
:10314000F4D43050C38E20C2A24017828B7011126B
:103150007A910D816CD90AA861E108C758660761A8
:103160005143061E4B5D05C145A7041A41110409D0
:103170003D9803713931034036DB0265339102D447
:10318000305402802E1D02632CEE01752AC501B059
:1031900028A001102781018F2564012B244B01E019
:1031A000223401AC211F018D200D01801FFC008401
:1031B0001EED00971DDF00B81CD200E61BC60020E4
:1031C0001BBC00641AB200B219A8000A19A0006A58
:1031D000189900D117910040178B00B51684003163
:1031E000167E00B31579003A157300C7146F0058A6
:1031F000146A00EE1366008813630025135E00C78F
:10320000125B006C12570015125400C1115100706E
:10321000114F0021114B00D61049008D1047004678
:1032200010440002104200C00F4000800F3E0042D8
:103230000F3C00060F3B00CB0E3800930E37005CAE
:103240000E3500270E3400F30D3200C10D31009011
:103250000D3000600D2E00320D2D00050D2C00D913
:103260000C2B00AE0C2900850C29005C0C270035C6
:103270000C27000E0C2600E80B2400C40B2400A031
:103280000B23007D0B23005A0B2100390B21001862
:103290000B2000F80A1F00D90A1E00BB0A1E009D61
:1032A0000A1D00800A1D00630A1C00470A1B002C2F
:1032B0000A1B00110A1A00F7091A00DD091900C4D7
:1032C000091900AB091900920917007B091800635E
:1032D0000917004C09160036091600200916000AC5
:1032E000091500F5081500E0081400CC081400B812
:1032F000081400A4081400900813007D0812006B45
:103300000813005808120046081200340811002360
:103310000811001208110001081100F0071000E068
:10332000071000D0071000C0071000B0070F00A161
:1033300007100091070E0083070F0074070F006548
:10334000070E0057070E0049070E003B070D002E21
:10335000070E0020070D0013070D0006070D00F9EA
:10336000060C00ED060D00E0060C00D4060C00C8AB
:10337000060C00BC060C00B0060C00A4060B00995D
:10338000060C008D060B0082060B0077060B006C06
:10339000060B0061060A0057060B004C060A0042A5
:1033A000060A0038060A002E060A0024060A001A39
:1033B000060A001006090007060A00FD050900F4C8
:1033C000050900EB050900E2050900D9050900D04F
:1033D000050900C7050900BE050900B5050800ADCF
:1033E000050800A50509009C050800940508008C47
:1033F000050800840508007C050800740508006CB9
:10340000050700650508005D050700560508004E24
:10341000050700470507004005080038050700318B
:103420000507002A050700230507001C05060016EE
:103430000507000F0507000805060002050700FB49
:10344000040600F5040700EE040600E8040600E2A6
:10345000040700DB040600D5040600CF040600C9FB
:10346000040600C3040600BD040600B7040600B14C
:10347000040500AC040600A6040600A00405009B99
:1034800004060095040500900406008A04050085E2
:10349000040500800406007A040500750405007028
:1034A0000405006B04050066040500610405005C6A
:1034B00004050057040500520405004D04050048AA
:1034C000040500430405003E0404003A04050035E9
:1034D000040500300404002C040500270404002324
:1034E0000405001E0404001A04040016040500115B
:1034F0000404000D04040009040500040404000091
:10350000040400FC030400F8030400F4030400F0C6
:10351000030400EC030400E8030400E4030400E0F7
:10352000030400DC030400D8030400D4030400D027
:10353000030400CC030400C8030300C503030024F4
:10354000F404D9201BC40C5C0E9804C4095F026506
:10355000077101F405F900FB04B30048048700C1BA
:103560000369005803550003034500BE023A008476
:1035700002310053022A002902250004022000E43F
:10358000011C00C8011900AF011700980114008444
:10359000011300710110006101100051010E004380
:1035A000010D0036010B002B010B0020010B001553
:1035B0000109000C01090003010800FB000800F3E9
:1035C000000800EB000700E4000600DE000600D85B
:1035D000000600D2000600CC000500C7000500C2AE
:1035E000000500BD000400B9000400B5000400B1EE
:1035F000000400AD000400A9000400A5000300A21F
:103600000003009F0004009B000300980003009546
:1036100000020093000300900003008D0002008B65
:10362000000300880002008600020084000300817D
:103630000002007F0002007D0002007B0002007992
:1036400000020077000100760002007400020072A0
:10365000000100710002006F0002006D0001006CAB
:103660000002006A000100690002006700010066B4
:1036700000010065000100640002006200010061B9
:10368000000100600001005F0002005D0001005CBD
:103690000001005B0001005A0001005900010058C0
:1036A00000010057000100560001005500010054C0
:1036B00000010053000000530001005200010051BE
:1036C000000100500001004F0001004E0000004EBC
:1036D0000001004D0001004C0001004B0000004BB8
:1036E0000001004A000100490001004800000048B4
:1036F00000010047000100460000004600010045AF
:1037000000000045000100440001004300000043A8
:1037100000010042000000420001004100000041A1
:10372000000100400001003F0000003F0001003E9A
:103730000000003E0001003D0000003D0001003C93
:103740000000003C0000003C0001003B0000003B8A
:103750000001003A0000003A000100390000003981
:103760000001003800000038000000380001003778
:10377000000000370001003600000036000000366F
:103780000001003500000035000000350001003464
:10379000000000340000003400010033000000335A
:1037A000000000330001003200000032000000324F
:1037B0000001003100000031000000310001003044
:1037C00000000030000000300001002F0000002F3A
:1037D0000000002F0000002F0001002E0000002E2E
:1037E0000000002E0001002D0000002D0000002D23
:1037F0000000002D0001002C0000002C0000002C17
:103800000000002C0001002B0000002B0000002B0A
:103810000000002B0001002A0000002A0000002AFE
:103820000000002A000100290000002900000029F2
:1038300000000029000000290001002800000028E5
:1038400000000028000000280000002800010027D8
:1038500000000027000000270000002700000027CC
:1038600000010026000000260000002600000026BF
:1038700000000026000100250000002500000025B2
:1038800000000025000000250000002500010024A4
:103890000000002400000024000000240000002498
:1038A000000100230000002300000023000000238B
:1038B000000000230000002300000023000100227C
:1038C0000000002200000022000000220000002270
:1038D0000000002200010021000000210000002162
:1038E0000000002100000021000000210000002154
:1038F0000001002000000020000000200000002047
:103900000000002000000020000000200000002037
:103910000001001F0000001F0000001F0000001F2A
:103920000000001F0000001F0000001F0001001E1B
:103930000000001E0000001E0000001E00000039F4
:103940003000003325000087190000B00F0000DBB5
:10395000080000BD040000740200003F01000020C8
:10396000436F756E7420583A00426564004531001B
:10397000626564002C2073797374656D2073746FB5
:103980007070656421204865617465725F49443ACE
:10399000200048656174696E67204661696C6564E2
:1039A0000048656174696E67206661696C656400D2
:1039B0004D3131322053687574646F776E0010009A
:1039C000C90210012C014001220170011801B0014F
:1039D0000E01F00104015002FA00B002F0003003C1
:1039E000E600D003DC009004D2007005C800A006F9
:1039F000BE000008B400B009AA00D00BA000600E01
:103A0000960060118C000015820020197800C01DFE
:103A10006E00A0226400B0275A00902C50000031A4
:103A20004600E0343C0010383200903A2800603CF8
:103A30001E00A03D1400803E0A00203F00005448B4
:103A400045524D414C2052554E4157415900546802
:103A500065726D616C2052756E6177617900457297
:103A6000723A204D415854454D50004D41585445EF
:103A70004D502074726967676572656400457272A3
:103A80003A204D494E54454D50004D494E54454DF8
:103A9000502074726967676572656400202F00208A
:103AA00042403A0020403A0020573A0020573A005E
:103AB000496E76616C6964206578747275646572AC
:103AC0000A007C3C3E5E2B3D3F2F5B5D3B2C2A2257
:103AD0005C0043616E6E6F74206F70656E2073754D
:103AE000626469722000534420496E697420466103
:103AF000696C0053442063617264206F6B0A006F2D
:103B000070656E526F6F74206661696C65640A003F
:103B1000766F6C756D652E696E6974206661696C6F
:103B200065640A004E6F20534420636172640A008A
:103B3000363726033C3D380E2E303E131A1C180A29
:103B4000FF4309070844000124F404D9201BC40CD6
:103B50005C0E9804C4095F0265077101F405F90061
:103B6000FB04B30048048700C103690058035500F3
:103B700003034500BE023A008402310053022A00CA
:103B80002902250004022000E4011C00C8011900DC
:103B9000AF01170098011400840113007101100097
:103BA0006101100051010E0043010D0036010B00B0
:103BB0002B010B0020010B00150109000C0109006D
:103BC00003010800FB000800F3000800EB000700F9
:103BD000E4000600DE000600D8000600D200060061
:103BE000CC000500C7000500C2000500BD000400B0
:103BF000B9000400B5000400B1000400AD000400E9
:103C0000A9000400A5000300A20003009F00040017
:103C10009B0003009800030095000200930003003E
:103C2000900003008D0002008B000300880002005A
:103C30008600020084000300810002007F00020071
:103C40007D0002007B000200790002007700010085
:103C50007600020074000200720001007100020090
:103C60006F0002006D0001006C0002006A0001009C
:103C700069000200670001006600010065000100A4
:103C800064000200620001006100010060000100A8
:103C90005F0002005D0001005C0001005B000100AC
:103CA0005A000100590001005800010057000100AE
:103CB00056000100550001005400010053000000AF
:103CC00053000100520001005100010050000100AA
:103CD0004F0001004E0000004E0001004D000100A9
:103CE0004C0001004B0000004B0001004A000100A5
:103CF00049000100480000004800010047000100A1
:103D0000460000004600010045000000450001009B
:103D10004400010043000000430001004200000095
:103D2000420001004100000041000100400001008C
:103D30003F0000003F0001003E0000003E00010087
:103D40003D0000003D0001003C0000003C00000080
:103D50003C0001003B0000003B0001003A00000075
:103D60003A0001003900000039000100380000006D
:103D70003800000038000100370000003700010063
:103D8000360000003600000036000100350000005B
:103D90003500000035000100340000003400000050
:103DA0003400010033000000330000003300010044
:103DB000320000003200000032000100310000003B
:103DC0003100000031000100300000003000000030
:103DD000300001002F0000002F0000002F00000025
:103DE0002F0001002E0000002E0000002E00010018
:103DF0002D0000002D0000002D0000002D0001000E
:103E00002C0000002C0000002C0000002C00010001
:103E10002B0000002B0000002B0000002B000100F5
:103E20002A0000002A0000002A0000002A000100E9
:103E300029000000290000002900000029000000DE
:103E400029000100280000002800000028000000D0
:103E500028000000280001002700000027000000C3
:103E600027000000270000002700010026000000B6
:103E700026000000260000002600000026000100A9
:103E8000250000002500000025000000250000009E
:103E9000250000002500010024000000240000008F
:103EA0002400000024000000240001002300000082
:103EB0002300000023000000230000002300000076
:103EC0002300000023000100220000002200000067
:103ED0002200000022000000220000002200010059
:103EE000210000002100000021000000210000004E
:103EF000210000002100000021000100200000003E
:103F00002000000020000000200000002000000031
:103F10002000000020000000200001001F00000021
:103F20001F0000001F0000001F0000001F00000015
:103F30001F0000001F0001001E0000001E00000006
:103F40001E0000001E00000024F4D43050C38E2058
:103F5000C2A24017828B7011127A910D816CD90A1E
:103F6000A861E108C7586607615143061E4B5D050D
:103F7000C145A7041A411104093D98037139310361
:103F80004036DB0265339102D4305402802E1D028C
:103F9000632CEE01752AC501B028A001102781010C
:103FA0008F2564012B244B01E0223401AC211F0139
:103FB0008D200D01801FFC00841EED00971DDF0089
:103FC000B81CD200E61BC600201BBC00641AB2005D
:103FD000B219A8000A19A0006A189900D117910017
:103FE00040178B00B516840031167E00B31579009A
:103FF0003A157300C7146F0058146A00EE13660078
:104000008813630025135E00C7125B006C12570013
:1040100015125400C111510070114F0021114B00B5
:10402000D61049008D10470046104400021042008F
:10403000C00F4000800F3E00420F3C00060F3B00C7
:10404000CB0E3800930E37005C0E3500270E34007F
:10405000F30D3200C10D3100900D3000600D2E00C7
:10406000320D2D00050D2C00D90C2B00AE0C2900B3
:10407000850C29005C0C2700350C27000E0C26004F
:10408000E80B2400C40B2400A00B23007D0B2300AD
:104090005A0B2100390B2100180B2000F80A1F00D1
:1040A000D90A1E00BB0A1E009D0A1D00800A1D00C1
:1040B000630A1C00470A1B002C0A1B00110A1A0085
:1040C000F7091A00DD091900C4091900AB09190024
:1040D000920917007B091800630917004C091600A4
:1040E00036091600200916000A091500F508150002
:1040F000E0081400CC081400B8081400A408140048
:10410000900813007D0812006B0813005808120075
:10411000460812003408110023081100120811008B
:1041200001081100F0071000E0071000D007100090
:10413000C0071000B0070F00A107100091070E0084
:1041400083070F0074070F0065070E0057070E0066
:1041500049070E003B070D002E070E0020070D003B
:1041600013070D0006070D00F9060C00ED060D0003
:10417000E0060C00D4060C00C8060C00BC060C00BF
:10418000B0060C00A4060B0099060C008D060B006F
:1041900082060B0077060B006C060B0061060A0016
:1041A00057060B004C060A0042060A0038060A00B1
:1041B0002E060A0024060A001A060A001006090044
:1041C00007060A00FD050900F4050900EB050900D2
:1041D000E2050900D9050900D0050900C705090055
:1041E000BE050900B5050800AD050800A5050900D4
:1041F0009C050800940508008C050800840508004B
:104200007C050800740508006C05070065050800BA
:104210005D050700560508004E0507004705070025
:104220004005080038050700310507002A0507008A
:10423000230507001C050600160507000F050700EB
:104240000805060002050700FB040600F504070048
:10425000EE040600E8040600E2040700DB040600A2
:10426000D5040600CF040600C9040600C3040600F6
:10427000BD040600B7040600B1040500AC04060046
:10428000A6040600A00405009B0406009504050092
:10429000900406008A0405008504050080040600D9
:1042A0007A04050075040500700405006B04050020
:1042B00066040500610405005C0405005704050060
:1042C000520405004D0405004804050043040500A0
:1042D0003E0404003A0405003504050030040400DF
:1042E0002C04050027040400230405001E04040018
:1042F0001A04040016040500110404000D0404004F
:10430000090405000404040000040400FC03040084
:10431000F8030400F4030400F0030400EC030400B9
:10432000E8030400E4030400E0030400DC030400E9
:10433000D8030400D4030400D0030400CC03040019
:10434000C8030300C5030300726F746174696F6E64
:10435000206D61747269783A0A0024F404D9201B34
:10436000C40C5C0E9804C4095F0265077101F40572
:10437000F900FB04B30048048700C1036900580337
:10438000550003034500BE023A0084023100530287
:104390002A002902250004022000E4011C00C801B3
:1043A0001900AF0117009801140084011300710176
:1043B00010006101100051010E0043010D00360193
:1043C0000B002B010B0020010B00150109000C0153
:1043D000090003010800FB000800F3000800EB00DF
:1043E0000700E4000600DE000600D8000600D20048
:1043F0000600CC000500C7000500C2000500BD0096
:104400000400B9000400B5000400B1000400AD00D0
:104410000400A9000400A5000300A20003009F00FF
:1044200004009B0003009800030095000200930025
:104430000300900003008D0002008B000300880041
:1044400002008600020084000300810002007F0059
:1044500002007D0002007B0002007900020077006C
:104460000100760002007400020072000100710079
:1044700002006F0002006D0001006C0002006A0083
:10448000010069000200670001006600010065008C
:104490000100640002006200010061000100600090
:1044A00001005F0002005D0001005C0001005B0094
:1044B00001005A0001005900010058000100570096
:1044C0000100560001005500010054000100530096
:1044D0000000530001005200010051000100500093
:1044E00001004F0001004E0000004E0001004D0091
:1044F00001004C0001004B0000004B0001004A008D
:104500000100490001004800000048000100470088
:104510000100460000004600010045000000450083
:10452000010044000100430000004300010042007C
:104530000000420001004100000041000100400075
:1045400001003F0000003F0001003E0000003E006F
:1045500001003D0000003D0001003C0000003C0067
:1045600000003C0001003B0000003B0001003A005D
:1045700000003A0001003900000039000100380055
:10458000000038000000380001003700000037004C
:104590000100360000003600000036000100350042
:1045A0000000350000003500010034000000340038
:1045B000000034000100330000003300000033002D
:1045C0000100320000003200000032000100310022
:1045D0000000310000003100010030000000300018
:1045E0000000300001002F0000002F0000002F000D
:1045F00000002F0001002E0000002E0000002E0001
:1046000001002D0000002D0000002D0000002D00F5
:1046100001002C0000002C0000002C0000002C00E9
:1046200001002B0000002B0000002B0000002B00DD
:1046300001002A0000002A0000002A0000002A00D1
:1046400001002900000029000000290000002900C5
:1046500000002900010028000000280000002800B8
:1046600000002800000028000100270000002700AB
:10467000000027000000270000002700010026009E
:104680000000260000002600000026000000260092
:104690000100250000002500000025000000250085
:1046A0000000250000002500010024000000240077
:1046B000000024000000240000002400010023006A
:1046C000000023000000230000002300000023005E
:1046D000000023000000230001002200000022004F
:1046E0000000220000002200000022000000220042
:1046F0000100210000002100000021000000210035
:104700000000210000002100000021000100200025
:104710000000200000002000000020000000200019
:1047200000002000000020000000200001001F0009
:1047300000001F0000001F0000001F0000001F00FD
:1047400000001F0000001F0001001E0000001E00EE
:1047500000001E0000001E00000024F4D43050C3EE
:104760008E20C2A24017828B7011127A910D816C3B
:10477000D90AA861E108C7586607615143061E4B74
:104780005D05C145A7041A411104093D980371391B
:1047900031034036DB0265339102D4305402802E5F
:1047A0001D02632CEE01752AC501B028A001102757
:1047B00081018F2564012B244B01E0223401AC21BF
:1047C0001F018D200D01801FFC00841EED00971D30
:1047D000DF00B81CD200E61BC600201BBC00641A18
:1047E000B200B219A8000A19A0006A189900D117DE
:1047F000910040178B00B516840031167E00B3156A
:1048000079003A157300C7146F0058146A00EE134C
:1048100066008813630025135E00C7125B006C12EC
:10482000570015125400C111510070114F00211191
:104830004B00D61049008D1047004610440002106E
:104840004200C00F4000800F3E00420F3C00060FA8
:104850003B00CB0E3800930E37005C0E3500270E60
:104860003400F30D3200C10D3100900D3000600DA9
:104870002E00320D2D00050D2C00D90C2B00AE0C96
:104880002900850C29005C0C2700350C27000E0C34
:104890002600E80B2400C40B2400A00B23007D0B92
:1048A00023005A0B2100390B2100180B2000F80AB5
:1048B0001F00D90A1E00BB0A1E009D0A1D00800AA7
:1048C0001D00630A1C00470A1B002C0A1B00110A6A
:1048D0001A00F7091A00DD091900C4091900AB090B
:1048E0001900920917007B091800630917004C0989
:1048F000160036091600200916000A091500F508E9
:104900001500E0081400CC081400B8081400A4082E
:104910001400900813007D0812006B08130058085B
:104920001200460812003408110023081100120872
:10493000110001081100F0071000E0071000D00777
:104940001000C0071000B0070F00A107100091076A
:104950000E0083070F0074070F0065070E0057074E
:104960000E0049070E003B070D002E070E00200722
:104970000D0013070D0006070D00F9060C00ED06EB
:104980000D00E0060C00D4060C00C8060C00BC06A6
:104990000C00B0060C00A4060B0099060C008D0656
:1049A0000B0082060B0077060B006C060B006106FD
:1049B0000A0057060B004C060A0042060A00380699
:1049C0000A002E060A0024060A001A060A0010062B
:1049D000090007060A00FD050900F4050900EB05BA
:1049E0000900E2050900D9050900D0050900C7053D
:1049F0000900BE050900B5050800AD050800A505BC
:104A000009009C050800940508008C050800840531
:104A100008007C050800740508006C0507006505A2
:104A200008005D050700560508004E05070047050C
:104A300007004005080038050700310507002A0572
:104A40000700230507001C050600160507000F05D3
:104A500007000805060002050700FB040600F50430
:104A60000700EE040600E8040600E2040700DB0489
:104A70000600D5040600CF040600C9040600C304DE
:104A80000600BD040600B7040600B1040500AC042E
:104A90000600A6040600A00405009B040600950479
:104AA0000500900406008A040500850405008004C2
:104AB00006007A04050075040500700405006B0407
:104AC000050066040500610405005C040500570448
:104AD0000500520405004D04050048040500430488
:104AE00005003E0404003A040500350405003004C6
:104AF00004002C04050027040400230405001E0400
:104B000004001A04040016040500110404000D0436
:104B10000400090405000404040000040400FC036C
:104B20000400F8030400F4030400F0030400EC03A1
:104B30000400E8030400E4030400E0030400DC03D1
:104B40000400D8030400D4030400D0030400CC0301
:104B50000400C8030300C503030024F404D9201B88
:104B6000C40C5C0E9804C4095F0265077101F4056A
:104B7000F900FB04B30048048700C103690058032F
:104B8000550003034500BE023A008402310053027F
:104B90002A002902250004022000E4011C00C801AB
:104BA0001900AF011700980114008401130071016E
:104BB00010006101100051010E0043010D0036018B
:104BC0000B002B010B0020010B00150109000C014B
:104BD000090003010800FB000800F3000800EB00D7
:104BE0000700E4000600DE000600D8000600D20040
:104BF0000600CC000500C7000500C2000500BD008E
:104C00000400B9000400B5000400B1000400AD00C8
:104C10000400A9000400A5000300A20003009F00F7
:104C200004009B000300980003009500020093001D
:104C30000300900003008D0002008B000300880039
:104C400002008600020084000300810002007F0051
:104C500002007D0002007B00020079000200770064
:104C60000100760002007400020072000100710071
:104C700002006F0002006D0001006C0002006A007B
:104C80000100690002006700010066000100650084
:104C90000100640002006200010061000100600088
:104CA00001005F0002005D0001005C0001005B008C
:104CB00001005A000100590001005800010057008E
:104CC000010056000100550001005400010053008E
:104CD000000053000100520001005100010050008B
:104CE00001004F0001004E0000004E0001004D0089
:104CF00001004C0001004B0000004B0001004A0085
:104D00000100490001004800000048000100470080
:104D1000010046000000460001004500000045007B
:104D20000100440001004300000043000100420074
:104D3000000042000100410000004100010040006D
:104D400001003F0000003F0001003E0000003E0067
:104D500001003D0000003D0001003C0000003C005F
:104D600000003C0001003B0000003B0001003A0055
:104D700000003A000100390000003900010038004D
:104D80000000380000003800010037000000370044
:104D9000010036000000360000003600010035003A
:104DA0000000350000003500010034000000340030
:104DB0000000340001003300000033000000330025
:104DC000010032000000320000003200010031001A
:104DD0000000310000003100010030000000300010
:104DE0000000300001002F0000002F0000002F0005
:104DF00000002F0001002E0000002E0000002E00F9
:104E000001002D0000002D0000002D0000002D00ED
:104E100001002C0000002C0000002C0000002C00E1
:104E200001002B0000002B0000002B0000002B00D5
:104E300001002A0000002A0000002A0000002A00C9
:104E400001002900000029000000290000002900BD
:104E500000002900010028000000280000002800B0
:104E600000002800000028000100270000002700A3
:104E70000000270000002700000027000100260096
:104E8000000026000000260000002600000026008A
:104E9000010025000000250000002500000025007D
:104EA000000025000000250001002400000024006F
:104EB0000000240000002400000024000100230062
:104EC0000000230000002300000023000000230056
:104ED0000000230000002300010022000000220047
:104EE000000022000000220000002200000022003A
:104EF000010021000000210000002100000021002D
:104F0000000021000000210000002100010020001D
:104F10000000200000002000000020000000200011
:104F200000002000000020000000200001001F0001
:104F300000001F0000001F0000001F0000001F00F5
:104F400000001F0000001F0001001E0000001E00E6
:104F500000001E0000001E00000024F4D43050C3E6
:104F60008E20C2A24017828B7011127A910D816C33
:104F7000D90AA861E108C7586607615143061E4B6C
:104F80005D05C145A7041A411104093D9803713913
:104F900031034036DB0265339102D4305402802E57
:104FA0001D02632CEE01752AC501B028A00110274F
:104FB00081018F2564012B244B01E0223401AC21B7
:104FC0001F018D200D01801FFC00841EED00971D28
:104FD000DF00B81CD200E61BC600201BBC00641A10
:104FE000B200B219A8000A19A0006A189900D117D6
:104FF000910040178B00B516840031167E00B31562
:1050000079003A157300C7146F0058146A00EE1344
:1050100066008813630025135E00C7125B006C12E4
:10502000570015125400C111510070114F00211189
:105030004B00D61049008D10470046104400021066
:105040004200C00F4000800F3E00420F3C00060FA0
:105050003B00CB0E3800930E37005C0E3500270E58
:105060003400F30D3200C10D3100900D3000600DA1
:105070002E00320D2D00050D2C00D90C2B00AE0C8E
:105080002900850C29005C0C2700350C27000E0C2C
:105090002600E80B2400C40B2400A00B23007D0B8A
:1050A00023005A0B2100390B2100180B2000F80AAD
:1050B0001F00D90A1E00BB0A1E009D0A1D00800A9F
:1050C0001D00630A1C00470A1B002C0A1B00110A62
:1050D0001A00F7091A00DD091900C4091900AB0903
:1050E0001900920917007B091800630917004C0981
:1050F000160036091600200916000A091500F508E1
:105100001500E0081400CC081400B8081400A40826
:105110001400900813007D0812006B081300580853
:10512000120046081200340811002308110012086A
:10513000110001081100F0071000E0071000D0076F
:105140001000C0071000B0070F00A1071000910762
:105150000E0083070F0074070F0065070E00570746
:105160000E0049070E003B070D002E070E0020071A
:105170000D0013070D0006070D00F9060C00ED06E3
:105180000D00E0060C00D4060C00C8060C00BC069E
:105190000C00B0060C00A4060B0099060C008D064E
:1051A0000B0082060B0077060B006C060B006106F5
:1051B0000A0057060B004C060A0042060A00380691
:1051C0000A002E060A0024060A001A060A00100623
:1051D000090007060A00FD050900F4050900EB05B2
:1051E0000900E2050900D9050900D0050900C70535
:1051F0000900BE050900B5050800AD050800A505B4
:1052000009009C050800940508008C050800840529
:1052100008007C050800740508006C05070065059A
:1052200008005D050700560508004E050700470504
:1052300007004005080038050700310507002A056A
:105240000700230507001C050600160507000F05CB
:1052500007000805060002050700FB040600F50428
:105260000700EE040600E8040600E2040700DB0481
:105270000600D5040600CF040600C9040600C304D6
:105280000600BD040600B7040600B1040500AC0426
:105290000600A6040600A00405009B040600950471
:1052A0000500900406008A040500850405008004BA
:1052B00006007A04050075040500700405006B04FF
:1052C000050066040500610405005C040500570440
:1052D0000500520405004D04050048040500430480
:1052E00005003E0404003A040500350405003004BE
:1052F00004002C04050027040400230405001E04F8
:1053000004001A04040016040500110404000D042E
:105310000400090405000404040000040400FC0364
:105320000400F8030400F4030400F0030400EC0399
:105330000400E8030400E4030400E0030400DC03C9
:105340000400D8030400D4030400D0030400CC03F9
:105350000400C8030300C503030070012C01900181
:105360002701B0012201C0011D01F0011801100246
:10537000130130020E016002090190020401C00213
:10538000FF000003FA004003F5008003F000D003A3
:10539000EB002004E6007004E100E004DC004005BE
:1053A000D700C005D2004006CD00D006C800800757
:1053B000C3003008BE00F008B900C009B400B00A4C
:1053C000AF00B00BAA00D00CA500000EA000500F3B
:1053D0009B00C01096005012910000148C00C01564
:1053E0008700B0178200B0197D00D01B7800001E26
:1053F000730040206E0090226900F0246400402772
:105400005F0090295A00E02B5500102E50002030EC
:105410004B0010324600E033410090353C0010371D
:10542000370070383200A0392D00B03A2800A03B78
:105430002300603C1E00103D1900903D1400103EFA
:105440000F00703E0A00C03E0500003F0000403FD4
:10545000FBFF803FF6FFC03FF1FF1000C9021001C3
:105460002C014001220170011801B0010E01F00170
:1054700004015002FA00B002F0003003E600D0034D
:10548000DC009004D2007005C800A006BE00000831
:10549000B400B009AA00D00BA000600E9600601105
:1054A0008C000015820020197800C01D6E00A0221B
:1054B0006400B0275A00902C500000314600E034C0
:1054C0003C0010383200903A2800603C1E00A03D9D
:1054D0001400803E0A00203F00005A5F6D6F766521
:1054E0005F636F6D700A0047323858004732385991
:1054F000004732385A004732384F0A4D343820506E
:105500003130004D3834004732395034523939394E
:105510005400473239503454004732380A47323643
:1055200043504930004732380A47323643504931F8
:10553000004732394A30004732395033543000473F
:1055400032395032425430004732380A4D31393006
:1055500049300A4D31303949300A47323950310A21
:105560004D31303453300A4D3134305330004732EE
:10557000380A4D31393049310A4D31303949310A13
:1055800047323950310A4D31303453300A4D3134BD
:10559000305330004732394E5031004732395031A4
:1055A00043004732394900473239543000473239D5
:1055B000543100473239532D310047323949393996
:1055C000390A4732395032425430004732394E504E
:1055D0003100473239503354300047323950345259
:1055E0003939395400473239503452393939540035
:1055F0004732394400473239410047323957004178
:105600007869732000206D696E3A00206D61783AE8
:10561000004641535400534C4F570005000006010B
:105620000004000601000605000000060004004515
:1056300072726F722077726974696E6720746F205E
:10564000454550524F4D210A0053544F5050454448
:105650002E20005072696E7465722073746F7070C2
:1056600065642064756520746F206572726F727353
:105670002E2046697820746865206572726F7220EA
:10568000616E6420757365204D39393920746F203F
:10569000726573746172742E202854656D70657222
:1056A00061747572652069732072657365742E204C
:1056B0005365742069742061667465722072657325
:1056C00074617274696E67290A004E6F20436865C1
:1056D000636B73756D2077697468206C696E6520E3
:1056E0006E756D6265722C204C617374204C696E0E
:1056F000653A20004E6F20436865636B73756D20BB
:1057000077697468206C696E65206E756D6265726C
:105710002C204C617374204C696E653A20006368DC
:1057200065636B73756D206D69736D617463682C4F
:10573000204C617374204C696E653A20004C696E90
:1057400065204E756D626572206973206E6F7420DE
:105750004C617374204C696E65204E756D62657284
:105760002B312C204C617374204C696E653A2000FB
:105770004D3131300053657269616C20737461740E
:105780007573206D69736D617463680A0077616970
:10579000740A0053442072656164206572726F72EE
:1057A0000A00486F74656E642049646C6520546912
:1057B0006D656F757400486F74656E642049646C24
:1057C000652054696D656F75740A002121204B496D
:1057D0004C4C20636175736564206279204B494CA1
:1057E0004C20627574746F6E2F70696E0A002121EF
:1057F000204B494C4C2063617573656420627920AD
:10580000746F6F206D75636820696E61637469766B
:10581000652074696D65202D2063757272656E74E4
:1058200020636F6D6D616E643A2000706175736501
:10583000004D363030002066696C616D656E745FB6
:1058400072756E6F7574200066696C616D656E743B
:105850005F72756E6F757420540046696C616D657A
:105860006E7452756E6F75742054004D6564696175
:105870002052656D6F766564004D656469612049ED
:105880006E736572746564004D3130303053006260
:105890007573793A2070617573656420666F722044
:1058A000696E7075740A00627573793A207061755B
:1058B00073656420666F7220757365720A00627585
:1058C00073793A2070726F63657373696E670A004B
:1058D000506C656173652052657365740050524960
:1058E0004E5445522048414C5445440025533A20DB
:1058F000255300706F7765726F6666004B494C4C9C
:1059000045442E20005072696E7465722068616C87
:105910007465642E206B696C6C28292063616C6C43
:105920006564210A0053544F505045442E200050C6
:1059300072696E7465722073746F70706564206430
:10594000756520746F206572726F72732E204669C0
:105950007820746865206572726F7220616E6420B1
:10596000757365204D39393920746F2072657374F1
:105970006172742E202854656D7065726174757241
:10598000652069732072657365742E2053657420D9
:1059900069742061667465722072657374617274D3
:1059A000696E67290A006563686F3A004572726F15
:1059B000723A00204A0020204D3432312049002024
:1059C0002047323920493939390A006163746976D0
:1059D000650A00696E00002053797374656D207646
:1059E000312E303120002020207C0A004E414E0014
:1059F00020202E20202000207C004C43443A0A0026
:105A00004353563A0A0020666F7220003A0A0A0091
:105A10000A42656420546F706F6772617068792004
:105A20005265706F72740050726F62696E672046C3
:105A300061696C65640A0050726F62696E67204626
:105A400061696C656400205A3A200020593A2000B0
:105A500042656420583A20004732384C3000446F89
:105A60006E652E0A003F496E76616C69642073741E
:105A70006F7261676520736C6F742E0A3F55736592
:105A8000203020746F20003F454550524F4D207309
:105A9000746F72616765206E6F7420617661696CE6
:105AA00061626C652E0A00446F6E652E0A003F49E4
:105AB0006E76616C69642073746F726167652073C0
:105AC0006C6F742E0A3F557365203020746F200070
:105AD0003F454550524F4D2073746F72616765208A
:105AE0006E6F7420617661696C61626C652E0A006C
:105AF0004732392050322066696E69736865642EBA
:105B00000A005859206F7574736964652070726952
:105B10006E7461626C65207261646975732E0A002F
:105B20003F4572726F7220696E20427573696E65AF
:105B300073732043617264206D6561737572656D66
:105B4000656E742E0A004D616E75616C6C79207003
:105B5000726F62696E6720756E72656163686162FB
:105B60006C6520706F696E74732E0A00292E0A0A04
:105B70000050726F62696E672061726F756E64208B
:105B800028004D65736820696E76616C6964617484
:105B900065642E2050726F62696E67206D65736850
:105BA0002E0A004D657368207A65726F65642E0A4F
:105BB0000044656661756C742073746F726167650B
:105BC00020736C6F7420302073656C65637465643A
:105BD0002E0A004C6F6164696E6720746573745F90
:105BE0007061747465726E2076616C7565732E0ACF
:105BF0000A00496E76616C696420746573745F7025
:105C000061747465726E2076616C75652E20282D26
:105C10003120746F2032290A0A0020696E76616C87
:105C20006964617465642E0A0A004C6F636174696B
:105C30006F6E7300456E74697265204D6573680000
:105C40005374616E6461726420446576696174693D
:105C50006F6E3A20004D65616E204D657368204877
:105C600065696768743A200023206F662073616D50
:105C7000706C65733A20000A4D657368206F6E6C16
:105C800079207061727469616C6C7920706F7075C5
:105C90006C617465642E0A0A0050726F62696E67E7
:105CA00020506F696E740025532025692F256900E7
:105CB0002E0A002F0050726F62696E67206D657347
:105CC0006820706F696E74200020616E64207461BA
:105CD0006B652061206D6561737572656D656E74AD
:105CE0002E0A006D6D20746869636B2E0A00427580
:105CF00073696E6573732043617264206973200059
:105D000052656D6F76652026204D656173757265ED
:105D1000204265640052656D6F7665207368696D19
:105D200000506C616365207368696D20756E6465F1
:105D300072206E6F7A7A6C65000A4D657368206F09
:105D40006E6C79207061727469616C6C7920706F0F
:105D500070756C617465642E0A004D65736820501F
:105D60006F696E74204D656173757265642061742E
:105D70003A20004D65617375726500506C61636512
:105D8000205368696D2026204D656173757265002A
:105D90004D6F76696E6720746F206E657874004D64
:105DA0006573682045646974696E672053746F7009
:105DB00070656400446F6E652045646974696E6740
:105DC000204D6573680A00446F6E652045646974F0
:105DD000696E67204D6573680046696E652054756D
:105DE0006E696E67204D6573680028582C5929200C
:105DF0006F757473696465207072696E7461626C2A
:105E000065207261646975732E0A004F666673655A
:105E100074206F7574206F6620626F756E64732EC8
:105E200020283020746F2031306D6D290A0A004916
:105E30006E76616C6964206D617020747970652E76
:105E40000A0A003F28462961646520686569676819
:105E50007420666F7220426564204C6576656C2004
:105E6000436F7272656374696F6E206E6F74207019
:105E70006C61757369626C652E0A0A003F43616E3E
:105E8000277420616374697661746520616E642093
:105E900064656163746976617465206174207468F7
:105EA000652073616D652074696D652E0A0A004274
:105EB0006F7468205820262059206C6F63617469C4
:105EC0006F6E73206D7573742062652073706563E7
:105ED00069666965642E0A0A003F496E76616C69DD
:105EE0006420677269642073697A6520284A2920D2
:105EF0007370656369666965642028322D39292EBF
:105F00000A0A003F285029686173652076616C7524
:105F10006520696E76616C69642028302D36292EE3
:105F20000A0A003F2856296572626F7365206C6506
:105F300076656C20696D706C61757369626C652043
:105F400028302D34292E0A0A003F28522965706511
:105F5000746974696F6E20636F756E7420696E76F4
:105F6000616C69642028312B292E0A0A00446F696C
:105F70006E6720473239002A56255620561B565D3B
:105F80000A0062656420706C616E65206E6F726DD0
:105F9000616C203D205B00436F756C64206E6F74F4
:105FA00020636F6D706C657465204C53462100430F
:105FB0006F727265637465645F5A3D0025532025D6
:105FC000692F2569000A0A002F0054696C74696EF4
:105FD00067206D65736820706F696E7420003F459F
:105FE00072726F722070726F62696E6720706F6973
:105FF0006E742E2041626F7274696E67206F7065D7
:10600000726174696F6E2E0A00436F7272656374F9
:1060100065645F5A3D00255320332F330054696C6B
:1060200074696E67206D6573682028332F33290AE1
:1060300000436F727265637465645F5A3D00255357
:1060400020322F330054696C74696E67206D65735C
:10605000682028322F33290A00436F7272656374F7
:1060600065645F5A3D0054696C74696E6720506FB7
:10607000696E7400255320312F330054696C7469A4
:106080006E67206D6573682028312F33290A0064FC
:106090006F6E650A00496E73756666696369656E41
:1060A0007420646174610A000000803F6666724279
:1060B0006666F042CCCC334366666F4300809543FE
:1060C0000000803F666672426666F042CCCC334385
:1060D00066666F43008095434578747261706F6C9B
:1060E0006174696E67206D6573682E2E2E00212104
:1060F0002053544F502063616C6C6564206265636B
:1061000061757365206F6620424C546F756368201B
:106110006572726F72202D207265737461727420C3
:1061200077697468204D3939390A00212120535488
:106130004F502063616C6C656420626563617573A8
:1061400065206F6620424C546F75636820657272DB
:106150006F72202D20726573746172742077697478
:1061600068204D3939390A005072696E74696E675A
:10617000204F626A656374002553202569002F2F24
:10618000616374696F6E3A00737461727400707247
:106190006F6D70745F00656E6400486F74656E6447
:1061A00020746F6F20636F6C640A0053656E642007
:1061B0004D31303820746F20726573756D650A003B
:1061C000496E736572742066696C616D656E7420CA
:1061D000616E642073656E64204D3130380A005260
:1061E000656865617420446F6E650052656865611D
:1061F00074696E672E2E2E005265686561740048C2
:1062000065617465722054696D656F7574005365BE
:106210006E64204D31303820746F206865617420C1
:106220006E6F7A7A6C650A004E6F7A7A6C652050D0
:1062300061726B65640070617573656400506175AF
:10624000736500726573756D656400526573756D75
:10625000696E67004732362043616E63656C656422
:10626000004732362048656174696E67204E6F7A48
:106270007A6C65004732362048656174696E672024
:106280004265640057616974696E6720666F7220A9
:106290006865617475702E0A004669786564204CE3
:1062A000656E677468205072696D6500446F6E6535
:1062B000205072696D696E67004D616E75616C206A
:1062C0007072696D696E672E2E2E004C656176695D
:1062D0006E6720473236003F5370656369666965B3
:1062E0006420582C5920636F6F7264696E61746505
:1062F000206F7574206F6620626F756E64732E0A4E
:10630000003F28522965706561742076616C75655F
:10631000206E6F7420706C61757369626C653B20D0
:106320006D757374206265206174206C656173748F
:1063300020312E0A003F53706563696669656420E9
:106340006E6F7A7A6C652074656D706572617475B4
:106350007265206E6F7420706C61757369626C6514
:106360002E0A003F5370656369666965642066693B
:106370006C616D656E742073697A65206E6F742030
:10638000706C61757369626C652E0A003F537065AD
:10639000636966696564207072696D65206C656EFD
:1063A000677468206E6F7420706C61757369626CBD
:1063B000652E0A003F537065636966696564206EE7
:1063C0006F7A7A6C652073697A65206E6F742070BD
:1063D0006C61757369626C652E0A003F5265747258
:1063E000616374696F6E204D756C7469706C69655A
:1063F00072206D75737420626520737065636966C1
:106400006965642E0A003F53706563696669656457
:106410002052657472616374696F6E204D756C747F
:1064200069706C696572206E6F7420706C61757331
:1064300069626C652E0A003F537065636966696521
:1064400064206C6179657220686569676874206E84
:106450006F7420706C61757369626C652E0A0043FD
:10646000292E0A003F53706563696669656420627E
:1064700065642074656D7065726174757265206EF7
:106480006F7420706C61757369626C65202834309C
:106490002D00473236207374617274696E672E2E38
:1064A0002E0A0041425300504C41000A4D32340044
:1064B0004D3233202573002E0A006F70656E206602
:1064C00061696C65642C2046696C653A20004669F8
:1064D0006C652073656C65637465640A002053699C
:1064E0007A653A200046696C65206F70656E656458
:1064F0003A2000454E4420535542524F5554494E80
:10650000450A002220706F73002220706172656E50
:10651000743A2200535542524F5554494E45204338
:10652000414C4C207461726765743A220053756265
:1065300063616C6C204F766572666C6F770045788E
:10654000636565646564206D617820535542524FE0
:106550005554494E452064657074683A002E0A000F
:1065600044656C6574696F6E206661696C65642C46
:106570002046696C653A200046696C652064656C4C
:10658000657465643A005344207072696E74696E74
:1065900067206279746520004E6F74205344207028
:1065A00072696E74696E670A002F6175746F256376
:1065B0002E670057726974696E6720746F20666970
:1065C0006C653A2000667265736800646F696E6777
:1065D000002066696C653A20004E6F77200002FD4E
:1065E00055555555555FFFFFFFFFFFFFFFFFFFFEAE
:1065F00000000000003FFFFFFFFFFFFFFFFFFFFD68
:10660000000007FFFFFFFFFFFFFFFFFFFFFFFFFE91
:1066100007C00555555555555FFFFFFFFFFFFFFCB0
:106620000A200600000000003FFFFFFFFFFFFFFE03
:10663000141005000007FFFFFFFFFFFFFFFFFFFC37
:1066400028080607C00555555555555FFFFFFFFE45
:106650005404040A200600000000003FFFFFFFFC76
:10666000600406141005000007FFFFFFFFFFFFFE98
:1066700050040428080607C00555555555555FFCBC
:106680006004065404040A200600000000003FFED7
:1066900054041C60040614100500000000001FFCD8
:1066A00028082E50040428080607C00001F03FFE09
:1066B0001410546004065404040A200002081FFC4D
:1066C0000A206654041C60040614100005043FFEF2
:1066D00007C05428082E5004042808000A021FFC92
:1066E00000002E14105460040654040015013FFEEF
:1066F00000001C0A206654041C60040018011FFCE2
:1067000000000607C05428082E50040014013FFE64
:1067100000000400002E14105460040018011FFC37
:10672000FFFFFE00001C0A206654041C15013FFEFA
:10673000D5555400000607C05428082A0A021FFC39
:1067400084104600000400002E14105105043FFE82
:10675000C41044FFFFFE00001C0A206102881FFCD9
:10676000841046D5555400000607C05101F03FFE85
:1067700084104484104600000400002A00001FFC1E
:10678000C41046C41044FFFFFE00001C00003FFE82
:10679000841044841046D5555400000000001FFCAE
:1067A000D5555684104484104600000000003FFC7C
:1067B000FFFFFCC41046C41044FFFFFFFFFF9FFE15
:1067C000000006841044841046D555555555BFFD2C
:1067D000555554D5555684104484104104109FFFDC
:1067E000FFFFFCFFFFFCC41046C410410411BFFFB3
:1067F000FFFFFE00000684104484104104109FFF38
:10680000FFFFFD555554D5555684104104109FFF88
:10681000FFFFFFFFFFFCFFFFFCC410410411BFFF9F
:10682000FFFFFFFFFFFE00000684104104109FFFE2
:10683000FFFFFFFFFFFD555554D555555555BFFF7B
:10684000FFFFFFFFFFFFFFFFFCFFFFFFFFFF9FFFBB
:10685000FFFFFFFFFFFFFFFFFE00000000003FFF04
:10686000FFFFFFFFFFFFFFFFFD55555555555FFF2C
:10687000FFFFFFFFFFFFFFFFFFFFFFFFFFFFFFFF28
:10688000FFFFFFFFFFFFFFFFFFFFFFFFFFFFFFFF18
:10689000FFFFFFFFFFFFFFFFFFFFFFFFFFFFFFFF08
:1068A000FFFFFFFFFFFFFFFFFFFFFFFFFFFFFFE017
:1068B0002EFB7DFBFBCFC1DFBB3EC0E1FE3C1FFDDD
:1068C000EE7B39F9F3CF9EDFBB3EDFDEFCDDE7FD7B
:1068D000EE3BBBF9EBD7BF5FBB5EDFDEFDEDF7FD47
:1068E000EEBBD3FAEBB73FDFBB4EDFDFFFCDF3FDEF
:1068F000EEDBC7FAEBBB7FC03B6EC0E3FF1DF3FDD1
:10690000EECBEFFADBBB7FDFBB66DFF8FFCDF3FD3D
:10691000EEEBEFFB5B033F5FBB76DFFE7FEDF3FD4E
:10692000EEF3EFFB5B79BEDFBB7ADFDE7DEDF7FDDB
:10693000EEF3EFFBBAFD9EDFBB7CDFDEFDCDE7FDB6
:10694000EEFBEFFBBAFDC1DFBB7EC0E0FE1C1F6D9E
:1069500061726C696E66772E6F726700322E302E10
:10696000375F4457372E33001FFFFFFFFFFFFF60E5
:106970000000000001FF400000000000FF80000058
:106980000000007F83CF00000C303F87FF80000CA9
:10699000301F867980000C000F8C30C7838C30E765
:1069A0008C30CFC7CC31F38C30DCECEC33B98C308D
:1069B000D86C6C33198C30D06C0C33198C30D86C8B
:1069C0000C33198C30DC6C0E3B198C30CF7C079F5C
:1069D000198C30C77C038F19400000000000026052
:1069E0000000000000061FFFFFFFFFFFF870012CF2
:1069F0000190012701B0012201C0011D01F0011821
:106A0000011002130130020E01600209019002041C
:106A100001C002FF000003FA004003F5008003F00C
:106A200000D003EB002004E6007004E100E004DC89
:106A3000004005D700C005D2004006CD00D006C8F2
:106A4000008007C3003008BE00F008B900C009B4D8
:106A500000B00AAF00B00BAA00D00CA500000EA039
:106A600000500F9B00C01096005012910000148C33
:106A700000C0158700B0178200B0197D00D01B78C8
:106A800000001E730040206E0090226900F0246414
:106A90000040275F0090295A00E02B5500102E502F
:106AA0000020304B0010324600E033410090353C6E
:106AB000001037370070383200A0392D00B03A2866
:106AC00000A03B2300603C1E00103D1900903D14C7
:106AD00000103E0F00703E0A00C03E0500003F005F
:106AE00000403FFBFF803FF6FFC03FF1FF202050FA
:106AF0006C616E6E65724275666665724279746528
:106B0000733A20002046726565204D656D6F72797D
:106B10003A2000436F6D70696C65643A2041707271
:106B200020323420323032310A00204C617374201C
:106B3000557064617465643A20323032312D3034DE
:106B40002D3138207C20417574686F723A20546969
:106B50006E794D616368696E657333440A00322E45
:106B6000302E375F4457372E330A004D61726C69FF
:106B70006E0020536F66747761726520526573658D
:106B8000740A00205761746368646F6720526573EC
:106B900065740A002042726F776E206F7574205200
:106BA000657365740A002045787465726E616C20A7
:106BB00052657365740A00506F77657255700A00EC
:106BC00073746172740A004732385859004D31307D
:106BD0003031006572726F722077726974696E6706
:106BE00020746F2066696C650A00446F6E652073BF
:106BF0006176696E672066696C652E0A004D3239D0
:106C000000456E6473746F707300255320256320F4
:106C1000256320256320256300205A3A0020593A35
:106C20000020583A00656E6473746F707320686951
:106C3000743A200000000A0B02090C0D0E0807032D
:106C4000040100000000000000000000000000003F
:106C50000000000000000000000000000000000034
:106C600012111000000000000000000000000000F1
:106C700000000000000000000000004D6F7665205D
:106C800025736D6D004D6F766520302E316D6D0072
:106C90004D6F766520316D6D004D6F76652031301A
:106CA0006D6D004D6F76652041786973004578748D
:106CB0007275646572004D6F7665205A004D6F766F
:106CC000652059004D6F7665205800A764A3644382
:106CD00068616E67652046696C616D656E7400550C
:106CE0006E6C6F61642046696C616D656E74004CFA
:106CF0006F61642046696C616D656E7400507265E9
:106D00006865617420437573746F6D0050726568B7
:106D10006561742024004261636B0073686F7700C3
:106D2000627574746F6E00626567696E00446973A2
:106D300061626C6552756E6F75740050757267652F
:106D40004D6F72650050617573656400436F6E74BA
:106D5000696E7565004C6F61642046696C616D6594
:106D60006E74205400496E736572742066696C619C
:106D70006D656E7420616E642073656E64204D31A4
:106D800030380A00220A00556E6B6E6F776E2063F2
:106D90006F6D6D616E643A20220020420020500029
:106DA0006F6B00204500205A00205900204D3932D9
:106DB00020580020453A00205A3A0020593A0058FD
:106DC0003A0020746F6F206C6F6E67206578747264
:106DD0007573696F6E2070726576656E7465640A8E
:106DE0000020636F6C6420657874727573696F6ED0
:106DF0002070726576656E7465640A00526573650D
:106E00006E643A20006E6F74696669636174696FBD
:106E10006E200000002200250028002B002E0031EB
:106E200000340002010000050108010B01000021EF
:106E300000240027002A002D00300033000101004B
:106E400000040107010A01050505050705080808F2
:106E500008020202020A0A080804040404010101EB
:106E600001010101010303030303030303040707F3
:106E7000070C0C0C0C0C0C0C0C0202020206060691
:106E800006060606060B0B0B0B0B0B0B0B01021079
:106E90002020080810204010204080020102010834
:106EA00004020101020408102040808040201008E4
:106EB000040201800402018040201008040201083D
:106EC000040201010204081020408001020408109D
:106ED00020408000D9013D0211241FBECFEFD1E236
:106EE000DEBFCDBF00E00CBF17E0A0E0B2E0E2E4FF
:106EF000FEE803E00BBF02C007900D92AC31B10772
:106F0000D9F72CE1ACE1B7E001C01D92AF34B20774
:106F1000E1F717E3CBE6D7E300E006C021970109CC
:106F2000802FFE010F9424C2CA36D10780E00807E3
:106F3000A9F70F9412B00D940FC70C940000609144
:106F4000390270913A02072E000C880B990B0F94AE
:106F500042BB2AE037ED43E25CE30F94A1BB2091F2
:106F600013093091140940911509509116090F9495
:106F7000A1BB6093860270938702809388029093EE
:106F800089020895E091450CE23030F4F0E0E455D8
:106F9000F24F8091330C808308958091381A8823B2
:106FA000C1F081508093381AE4E6FAE1882351F069
:106FB0008150990B2BE1289FF001299FF00D11249E
:106FC000E656F54E8BE1AFE7BAE101900D928A9556
:106FD000E1F72091381A211105C08091431A80628F
:106FE0008093431A81E090E0A0E0B0E0211103C05B
:106FF00080E090E0DC0180932B0C90932C0CA0930C
:107000002D0CB0932E0C1092300C81E080932A0C42
:1070100083E080937A0208950E944F8D8DE69DE073
:107020009093D30B8093D20B0895CF93DF93EC0111
:10703000CB01BA010F9442BB29EC38EC48EC5EE37B
:107040000F9427C320E030E040E05FE30F942DC2AF
:107050000F94A0C36883DF91CF910895E091450C10
:1070600086E0E802F0011124EA5EF34F8091330CD0
:1070700090E09583848308958F929F92AF92BF9200
:10708000CF92DF92EF92FF92CF936B017C0120E0D1
:1070900030E0A9010F943BBB87FD9FC06DEB77E308
:1070A00086E095E3A70196010F942DC26B017C0148
:1070B00020E030E040E251E40F94A1BB20E030E05A
:1070C00048EC52E40F94A1BB4B015C0120E030E09E
:1070D000A901C701B6010F943BBB20E030E040EAB4
:1070E00050E487FF04C020E030E040EA50ECC501E6
:1070F000B4010F942DC220E030E040E251E40F943F
:1071000027C30F9499C36B017C018BE2F7FE09C082
:10711000F094E094D094C094C11CD11CE11CF11CEB
:107120008DE280933C0CC701B60120E137E240E0DC
:1071300050E00F94A1C18AE0882E912CA12CB12C93
:10714000CA01B901A50194010F94A1C1605D6093CA
:107150003D0CC701B60128EE33E040E050E00F944B
:10716000A1C1CA01B901A50194010F94A1C1605D3B
:1071700060933E0CC701B60124E630E040E050E0E9
:107180000F94A1C1CA01B901A50194010F94A1C135
:10719000605D60933F0C8EE28093400CC701B601A6
:1071A000A50194010F94A1C1C62FCA01B901A5017F
:1071B00094010F94A1C1605D6093410CC05DC093C8
:1071C000420C8CE39CE0CF91FF90EF90DF90CF904A
:1071D000BF90AF909F908F9008956DEB77E386E01E
:1071E00095EB60CF8F929F92AF92BF92CF92DF923A
:1071F000EF92FF926B017C0120E030E0A9010F9437
:107200003BBB87FD6BC06DEB77E386E095E3A701A1
:1072100096010F942DC26B017C0120E030E040E22A
:1072200051E40F94A1BB20E030E040E251E40F9420
:10723000A1BB4B015C0120E030E0A901C701B60110
:107240000F943BBB20E030E040EA50E487FF04C0ED
:1072500020E030E040EA50ECC501B4010F942DC2AB
:1072600020E030E040E251E40F9427C30F9499C32B
:107270009B018BE237FF05C022273327261B370BE4
:107280008DE280933E0CC90164E670E00F9410C259
:10729000CB01EAE0F0E0BF010F9410C2805D809363
:1072A0003F0CC901BF010F9410C2282FCB01BF01B1
:1072B0000F9410C2805D8093400C8EE28093410C4D
:1072C000205D2093420C8EE39CE0FF90EF90DF90D6
:1072D000CF90BF90AF909F908F9008956DEB77E324
:1072E00086E095EB94CF8F929F92AF92BF92CF9210
:1072F000DF92EF92FF92CF936B017C0120E030E0B0
:10730000A9010F943BBB87FDAAC06DEB77E386E034
:1073100095E3A70196010F942DC26B017C0120E03B
:1073200030E0A9010F943BBB87FF9EC0C701B601A7
:10733000905820E030E040E251E40F94A1BB20E0FF
:1073400030E040E251E40F94A1BB20E030E040EA9D
:1073500050E40F942DC220E030E040E251E40F945D
:1073600027C30F9499C36B017C0180E280933C0C8E
:1073700060E280E1C81687E2D806E104F1048CF0EF
:10738000C701B60120E137E240E050E00F94A1C10F
:10739000CA01B9012AE030E040E050E00F94A1C1F9
:1073A000605D60933D0C60E288EEC81683E0D8060D
:1073B000E104F1048CF0C701B60128EE33E040E0AF
:1073C00050E00F94A1C1CA01B9012AE030E040E0C9
:1073D00050E00F94A1C1605D60933E0C60E284E6D2
:1073E000C816D104E104F1048CF0C701B60124E60B
:1073F00030E040E050E00F94A1C1CA01B9012AE099
:1074000030E040E050E00F94A1C1605D60933F0C1C
:107410008AE0882E912CA12CB12CC701B601A501C0
:1074200094010F94A1C1C62FCA01B901A50194010D
:107430000F94A1C1605D6093400C8EE28093410C7B
:10744000C05DC093420C8CE39CE0CF91FF90EF9025
:10745000DF90CF90BF90AF909F908F9008956DEB8D
:1074600077E386E095EB55CF20E030E040E251E451
:10747000C701B60162CFCF93DF93EC01CB01BA0114
:107480000F9442BB20E030E040E251E40F9427C368
:1074900020E030E0A9010F942DC2688379838A83AC
:1074A0009B83DF91CF910895CF93DF93EC01CB01C4
:1074B000BA010F9442BB20E030E040E251E40F9467
:1074C00027C320E030E0A9010F942DC2688379839F
:1074D0008A839B83DF91CF9108950F9442BB20E074
:1074E00030E040E251E40F9427C320E030E0A901EE
:1074F0000F942DC20C947339CF93DF93EC01CB0121
:10750000BA010F9442BB20E030E040E251E40F9416
:1075100027C320E030E0A9010F942DC2688379834E
:107520008A839B83DF91CF9108950F9442BB20E023
:1075300030E040E251E40F9427C320E030E0A9019D
:107540000F942DC20C94F238CF93DF93EC01CB0152
:10755000BA010F9442BB2AE037ED43E25DE30F949A
:1075600027C320E030E0A9010F942DC20F94A0C3DF
:10757000688379838A839B83DF91CF910895CF932A
:10758000DF93EC01CB01BA010F9442BB2AE037ED47
:1075900043E25DE30F9427C320E030E0A9010F949C
:1075A0002DC2688379838A839B83DF91CF9108956D
:1075B000CF93DF93EC01CB01BA010F9442BB20E0E3
:1075C00030E0A9010F942DC2688379838A839B835D
:1075D000DF91CF910895CF93DF93EC01CB01BA01F6
:1075E0000F9442BB20E030E0A9010F942DC26883C4
:1075F00079838A839B83DF91CF910895CF93DF9323
:10760000EC01CB01BA010F9442BB20E030E048EC22
:1076100052E40F9427C320E030E0A9010F942DC25B
:10762000688379838A839B83DF91CF910895CF9379
:10763000DF93EC01CB01BA010F9442BB20E030E0B4
:1076400048EC52E40F9427C320E030E0A9010F94E6
:107650002DC2688379838A839B83DF91CF910895BC
:107660000F9442BB20E030E048EC52E40F9427C373
:1076700020E030E0A9010F942DC20C943C38CF9348
:10768000DF93EC01CB01BA010F9442BB20E030E064
:10769000A9010F942DC20F9499C379836883DF9158
:1076A000CF910895CF93DF93EC01CB01BA010F94F2
:1076B00042BB20E030E0A9010F942DC2688379839A
:1076C0008A839B83DF91CF910895CF93DF93EC0161
:1076D000CB01BA010F9442BB20E030E04AE754E40A
:1076E0000F9427C320E030E0A9010F942DC26883D6
:1076F00079838A839B83DF91CF9108952CEA35ECBF
:1077000047E25EE360911C0770911D0780911E07A0
:1077100090911F070F9427C360933E1970933F19F0
:10772000809340199093411908952CEA35EC47E273
:107730005EE360912007709121078091220790916C
:1077400023070F94A1BB60933A1970933B19809360
:107750003C1990933D1908950F9442BB20E030E00E
:10776000A9010F942DC20F9499C3CB010D94071951
:107770008091D1199091D219891B8F70B9F48091A1
:10778000CF0B8770873051F01092CF0B10921209F7
:1077900088E094E19093D30B8093D20B20E040E0FB
:1077A00070E060E084ED90E40C94CC8C089520E0CF
:1077B00040E070E060E089E19CE40C94CC8C809126
:1077C000BE0D811114C080918A0290918B020197A5
:1077D00020913119309132192817390744F420E0EB
:1077E00040E070E060E08EE19CE40C94CC8C0C9462
:1077F000D73B21E020933107FC0180819181A28158
:10780000B3818093110290931202A0931302B0935C
:10781000140220E040E070E060E08091260C90913E
:10782000270C0C94CC8CCF93DF9300D01F92CDB754
:10783000DEB78DEC9CECACECBCE389839A83AB8324
:10784000BC83CE0101960E94F93B0F900F900F90E0
:107850000F90DF91CF910895CF93DF9300D01F92C7
:10786000CDB7DEB78DEC9CECACECBDE389839A839D
:10787000AB83BC83CE0101960E94F93B0F900F9021
:107880000F900F90DF91CF910895CF93DF9300D0A9
:107890001F92CDB7DEB780E090E0A0E8BFE3898318
:1078A0009A83AB83BC83CE0101960E94F93B0F9073
:1078B0000F900F900F90DF91CF910895CF93DF93AA
:1078C00000D01F92CDB7DEB780E090E0A0E2B1E437
:1078D00089839A83AB83BC83CE0101960E94F93BD6
:1078E0000F900F900F900F90DF91CF9108958FEF31
:1078F0008093330C20E040E070E060E081E99FE796
:107900000C94CC8C8F929F92AF92BF92CF92DF92C9
:10791000EF92FF920F931F93CF93DF9361E081E08B
:107920000E946E8CC091300C85E0982E9C0E9FE1D9
:10793000E92E94E1F92ED3E0DC1B25E3C22E24E1ED
:10794000D22E12E01C1B3BE4A32E34E1B32E01E047
:107950000C1B8C2E8194C11133C080912F0C882375
:10796000B1F080917A02882359F081E090912F0C38
:10797000911180E024E045E455E1682D0F943297A1
:10798000CF5FC911E8CF84E08093290C0CC08091AF
:10799000280C1092280C882321F30E94B48D80912A
:1079A0002A0C8823F1F2DF91CF911F910F91FF9064
:1079B000EF90DF90CF90BF90AF909F908F90089501
:1079C000C13001F590912F0C913069F080917A02CD
:1079D0008823B1F281E0913009F080E020E24BE3AE
:1079E00054E1602FCBCF8091280C1092280C882373
:1079F00069F3B092D30BA092D20B80912A0C88230A
:107A000029F3D1CFC23081F590912F0C923071F0D3
:107A100080917A02882309F4B3CF81E0923009F093
:107A200080E020E246E254E1612FA8CF8091280C4B
:107A30001092280C882361F3D092D30BC092D20B02
:107A400080912A0C882321F3AECF8091280C1092CC
:107A5000280C882381F0F092D30BE092D20B809116
:107A60002A0C882341F09FCFC33009F089CF909131
:107A70002F0C933051F380917A02882309F480CF40
:107A800081E0933009F080E020E24CE054E16D2F7A
:107A900075CF3F924F925F926F927F928F929F929B
:107AA000AF92BF92CF92DF92EF92FF920F931F930C
:107AB000CF93DF9361E081E00E946E8CC091300C27
:107AC00085E0482E4C0E9FE4E92E9DE8F92E26EA2B
:107AD000C22E22E1D22ED4E0DC1B35E6A32E32E109
:107AE000B32E83E0782E7C1A4CE7842E42E1942E4C
:107AF00082E0682E6C1A81E0582E5C1A3C2E31947C
:107B0000C11133C080912F0C882389F080917A02B3
:107B1000882309F448C081E090912F0C911180E0F6
:107B200024E04CE954E1632D0F9432973CC08091DE
:107B3000280C1092280C882349F30E94B48D809160
:107B40002A0C882319F3DF91CF911F910F91FF9099
:107B5000EF90DF90CF90BF90AF909F908F907F90ED
:107B60006F905F904F903F900895C130D1F5809114
:107B70002F0C8130F9F080917A028823A1F011E076
:107B800080912F0C813009F010E080910E029091CD
:107B90000F020F94071900E09C0144E852E1652DA3
:107BA000812F0E94F49ACF5FC411AACF85E0809301
:107BB000290CC9CF8091280C1092280C8823D9F267
:107BC00006E013E429E030E050E040E06EE072E0CF
:107BD00084E892E10F94059A80912A0C882359F247
:107BE000B2CFC23009F04EC090912F0C923069F0A4
:107BF00080917A028823B9F281E0923009F080E026
:107C000020E24EE652E1662D8FCF8091280C109233
:107C1000280C882369F39092D30B8092D20B809129
:107C20002A0C882329F38FCF90912F0C933071F079
:107C300080917A02882309F4B6CF81E0933009F06D
:107C400080E020E246E552E1672D6ECF8091280C5E
:107C50001092280C882361F3B092D30BA092D20B20
:107C600080912A0C882321F36ECF8091280C1092EA
:107C7000280C882381F00E944F8D80912A0C882344
:107C800051F061CFC33081F2C43009F08CCF8091C4
:107C90002F0C843051F380917A02882309F483CF2A
:107CA000FF92EF92DF92CF92DF9381E090912F0CC1
:107CB000943009F080E08F930E94388C0F900F90E1
:107CC0000F900F900F900F906ECF9F92AF92BF9238
:107CD000CF92DF92EF92FF920F931F93CF93DF9398
:107CE00061E081E00E946E8CC091300C85E0E82E4E
:107CF000EC0E9FE4C92E9DE8D92E26EAA22E22E1A1
:107D0000B22ED2E0DC1B81E0F82EFC1A9C2E91945E
:107D1000C11132C080912F0C8823B1F080917A027A
:107D2000882359F081E090912F0C911180E024E09C
:107D30004FE554E1692D0F943297CF5FCE11E8CF14
:107D400083E08093290C0CC08091280C1092280CA1
:107D5000882321F30E94B48D80912A0C8823F1F2AC
:107D6000DF91CF911F910F91FF90EF90DF90CF9017
:107D7000BF90AF909F900895C130A1F580912F0CD6
:107D80008130C9F080917A028823B9F211E08091A4
:107D90002F0C813009F010E08091060290910702CB
:107DA0000F94071900E09C0141E651E16F2D812FEE
:107DB0000E94F49AC2CF8091280C1092280C88233C
:107DC00009F30DE418E429E030E047EF5FEF66E0E7
:107DD00072E081E691E10F94059A80912A0C882344
:107DE00089F2BECFC23009F0A8CF80912F0C82302B
:107DF000D1F080917A02882309F49FCFDF92CF924D
:107E0000BF92AF92DF9381E090912F0C923009F0F6
:107E100080E08F930E94388C0F900F900F900F90FE
:107E20000F900F908ACF8091280C1092280C8823F5
:107E300001F30E944F8D80912A0C8823D1F290CFBC
:107E40005F926F927F928F929F92AF92BF92CF92EA
:107E5000DF92EF92FF920F931F93CF93DF9361E036
:107E600081E00E946E8CC091300C85E0982E9C0EB3
:107E7000D1E093EAE92E9AE0F92E882483947D2EAE
:107E80007C1A6C2E619425E8C22E2AE0D22E12E0D4
:107E90001C1B33E0532E45EEA42E40E0B42EC1113E
:107EA00041C0DD23D9F080912F0C1816BCF0409111
:107EB0002B0C50912C0C60912D0C70912E0C4F5F5F
:107EC0005F4F6F4F7F4F40932B0C50932C0C609360
:107ED0002D0C70932E0C8F5F80932F0C80917A0263
:107EE000882341F030E020E041E06EEA7AE0862D20
:107EF0000E94BF9880916E0C882309F487C0C2301D
:107F000051F480912F0C823009F445C080917A029F
:107F100081115AC0D0E0CF5F9C12C1CF83E0809323
:107F2000290C18C0C13031F790912F0C913031F0ED
:107F300080917A0281111EC0D0E0DCCF8091280CA4
:107F40001092280C8823A1F3C0936F0C80912A0C07
:107F5000882371F3DF91CF911F910F91FF90EF90E4
:107F6000DF90CF90BF90AF909F908F907F906F9059
:107F70005F9008951F92FF92EF927F9281E091307F
:107F800009F080E08F930E94388C0F900F900F9033
:107F90000F900F90D1CF8091280C1092280C88233D
:107FA00009F4B4CF809159028825809359025092E8
:107FB0007A02A114B10411F00F94523180912A0C6D
:107FC000882309F4A3CFC6CF81E090912F0C923083
:107FD00009F080E09091590222E93AE0911102C043
:107FE0002EE83AE001E045E95AE0612F0E94F49A58
:107FF00091CF8091280C1092280C882371F0C093A7
:108000006F0C80912A0C882341F0A4CFC23009F074
:1080100082CF90912F0C923061F380917A02882365
:1080200009F478CF1F92DF92CF921F9381E09230B4
:1080300009F080E08F930E94388C0F900F900F9082
:108040000F900F9067CF62E57BE38CEB94E60C9486
:10805000589A65E178E38BE199E40C94589A64E5C9
:108060007AE38DE69AE30C94589A6CE77AE385E913
:108070009AE30C94589A64EA7AE38FEB98E50C94AF
:10808000589A6FEB7AE381E099E50C94589A6BEE7D
:108090007AE380E199E50C94589A67E17BE380E309
:1080A0009BE30C94589A6BE37AE386E69FE40C9486
:1080B000589A6EEF7AE389E199E50C94589A6FE348
:1080C0007BE38CEA9BE30C94589A68ED7AE384EEA8
:1080D00092E80C94589A65E67BE380E293E80C946E
:1080E000589A61E083E39CE00D9497418F929F92B0
:1080F000AF92BF92CF92DF92EF92FF92CF93DF9336
:1081000000D000D01F921F92CDB7DEB780913C0700
:108110000F94023B4B015C0189829A82AB82BC8244
:1081200080913D070F946C3A6B017C01CD82DE8219
:10813000EF82F886CE0101960F947640882319F1DC
:108140008092730D9092740DA092750DB092760D81
:10815000C092770DD092780DE092790DF0927A0D61
:108160008EEF28960FB6F894DEBF0FBECDBFDF911D
:10817000CF91FF90EF90DF90CF90BF90AF909F9006
:108180008F900C94CF8F28960FB6F894DEBF0FBE59
:10819000CDBFDF91CF91FF90EF90DF90CF90BF9058
:1081A000AF909F908F90089581E0809331078091E8
:1081B0007A02882341F030E020E041E06DEF73E186
:1081C00082E00E94BF98809112098770873049F53C
:1081D00081E08093300780913D0760913C0770E01B
:1081E00096E0899F600D711D112420E040E082E13E
:1081F00091E40E94CC8C1092110210921202109203
:108200001302109214020E94764080E090E0A0E8F1
:10821000BFE38093110290931202A0931302B093D4
:10822000140208953F924F925F926F927F928F92C5
:108230009F92AF92BF92CF92DF92EF92FF920F93F5
:108240001F93CF93DF93CDB7DEB7C654D1090FB6D6
:10825000F894DEBF0FBECDBF80912F07882309F4AD
:10826000A0C08091280C1092280C882309F450C0DB
:1082700080913C070F94023B7E012DE3E20EF11C3E
:10828000870122E040E00F94CBB580913D070F9429
:108290006C3A5E01E3E3AE0EB11C850122E040E0E2
:1082A0000F94CBB5809110021F928F93BF92AF9223
:1082B000FF92EF9281EE93E19F938F931F9282E35F
:1082C0008F93025311091F930F930F9495BAC8010E
:1082D0000E94468C0FB6F894DEBF0FBECDBFCA5BBE
:1082E000DF4F0FB6F894DEBF0FBECDBFDF91CF9149
:1082F0001F910F91FF90EF90DF90CF90BF90AF90C4
:108300009F908F907F906F905F904F903F900895D7
:1083100081E08093310780912B0C90912C0CA091DF
:108320002D0CB0912E0CB7FF0CC083E290E0A0E0C2
:10833000B0E080932B0C90932C0CA0932D0CB09359
:108340002E0C80912B0C90912C0CA0912D0CB091A7
:108350002E0C8497A105B10544F010922B0C1092BD
:108360002C0C10922D0C10922E0C60912B0C7091F5
:108370002C0C80912D0C90912E0C26E030E040E0EA
:1083800050E00F947FC161502150243028F489E0DF
:10839000643028F086E003C084E06430D8F3809332
:1083A000100260912B0C70912C0C80912D0C9091EF
:1083B0002E0C26E030E040E050E00F947FC1322EDA
:1083C0004B0180917A02882309F400C18091311A0F
:1083D0008A3308F58091331A8930E8F081E0809380
:1083E0001D1A0EE224E349E063E28DEF99E10F9458
:1083F00069A58091311A863370F48091331A8B30DD
:1084000050F010921D1A0AE220E34BE065E28DEF76
:1084100099E10F9469A581E080931D1A1EE0809177
:10842000311A181798F08091331A811778F099E271
:10843000E92E01E021E0412F6E2D8DEF99E10F949F
:1084400069A598E0E90EE9E5EE12F3CF195F18335C
:1084500031F745E0431987E0489F402D1124455FDF
:10846000842F90E007962091311A2817190609F0F9
:108470007CF48091331A841758F0682D660F660FCC
:10848000660F6B5D07E028E08DEF99E10F9469A519
:1084900081E080931D1A8091311A883008F047C01E
:1084A000882D0F94023B6B017C01832D0F946C3A55
:1084B00020916B0D30916C0D40916D0D50916E0DB2
:1084C0000F942DC22B013C01A70196016091670D0D
:1084D0007091680D8091690D90916A0D0F942DC275
:1084E00069837A838B839C834D825E826F827886D8
:1084F00085E08093341A17E01093351A8FEB9DE6D0
:108500000E947E95CE0101960F94EF160E94469927
:108510008AE48093341A1093351A8AEF93E10E940B
:108520007E95CE0105960F94EF160E944699809194
:10853000311A813408F04AC08091331A873308F425
:1085400045C085E08093341A10E41093351A68E230
:1085500070E080E090E00E94AE92882D0F940E981B
:108560006CE270E080E090E00E94AE92832D0F9468
:108570000E9869E270E080E090E00E94AE928AE49A
:108580008093341A1093351A87EF93E10E947E95F9
:1085900086E0889D8001899D100D1124030D111D19
:1085A000000F111F000F111F005E164FF8016081B0
:1085B0007181828193819B01AC010F947AC58111F5
:1085C00020C0C8010F9473970E94469980913C0780
:1085D000082E000C990B8815990549F480913D07E8
:1085E000082E000C990B3816190609F478CE8092E3
:1085F0003C0730923D070E94764082E080937A02E9
:108600006ECE80EF93E10E947E95E0CF0F931F9393
:10861000CF93DF93CDB7DEB762970FB6F894DEBF86
:108620000FBECDBF80910F028F9380910E028F936A
:108630008BE492E19F938F938E010F5F1F4F1F93E7
:108640000F930F94D2BAC8010E9486CF0F900F905B
:108650000F900F900F900F9062960FB6F894DEBFB8
:108660000FBECDBFDF91CF911F910F9108955F9203
:108670006F927F928F929F92AF92BF92CF92DF9232
:10868000EF92FF920F931F93CF93DF93CDB7DEB797
:108690002C970FB6F894DEBF0FBECDBF61E081E02E
:1086A0000E946E8CF090300C85E0C82ECF0C93E0C9
:1086B000A92E92E1B92ECE0101964C012AE0622E3C
:1086C00022E1722E82E0E82EEF1881E0D82EDF182A
:1086D0005F2C5194F1103CC080912F0C8823B1F095
:1086E00080917A02882359F081E090912F0C9111AA
:1086F00080E024E04BE755E1652D0F943297F39429
:10870000FC10E8CF83E08093290C0CC08091280CEA
:108710001092280C882321F30E94B48D80912A0C9A
:108720008823F1F22C960FB6F894DEBF0FBECDBFB2
:10873000DF91CF911F910F91FF90EF90DF90CF903D
:10874000BF90AF909F908F907F906F905F900895B3
:1087500091E0F91234C080912F0C8130C9F08091E2
:108760007A02882361F211E080912F0C813009F0A8
:1087700010E080910C0290910D020F94071900E017
:108780009C0145E152E16D2D812F0E94F49AB7CFF3
:108790008091280C1092280C882309F310E000E047
:1087A00026E030E042E050E06CE072E085E192E1EA
:1087B0000F94059A80912A0C882389F2B3CF82E026
:1087C000F8129DCF80912F0C8230C1F080917A02F7
:1087D000882309F494CF1F927F926F92EF9281E0E9
:1087E00090912F0C923009F080E08F930E94388C8A
:1087F0000F900F900F900F900F9081CF8091280CC9
:108800001092280C882311F380910D028F93809190
:108810000C028F93BF92AF929F928F920F94D2BA15
:10882000C4010E94468C0F900F900F900F900F90F4
:108830000F9080912A0C882349F274CF0F931F93D5
:10884000CF93DF93CDB7DEB764970FB6F894DEBF52
:108850000FBECDBF80910B028F9380910A028F9340
:10886000809109028F93809108028F9384EB91E1AC
:108870009F938F938E010F5F1F4F1F930F930F9442
:10888000D2BAC8010E94468C0FB6F894DEBF0FBE64
:10889000CDBF64960FB6F894DEBF0FBECDBFDF919B
:1088A000CF911F910F9108952F923F924F925F9217
:1088B0006F927F928F929F92AF92BF92CF92DF92F0
:1088C000EF92FF920F931F93CF93DF9361E081E0CC
:1088D0000E946E8CC091300C3C2E85E0482E4C0ED0
:1088E0000FE41DE896EAE92E92E1F92ED4E0DC1BB4
:1088F000552453942EE1C22E24E4D22E34ECA32E20
:1089000031E1B32E83E0782E7C1A4DEC842E4CE6B8
:10891000942E82E0682E6C1A252C2C1AC1113AC0B4
:1089200080912F0C8823B9F080917A02882361F01E
:10893000632D619581E090912F0C911180E024E0EE
:108940004BE755E10F943297CF5FC411E7CF85E035
:108950008093290C0CC08091280C1092280C88233D
:1089600019F30E94B48D80912A0C8823E9F2DF91DB
:10897000CF911F910F91FF90EF90DF90CF90BF901C
:10898000AF909F908F907F906F905F904F903F90AF
:108990002F900895C13061F5EBECFCE68591949140
:1089A0001092450C9093470C8093460C90912F0C9D
:1089B000913069F080917A02882331F281E0913020
:1089C00009F080E020E245EE51E1622DBBCF8091BD
:1089D000280C1092280C882369F327EF31E130939B
:1089E000D30B2093D20B80912A0C882319F3BFCF8D
:1089F000C23009F05BC0F401859194915092450C0E
:108A00009093470C8093460C90912F0C923071F00C
:108A100080917A02882309F497CF81E0923009F09F
:108A200080E020E245EE51E1662D8CCF8091280C4C
:108A30001092280C882361F329ED31E13093D30B98
:108A40002093D20B80912A0C882311F390CF809130
:108A50002F0C833089F080917A02882309F474CF37
:108A6000DF92CF92BF92AF927F9281E090912F0CD4
:108A70009330A1F180E032C08091280C1092280C34
:108A8000882349F30E941E4480912A0C882319F3FD
:108A90006ECF8091280C1092280C882381F00E94C0
:108AA0004F8D80912A0C882351F061CFC33079F229
:108AB000C43009F049CF80912F0C843051F380915C
:108AC0007A02882309F440CF1F930F93FF92EF920D
:108AD000DF9381E090912F0C943061F68F930E9488
:108AE000388C0F900F900F900F900F900F902CCF0D
:108AF0000F931F93CF93DF93CDB7DEB7C054D10947
:108B00000FB6F894DEBF0FBECDBF809109028F93E0
:108B1000809108028F9380910B028F9380910A02BB
:108B20008F9383E291E19F938F938E010F5F1F4F8D
:108B30001F930F930F94D2BAC8010E94468C0FB6B0
:108B4000F894DEBF0FBECDBFC05CDF4F0FB6F89408
:108B5000DEBF0FBECDBFDF91CF911F910F91089562
:108B60008F929F92AF92BF92CF92DF92EF92FF923D
:108B70000F931F93CF93DF9361E081E00E946E8C8F
:108B8000C091300C85E0982E9C0E98E7C92E95E494
:108B9000D92E26E1A22E23E1B22ED3E0DC1B82E007
:108BA000F82EFC1A81E0E82EEC1A8C2E8194C1116B
:108BB00033C080912F0C8823B1F080917A028823F2
:108BC00059F081E090912F0C911180E024E04CE964
:108BD00054E1682D0F943297CF5FC911E8CF84E03C
:108BE0008093290C0CC08091280C1092280C8823AB
:108BF00021F30E94B48D80912A0C8823F1F2DF9139
:108C0000CF911F910F91FF90EF90DF90CF90BF9089
:108C1000AF909F908F900895C130A1F580912F0C57
:108C20008130C9F080917A028823B1F211E08091FD
:108C30002F0C813009F010E0809108029091090218
:108C40000F94071900E09C0149E451E16E2D812F3A
:108C50000E94F49AC1CF8091280C1092280C88238E
:108C600009F310E000E02CE231E04AEA50E068E06D
:108C700072E089E491E10F94059A80912A0C88238F
:108C800089F2BDCFC23009F03FC080912F0C8230F5
:108C9000B9F080917A02882309F49ECF11E0809187
:108CA0002F0C823009F010E080910A0290910B02A3
:108CB0000F94071900E09C0140E451E16F2DC7CFEC
:108CC0008091280C1092280C882319F310E000E002
:108CD0002CE830E045E050E06AE072E080E491E1A9
:108CE0000F94059A80912A0C882399F288CF80915D
:108CF000280C1092280C882371F00E9478458091EE
:108D00002A0C882341F07BCFC33009F065CF8091D6
:108D10002F0C833061F380917A02882309F45CCFB1
:108D2000DF92CF92BF92AF92DF9381E090912F0CB0
:108D3000933009F080E08F930E94388C0F900F9051
:108D40000F900F900F900F9047CFEF92FF920F93DD
:108D50001F93CF93DF93CDB7DEB7A8970FB6F894E4
:108D6000DEBF0FBECDBFF62EE72E90913B079F933F
:108D700090913A079F93282F082E000C330B3F93B6
:108D80008F9383E893E19F938F938E010F5F1F4F23
:108D90001F930F930F94D2BAF80101900020E9F7C6
:108DA000CF0120913B072F9320913A072F93EF9209
:108DB000FF9201979F938F930F94D2BAC8010E949C
:108DC00086CF0FB6F894DEBF0FBECDBFA8960FB604
:108DD000F894DEBF0FBECDBFDF91CF911F910F91F1
:108DE000FF90EF90089560EA73E183E50C94A54647
:108DF00061E973E18CE40C94A5462F923F924F9267
:108E00005F926F927F928F929F92AF92BF92CF921A
:108E1000DF92EF92FF920F931F93CF93DF9300D0D7
:108E20001F92CDB7DEB70E9465E69C838B8361E01D
:108E300081E00E946E8C5090300C25E0250D298336
:108E400011E0352D31953A83212E251883EF682EB8
:108E500086E4782E9EEAE92E93E1F92E83E0482EEF
:108E6000451828EFC22E26E4D22E3CEBA32E33E188
:108E7000B32E82E0382E35188B809C8081E0881AD2
:108E8000910851100AC080912F0C882309F445C025
:108E900080917A02811166C010E080913A0790912A
:108EA0003B0797FD06C02B813C81821793070CF48A
:108EB00065C031E0531229C01123D9F080912F0CE5
:108EC0008230BCF440912B0C50912C0C60912D0CF5
:108ED00070912E0C4F5F5F4F6F4F7F4F40932B0C65
:108EE00050932C0C60932D0C70932E0C8F5F8093FD
:108EF0002F0C80917A02882341F030E020E041E09D
:108F000066ED73E1822D0E94BF9882E0539439810F
:108F10003511B7CF8093290C0EC08091280C109288
:108F2000280C882309F4B4CF0E94B48D80912A0CB8
:108F3000882309F4ADCF0F900F900F900F90DF9121
:108F4000CF911F910F91FF90EF90DF90CF90BF9046
:108F5000AF909F908F907F906F905F904F903F90D9
:108F60002F90089581E090912F0C911180E024E0E2
:108F700045E455E16A810F9432978ECF81E0581213
:108F800035C080912F0C8130D9F080917A028823EE
:108F9000A1F011E080912F0C813009F010E0809158
:108FA0003A0790913B070F94071900E09C014AECA7
:108FB00053E1622D812F0E94F49A10E084E0A6CF45
:108FC0008091280C1092280C8823F9F210E000E020
:108FD000940150E040E06AE377E08AEC93E10F947B
:108FE000059A80912A0C882381F2A5CF92E059122C
:108FF00021C080912F0C823081F080917A028823E9
:10900000E1F2DF92CF92BF92AF923F9281E09091D6
:109010002F0C923029F180E023C08091280C10920F
:10902000280C882351F30E94F84680912A0C88234B
:1090300021F381CF23E05212C1CF80912F0C8330D6
:10904000C9F080917A02882309F4B7CF7F926F929A
:10905000FF92EF924F9281E090912F0C9330D9F6CE
:109060008F930E94388C0F900F900F900F900F905D
:109070000F90A3CF8091280C1092280C882309F31D
:109080000E94F34680912A0C8823D9F254CF0F9482
:10909000644183E992E10D9422460F931F93CF938D
:1090A000DF93CDB7DEB72D970FB6F894DEBF0FBEB6
:1090B000CDBF809106029091070207E010E01816DC
:1090C000190614F406E010E069E571E1CE0101969D
:1090D0000F9444BA809106029091070297FF03C053
:1090E0009195819591099F938F9385E591E19F9348
:1090F0008F9381E090E08C0F9D1F080F191F1F9325
:109100000F930F94D2BACE0101960E94468C0F9015
:109110000F900F900F900F900F902D960FB6F89420
:10912000DEBF0FBECDBFDF91CF911F910F9108958C
:10913000CF92DF92EF92FF92CF93DF9300D01F92F6
:10914000CDB7DEB781E08093310780912D079091F4
:109150002E07892B41F180912D0790912E072AE04F
:1091600037ED43EA5BEB1816190624F42AE037EDD5
:1091700043EA5BE3609136077091370780913807C7
:10918000909139070F942DC260933607709337077B
:10919000809338079093390710922E0710922D076D
:1091A00082E080937A0280917A028823C9F120E0DC
:1091B00030E04AE754E460913607709137078091B8
:1091C0003807909139070F94A1BB0F9499C36B0195
:1091D0007C0125E030E040E050E00F94A1C1A70100
:1091E0009601261B370B480B590BCA01B9010F9486
:1091F00042BB20E030E04AE754E40F9427C3698380
:109200007A838B839C83CE0101960F947397BC0164
:109210008BE191E10E944A99CE0101960E943F9113
:109220000F900F900F900F90DF91CF91FF90EF90E4
:10923000DF90CF9008950F9442BB29EC38EC48ECB6
:109240005EE30F9427C320E030E040E05FE30F943B
:109250002DC20F94A0C3862F0D943C192F923F92DC
:109260004F925F926F927F928F929F92AF92BF9236
:10927000CF92DF92EF92FF920F931F93CF93DF93E2
:1092800000D000D01F921F92CDB7DEB72091450CC1
:10929000288761E081E00E946E8C3091300C3F8322
:1092A000E8858E2F90E0880F991F9C012553334944
:1092B0003C832B8336E0E39FC0011124FC01E85E70
:1092C000F34FFA83E9839C012A5E334F79015F8073
:1092D00035E0432E450C11E0312E3518252C219414
:1092E000FE82ED82570134E0A30EB11C42E6C42E8B
:1092F0004CE8D42E85E0782E75184701E2E08E0EFA
:10930000911C82E0682E6518FF81F1115BC011236A
:10931000D9F080912F0C1816BCF040912B0C509175
:109320002C0C60912D0C70912E0C4F5F5F4F6F4F86
:109330007F4F40932B0C50932C0C60932D0C70930B
:109340002E0C8F5F80932F0C80917A02882351F02E
:10935000EB81FC816591749130E020E043E0822D47
:109360000E94BF98F50180818093330CFF81F23019
:1093700009F07AC028852093450C80912F0C82300B
:1093800009F45FC080917A02882391F011E0809106
:109390002F0C823009F010E08091330C0F943C19AF
:1093A00000E09C0142EA59E0662D812F0E94F49A68
:1093B00010E02F812F5F2F832411A6CF86E08093AA
:1093C000290C19C02F81213069F680912F0C813032
:1093D00031F080917A02811127C010E0C3CF8091D3
:1093E000280C1092280C8823A1F30E94B48D809140
:1093F0002A0C882371F328960FB6F894DEBF0FBEAF
:10940000CDBFDF91CF911F910F91FF90EF90DF9033
:10941000CF90BF90AF909F908F907F906F905F9014
:109420004F903F902F90089581E090912F0C9130B4
:1094300009F080E024E04CEA59E0632D0F94329764
:10944000CCCF8091280C1092280C882309F49ACF55
:109450006EE278E382EA99E00F94FE9A80912A0CFA
:10946000882309F48FCFC7CF3F81333091F58091A6
:109470002F0C8330C1F080917A02882309F498CFB1
:1094800011E080912F0C833009F010E0ED81FE8116
:10949000808191810F94071963E0651900E09C01B8
:1094A0004BE959E082CF8091280C1092280C882338
:1094B00011F310E000E02CE231E045E050E0B701AC
:1094C0008BE999E00F94059A80912A0C882399F2F0
:1094D00092CFFF81F43091F580912F0C8430B9F058
:1094E00080917A02882309F463CF11E080912F0CD8
:1094F000843009F010E0F401808191810F94071904
:1095000064E0651900E09C0147E959E04ECF809185
:10951000280C1092280C882319F310E000E02CE8A6
:1095200030E045E050E069817A8187E999E00F9465
:10953000059A80912A0C882399F25DCFFF81F5303E
:1095400009F037CF80912F0C8530E1F080917A02BD
:10955000882309F42DCFDF92CF9289ED99E09F9374
:109560008F937F9281E090912F0C953009F080E0ED
:109570008F930E94388C0F900F900F900F900F9048
:109580000F9016CF8091280C1092280C8823F1F2AE
:109590000E94628C80912A0C8823C1F22CCF0D94FA
:1095A000549E0D94549E0F9453430E94E6E20C94F3
:1095B0004F8D6FEF8091330C0D94729C4F925F92A0
:1095C0006F927F928F929F92AF92BF92CF92DF92D3
:1095D000EF92FF920F931F93CF93DF930091330C81
:1095E00061E081E00E946E8CC091300C10E0000FB1
:1095F000111F0553134995E0592E5C0E2CE9E22EFC
:1096000020E1F22ED3E0DC1B39EDC32E3AE4D32E59
:109610004EE8A42E40E1B42E82E0782E7C1A5FEB57
:10962000852E50E1952E81E0682E6C1A4C2E4194C7
:10963000C11137C080912F0C8823B1F080917A023C
:10964000882359F081E090912F0C911180E024E063
:109650004AEA50E1642D0F943297CF5F5C12E8CF55
:1096600084E08093290C0CC08091280C1092280C67
:10967000882321F30E94B48D80912A0C8823F1F273
:10968000DF91CF911F910F91FF90EF90DF90CF90DE
:10969000BF90AF909F908F907F906F905F904F9012
:1096A0000895C13059F5F801859194919093470C34
:1096B0008093460C80912F0C813081F080917A024A
:1096C000882359F21F929F928F926F9281E090911E
:1096D0002F0C913009F474C080E072C08091280C86
:1096E0001092280C882351F38091330C682F0F942B
:1096F000729C80912A0C882309F3C2CFC23009F0F2
:1097000042C0F801859194919093470C8093460C48
:1097100080912F0C8230D1F080917A02882309F455
:109720009CCFDF92CF92BF92AF927F9281E09091D7
:109730002F0C923009F080E08F930E94388C0F90AC
:109740000F900F900F900F900F9087CF8091280C63
:109750001092280C882301F30E94D94A80912A0C88
:109760008823D1F28DCF8091280C1092280C882369
:10977000C1F06091330C8FEF0F94729C80912A0C92
:10978000882379F07DCFC33009F067CFF801859148
:1097900094919093470C8093460C80912F0C8330CA
:1097A00011F380917A02882309F457CF1F92FF9218
:1097B000EF92DF9381E090912F0C933009F08CCFE2
:1097C0008F930E94388C0F900F900F900F900F90F6
:1097D00044CF81E0809331078091CF0B8770873031
:1097E00051F01092CF0B1092120988E094E19093FF
:1097F000D30B8093D20B8091820C8093330780E04F
:109800000F94384120E040E070E060E085E898E5A2
:109810000C94CC8C64E27FE482E00D946DAC69E240
:109820007FE481E00D946DAC6EE27FE480E00D9406
:109830006DAC6BED7CE483E00D946DACCF92DF9268
:10984000EF92FF920F931F938CECC82E8FE0D82ECF
:10985000F12CE12C0EEC1FE025E432E047ED5BE358
:109860006EED7FE083EE9FE00E94EF931F910F91DA
:10987000FF90EF90DF90CF900895CF92DF92EF921C
:10988000FF920F931F938FEBC82E8EE0D82EF12CF2
:10989000E12C0FE61FE025E432E040E05FE861ECF8
:1098A0007EE086EC9EE00E94EF931F910F91FF9067
:1098B000EF90DF90CF900895CF92DF92EF92FF92DA
:1098C0000F931F93CF93DF9300D01F92CDB7DEB7D6
:1098D0002091450C1C821B8280E2898380E22A3021
:1098E0002CF0822F6AE00F94EEC1805D8A83822F74
:1098F0006AE00F94EEC1905D9B8387E4C82E89E0F7
:10990000D82ECE0101967C0109E419E025E432E06D
:1099100047EE57E567E579E08AE599E00E94EF9325
:109920000F900F900F900F90DF91CF911F910F919B
:10993000FF90EF90DF90CF900895CF92DF92EF925B
:10994000FF920F931F9380E3C82E89E0D82EF12C4D
:10995000E12C02E319E021EF37E549E058E56DE33A
:1099600079E082E499E00E94EF931F910F91FF90BC
:10997000EF90DF90CF900895CF92DF92EF92FF9219
:109980000F931F9385EAC82E88E0D82EF12CE12C86
:1099900008EB18E030E020E048E95DE867EA78E0AD
:1099A0008EEA98E00E94EF931F910F91FF90EF9045
:1099B000DF90CF900895CF93DF9300D01F92CDB763
:1099C000DEB78091280C1092280C882359F0109251
:1099D00031070E94B48D0F900F900F900F90DF9180
:1099E000CF91089560912B0C70912C0C80912D0CCF
:1099F00090912E0C611571058105910561F10F940F
:109A000042BB2091110230911202409113025091F9
:109A100014020F94A1BB20917F0D3091800D4091D5
:109A2000810D5091820D0F942DC260937F0D709324
:109A3000800D8093810D9093820D83E00E94CF8FE3
:109A400081E080937A0210922B0C10922C0C1092D1
:109A50002D0C10922E0C80917A02882309F4BBCF32
:109A60002091220C3091230C4091240C5091250C14
:109A700060917F0D7091800D8091810D9091820D8C
:109A80000F942CC269837A838B839C83CE010196C9
:109A90000F947316BC018DEA9CE60E944A999BCFF5
:109AA0002F923F924F925F926F927F928F929F92EE
:109AB000AF92BF92CF92DF92EF92FF921F93CF931C
:109AC000DF93CDB7DEB72C970FB6F894DEBF0FBE8D
:109AD000CDBF1C01162F8091280C1092280C8823D2
:109AE000E1F0109231070E94B48D2C960FB6F894D5
:109AF000DEBF0FBECDBFDF91CF911F91FF90EF90E2
:109B0000DF90CF90BF90AF909F908F907F906F909D
:109B10005F904F903F902F90089580912B0C9091E3
:109B20002C0CA0912D0CB0912E0C8D839E83AF83B5
:109B3000B887892B8A2B8B2B09F460C080913B025C
:109B4000882309F4BDC080913C028111B9C0613005
:109B500009F494C0623009F4A2C080903D02909054
:109B60003E02A0903F02B0904002C0904902D090C7
:109B70004A02E0904B02F0904C02612E712C6D81F4
:109B80007E818F8198850F9442BB20911102309184
:109B9000120240911302509114020F94A1BBD30101
:109BA000AA0FBB1FAA0FBB1FBC87AB87AD58B24F14
:109BB000BA87A9872D913D914D915C910F942DC24B
:109BC0002B013C018D819E81AF81B885B7FF8FC08D
:109BD000A5019401C301B2010F943BBB87FD7FC077
:109BE000EB85FC85ED58F24F408251826282738290
:109BF000812F0E94CF8F81E080937A0210922B0CEC
:109C000010922C0C10922D0C10922E0C80917A0236
:109C1000882309F46ACFF4E01F9FC0011124FC01DE
:109C2000ED58F24F8959924FDC012D913D914D91A4
:109C30005C9160817181828193810F942DC26B014F
:109C40007C01C982DA82EB82FC822DEC3CEC4CEC8C
:109C50005DE3609111027091120280911302909164
:109C600014020F948DC487FD52C0CE0101960F944B
:109C70007316BC01C1010E944A9937CF80904102FE
:109C800090904202A0904302B0904402C0904D02D6
:109C9000D0904E02E0904F02F09050026ECF809034
:109CA000450290904602A0904702B0904802C090B2
:109CB0005102D0905202E0905302F09054025DCFD6
:109CC000812C30E5932E33ECA32E37ECB32EC12C30
:109CD00040E5D42E43ECE42E47E4F42E4ECFA98584
:109CE000BA858D929D92AD92BC92139781CFA701B8
:109CF0009601C301B2010F948DC418160CF070CFF9
:109D0000E985FA85C082D182E282F38271CF20E0B8
:109D100030E040E251E4C701B6010F94A1BB20E05E
:109D200030E04AE754E40F94A1BB4B015C0120E012
:109D300030E0A901C701B6010F943BBB20E030E041
:109D400040EA50E487FF04C020E030E040EA50ECF5
:109D5000C501B4010F942DC220E030E040E251E48F
:109D60000F9427C30F9499C36B017C01F7FC62C069
:109D700020EA36E841E050E00F94A1C1CA01B901E0
:109D80002AE030E040E050E00F94A1C1605D6093B4
:109D90003C0CC701B60120E137E240E050E00F94EF
:109DA000A1C18AE0882E912CA12CB12CCA01B90145
:109DB000A50194010F94A1C1605D60933D0CC701A2
:109DC000B60128EE33E040E050E00F94A1C1CA0193
:109DD000B901A50194010F94A1C1605D60933E0C8F
:109DE0008EE280933F0CC701B60124E630E040E0EC
:109DF00050E00F94A1C1CA01B901A50194010F94CB
:109E0000A1C1605D6093400CC701B601A50194013A
:109E10000F94A1C1162FCA01B901A50194010F9495
:109E2000A1C1605D6093410C105D1093420C8CE306
:109E30009CE01FCFF094E094D094C094C11CD11C3E
:109E4000E11CF11C6DE2A3CF62E086EB9CE60C9472
:109E5000504D61E08DEB9CE60C94504D60E084EC3D
:109E60009CE60C94504DCF92DF92EF92FF92CF93ED
:109E7000DF9300D01F92CDB7DEB76B017C0120E0ED
:109E800030E0A9010F943BBB87FD1BC06DEB77E36E
:109E900086E095E3A70196010F942DC269837A832A
:109EA0008B839C83CE0101960F9473160F900F90B5
:109EB0000F900F90DF91CF91FF90EF90DF90CF90B8
:109EC00008956DEB77E386E095EBE4CF0F9442BB0A
:109ED00020E030E040E251E40F9427C320E030E07E
:109EE000A9010F942DC20C94334FAF92BF92CF9221
:109EF000DF92EF92FF920F931F93CF93DF93CDB733
:109F0000DEB7ADB6BEB680917F166AE47CE08823EA
:109F100011F06FE776E1FB0101900020E9F7CF0136
:109F2000861B970B01962DB73EB7281B390B0FB632
:109F3000F8943EBF0FBE2DBF8DB79EB701967C0132
:109F400080E2EDB7FEB78183C70101960F94E0C6AA
:109F500082E9C82E8FE0D82E04E91FE025E432E024
:109F600048EC5FE460EA7FE087EA9FE00E94EF93BD
:109F70000FB6F894BEBE0FBEADBEDF91CF911F915C
:109F80000F91FF90EF90DF90CF90BF90AF9008952A
:109F90008AE49CE00F9494A90E944F8D80E00C9479
:109FA0001C8F3F924F925F926F927F928F929F92FF
:109FB000AF92BF92CF92DF92EF92FF920F931F93D7
:109FC000CF93DF9361E081E00E946E8CC091300CF2
:109FD0003C2E85E0482E4C0E90E7C92E9EE0D92EEF
:109FE00005EA1EE0D4E0DC1B2FE3A22E2EE0B22E09
:109FF0003AE8E32E3EE0F32E83E0782E7C1A40E12F
:10A00000842E4EE0942E82E0682E6C1A81E0582E49
:10A010005C1AC11139C080912F0C8823B9F080914E
:10A020007A02882361F0632D619581E090912F0C75
:10A03000911180E024E04AEB5EE00F943297CF5F0D
:10A04000C411E7CF85E08093290C0CC08091280CC7
:10A050001092280C882319F30E94B48D80912A0C49
:10A060008823E9F2DF91CF911F910F91FF90EF903C
:10A07000DF90CF90BF90AF909F908F907F906F9028
:10A080005F904F903F900895C13051F580912F0C13
:10A09000813089F080917A02882389F21F9284EBC3
:10A0A0009EE09F938F935F9281E090912F0C91306F
:10A0B00071F180E02CC08091280C1092280C88232C
:10A0C00049F388E99DE09093D30B8093D20B0E94D3
:10A0D0004D8C0E944F8D80912A0C8823D9F2C2CFDB
:10A0E000C23009F06AC080912F0C8230C9F0809193
:10A0F0007A02882309F4A3CF1F928CE99EE09F93F4
:10A100008F936F9281E090912F0C923091F68F9304
:10A110000E94388C0F900F900F900F900F908FCF60
:10A120008091280C1092280C882309F39092D30B6D
:10A130008092D20B0E944D8C0E944F8D80912A0CF0
:10A140008823A9F28FCF80912F0C833081F08091EA
:10A150007A02882309F473CF1F92FF92EF927F92C5
:10A1600081E090912F0C933009F0A3CFD0CF809154
:10A17000280C1092280C882351F3B092D30BA09294
:10A18000D20B0E944D8C0E944F8D80912A0C882307
:10A19000F1F268CF8091280C1092280C8823B1F03E
:10A1A000D092D30BC092D20B0E944D8C0E944F8D47
:10A1B00080912A0C882351F055CFC33021F2C4304E
:10A1C00009F03DCF80912F0C843021F380917A02E9
:10A1D000882309F434CF1F921F930F93DF9381E0FC
:10A1E00090912F0C943009F064CF91CF0F941F36CB
:10A1F0000F9467AA81E08093391A0F94A9AA0C944E
:10A200004F8D6F927F928F929F92AF92BF92CF921B
:10A21000DF92EF92FF920F931F93CF93DF9381E032
:10A220008093310761E00E946E8CC091300C85E014
:10A23000882E8C0ED1E006EF10E593E7E92E9DE025
:10A24000F92E82E0982E9C1A2CE0C22E28E3D22E02
:10A250003EE7A32E3DE0B32E7D2E7C1A6C2E61943A
:10A26000C11130C0DD23D9F080912F0C1816BCF03D
:10A2700040912B0C50912C0C60912D0C70912E0C58
:10A280004F5F5F4F6F4F7F4F40932B0C50932C0CC1
:10A2900060932D0C70932E0C8F5F80932F0C809108
:10A2A0007A02882341F030E020E041E06BE87DE075
:10A2B000862D0E94BF98CF5F8C12D2CF83E080930F
:10A2C000290C23C0C13081F580912F0C813089F099
:10A2D00080917A02882309F444C0DF92CF92BF9222
:10A2E000AF927F9281E090912F0C913089F180E0C4
:10A2F0002FC08091280C1092280C882349F30E94CB
:10A300000C3880912A0C882319F3DF91CF911F918B
:10A310000F91FF90EF90DF90CF90BF90AF909F9004
:10A320008F907F906F900895C23029F680912F0C06
:10A330008230C9F080917A02882399F01F930F939D
:10A34000FF92EF929F9281E090912F0C923079F6DC
:10A350008F930E94388C0F900F900F900F900F905A
:10A360000F90D0E0A8CF8091280C1092280C882361
:10A3700009F30E94F65080912A0C8823D9F2C5CFA8
:10A38000EF92FF920F931F93CF93DF93CDB7DEB77A
:10A3900065970FB6F894DEBF0FBECDBF8091280C35
:10A3A0001092280C882379F00E94B48D65960FB620
:10A3B000F894DEBF0FBECDBFDF91CF911F910F91FB
:10A3C000FF90EF90089560E085E00E946E8C009110
:10A3D000300C10E08AE3F82E90E2E92E011130C033
:10A3E00080917A02882341F030E020E043E06FE280
:10A3F0007DE0812F0E94BF98F982EA8242E150E01D
:10A4000067EF7CE0CE0103960F946CBA8C8987FDD0
:10A410001C8A0530C1F580917A02882349F09E019B
:10A420002F5F3F4F41E06DEE7CE0812F0E94BF988F
:10A430000F5F1F5F153091F687E08093290CB6CF30
:10A44000013051F480917A028823B1F230E020E0AB
:10A4500041E063E27DE0CDCF023009F580917A02E0
:10A46000882351F230E020E041E068E17DE0C1CF97
:10A4700080917A02882309F4BFCF30E020E041E0E8
:10A480006CE07DE0B6CF063099F680917A028823A1
:10A4900079F230E020E041E068ED7CE0C6CF0330A7
:10A4A00039F3043009F0A8CF80917A02882309F4A7
:10A4B000A3CF30E020E041E069EF7CE09ACFEF925B
:10A4C000FF920F931F93CF93DF93CDB7DEB76597BE
:10A4D0000FB6F894DEBF0FBECDBF8091280C10924E
:10A4E000280C882379F00E94B48D65960FB6F894F5
:10A4F000DEBF0FBECDBFDF91CF911F910F91FF90B7
:10A50000EF90089560E085E00E946E8C0091300C21
:10A5100010E08AE3F82E90E2E92E01110CC0809140
:10A520007A02882341F030E020E043E067EC7CE0F1
:10A53000812F0E94BF98F982EA8242E150E060ECEC
:10A540007CE0CE0103960F946CBA8C8987FD1C8A3F
:10A55000013069F480917A02882349F09E012F5FCF
:10A560003F4F41E06BEB7CE0812F0E94BF98F98266
:10A57000EA8242E150E067EB7CE0CE0103960F9463
:10A580006CBA8C8987FD1C8A023069F480917A024A
:10A59000882349F09E012F5F3F4F41E06EEA7CE047
:10A5A000812F0E94BF98F982EA8242E150E066EA78
:10A5B0007CE0CE0103960F946CBA8C8987FD1C8ACF
:10A5C000033069F480917A02882349F09E012F5F5D
:10A5D0003F4F41E062EA7CE0812F0E94BF980F5F0D
:10A5E0001F5F153009F099CF84E08093290C7DCF4F
:10A5F000EF92FF920F931F93CF93DF93CDB7DEB708
:10A6000065970FB6F894DEBF0FBECDBF8091280CC2
:10A610001092280C882379F00E94B48D65960FB6AD
:10A62000F894DEBF0FBECDBFDF91CF911F910F9188
:10A63000FF90EF90089560E085E00E946E8C00919D
:10A64000300C10E08AE3F82E90E2E92E01110CC0E4
:10A6500080917A02882341F030E020E042E063E913
:10A660007CE0812F0E94BF98F982EA8242E150E0AB
:10A6700061E97CE0CE0103960F946CBA8C8987FD6A
:10A680001C8A013069F480917A02882349F09E0186
:10A690002F5F3F4F40E068E87CE0812F0E94BF9829
:10A6A000F982EA8242E150E064E87CE0CE01039660
:10A6B0000F946CBA8C8987FD1C8A023009F04EC059
:10A6C00080917A02882349F09E012F5F3F4F40E03E
:10A6D0006BE77CE0812F0E94BF98F982EA8242E119
:10A6E00050E066E57CE0CE0103960F946CBA8C894D
:10A6F00087FD1C8A053069F480917A02882349F02D
:10A700009E012F5F3F4F40E068E87CE0812F0E9470
:10A71000BF98F982EA8242E150E062E57CE0CE0136
:10A7200003960F946CBA8C8987FD1C8A063089F5D4
:10A7300080917A02882349F09E012F5F3F4F40E0CD
:10A740006BE77CE0812F0E94BF980F5F1F5F153081
:10A7500009F07CCF88E08093290C60CF033059F456
:10A7600080917A02882309F4B8CF30E020E040E0FD
:10A7700069E67CE0AFCF043009F0AFCF80917A0278
:10A78000882309F4AACF30E020E042E068E57CE0CD
:10A79000A1CF0730D1F680917A028823B1F230E060
:10A7A00020E040E069E67CE0CDCF2F923F924F92CF
:10A7B0005F926F927F928F929F92AF92BF92CF9251
:10A7C000DF92EF92FF920F931F93CF93DF93CDB75A
:10A7D000DEB7E2970FB6F894DEBF0FBECDBF809113
:10A7E000280C1092280C8823D9F00E94B48DE29690
:10A7F0000FB6F894DEBF0FBECDBFDF91CF911F9192
:10A800000F91FF90EF90DF90CF90BF90AF909F900F
:10A810008F907F906F905F904F903F902F90089512
:10A820008091BC0B9091BD0B9CA78BA7A091BE0BF8
:10A83000B091BF0BBEA7ADA74090C00B5090C10B0D
:10A840006090C20B7090C30B8091C40B9091C50BAC
:10A85000A091C60BB091C70B8FA798ABA9ABBAABB1
:10A860008090C80B9090C90BA090CA0BB090CB0BF6
:10A8700060E085E00E946E8C0091300C10E0DE01FB
:10A8800056967D018AE0C82ED12C97EF292E9BE0A9
:10A89000392E6FE47CE0CE0101960F9444BA8BA56B
:10A8A0009CA50F94DC18BC01CE0103960F94E0C662
:10A8B00001110DC080917A02882349F09E012F5F1B
:10A8C0003F4F40E063E47CE0812F0E94BF9860E44A
:10A8D0007CE0CE0101960F9444BA8DA59EA50F94FD
:10A8E000DC18BC01CE0103960F94E0C6013009F0DC
:10A8F0004CC080917A02882349F09E012F5F3F4F20
:10A9000040E066E37CE0812F0E94BF9820E030E0C9
:10A9100048EC52E4C501B4010F9427C30F9499C3C6
:10A92000CB01B6010F9410C29F938F9320E030E0CB
:10A930004AE754E4C501B4010F9427C30F9499C3A7
:10A940009F938F937F936F933F922F92FF92EF92FB
:10A950000F94D2BA0FB6F894DEBF0FBECDBF07304A
:10A9600059F480917A02882339F0970140E064EF2E
:10A970007BE0812F0E94BF980F5F1F5F153009F0A9
:10A9800088CF88E08093290C32CF023059F480912F
:10A990007A02882309F4BACF30E020E040E065E293
:10A9A0007CE0B1CF033099F480917A02882309F4D6
:10A9B000ADCF49825A826B827C82B701CE0101966B
:10A9C0000E943AA49C0140E062E27CE09CCF04300B
:10A9D00009F04CC080917A02882341F030E020E0F9
:10A9E00040E061E17CE0812F0E94BF9820E030E0F0
:10A9F00048EC52E4C501B4010F9427C30F9499C3E6
:10AA0000CB01B6010F9410C29F938F9320E030E0EA
:10AA10004AE754E4C501B4010F9427C30F9499C3C6
:10AA20009F938F937F936F933F922F92FF92EF921A
:10AA30000F94D2BA0FB6F894DEBF0FBECDBF9CCF35
:10AA400080917A02882391F28FA598A9A9A9BAA921
:10AA500089839A83AB83BC83B701CE0101960E94A0
:10AA60003AA49C0140E06EE07CE04DCF053041F31C
:10AA7000063009F04BCF80917A02882309F4B6CFD3
:10AA800030E020E040E06FEF7BE03DCF2F923F923F
:10AA90004F925F926F927F928F929F92AF92BF92EE
:10AAA000CF92DF92EF92FF920F931F93CF93DF939A
:10AAB0004C010F944BBA01968401080F191FC8016D
:10AAC0000F944BBA01966801C80ED91EF801608038
:10AAD000C1E0611001C0C0E0F6013080D1E031106A
:10AAE00001C0D0E0AA24A3946110A12C60E085E00D
:10AAF0000E946E8C5090300C752C9EE0E92EF12C4B
:10AB0000252C21948A2D90E001965C01AC0EB11C9D
:10AB1000AD0EB11C71101DC080917A028823A1F086
:10AB2000E0910502E2506EEB7AE0E33038F4F0E0B9
:10AB3000EE0FFF1FE854FD4F6081718130E020E08F
:10AB400043E0822D0E94BF98D1E0611013C0D2E093
:10AB500011C0D2E06110D1E0D7110CC080917A020F
:10AB6000882341F030E020E041E0B4018D2F8519C9
:10AB70000E94BF98C1E0CD0F472C4518662079F0A0
:10AB8000C7110BC080917A02882339F030E020E0B1
:10AB900041E0B801842D0E94BF98C2E0CD0F332060
:10ABA00071F0C7110BC080917A02882339F030E030
:10ABB00020E041E0B601842D0E94BF98CF5FF3E012
:10ABC000AF16B1040CF4CF5FC71162C080917A0256
:10ABD000882309F45AC030E020E042E06BEC7AE0D0
:10ABE000842D0E94BF98D0912B0793EF9E0D9093D8
:10ABF0002A078EEF8E0D8093440C2091311A2E156A
:10AC00001F0411F00CF041C02091331A9217E8F59F
:10AC10009EE39093341A8093351A65E470E080E0E7
:10AC200090E00E94AE9261E36D0F062E000C770B50
:10AC3000880B990B0E94AE9260E270E080E090E099
:10AC40000E94AE9280913119909132190F94071998
:10AC50000E9446996FE270E080E090E00E94AE9220
:10AC60000E942E90811109C085E08D9FF001112472
:10AC7000E753F64F8481811108C080913319909178
:10AC800034190F9407190E94469992E090937A0222
:10AC9000ECE0EE0EF11C7394FAE4EF16F10409F007
:10ACA00039CFCF5FC093290CDF91CF911F910F91C6
:10ACB000FF90EF90DF90CF90BF90AF909F908F90DC
:10ACC0007F906F905F904F903F902F90089586ED0A
:10ACD0009AE00C94465583EE9AE00C94465585E034
:10ACE0009BE00C94465580EA9BE00C9446558BE51E
:10ACF0009BE00C94465588E89BE00C9446558BED00
:10AD00009BE00C9446558EEB9BE00C9446558EE3ED
:10AD10009BE00C9446558FE19BE00C94465584E0F3
:10AD20000D94429B83E00D94429B82E00D94429BE4
:10AD3000CF93DF9300D01F92CDB7DEB784EF91E0C1
:10AD4000A0E0B0E089839A83AB83BC83BE016F5FD0
:10AD50007F4F88E70F94AF440F900F900F900F90A4
:10AD6000DF91CF9108956F927F928F929F92AF92D1
:10AD7000BF92CF92DF92EF92FF920F931F93CF93E8
:10AD8000DF9361E081E00E946E8CC091300C6C2EEC
:10AD900085E0782E7C0E95EBE92E91E0F92E2FE7D9
:10ADA000C22E29E0D22ED5E0DC1B31E1A32E32E009
:10ADB000B32E14E01C1B03E00C1B82E0982E9C1A9F
:10ADC00081E0882E8C1AC11136C080912F0C882307
:10ADD000B9F080917A02882361F0662D619581E057
:10ADE00090912F0C911180E024E04CEA59E00F94EF
:10ADF0003297CF5FC711E7CF86E08093290C0CC054
:10AE00008091280C1092280C882319F30E94B48D8D
:10AE100080912A0C8823E9F2DF91CF911F910F9145
:10AE2000FF90EF90DF90CF90BF90AF909F908F906A
:10AE30007F906F900895C13029F580912F0C81305B
:10AE4000A1F080917A028823A1F28FEB92E09F9388
:10AE50008F9381E999E09F938F938F9281E09091F6
:10AE60002F0C913049F180E027C08091280C10927E
:10AE7000280C882331F30F94204580912A0C8823D5
:10AE800001F3CACFC23009F085C080912F0C823007
:10AE9000E9F080917A02882309F4ABCF88E996E53E
:10AEA0009F938F9387E899E09F938F939F9281E080
:10AEB00090912F0C9230B9F68F930E94388C0F909E
:10AEC0000F900F900F900F900F9093CF8091280CC0
:10AED0001092280C8823E9F20E94985680912A0C3F
:10AEE0008823B9F299CF80912F0C8330A9F08091FB
:10AEF0007A02882309F47DCF89ED92E09F938F93A6
:10AF000088E799E09F938F930F9381E090912F0CA6
:10AF1000933009F0A8CFD0CF8091280C1092280C44
:10AF2000882329F30F94EA4480912A0C8823F9F2AC
:10AF300073CF80912F0C843099F080917A0288230E
:10AF400009F457CFBF92AF9283E799E09F938F9315
:10AF50001F9381E090912F0C943009F084CFACCFF7
:10AF60008091280C1092280C882339F30F94CF4439
:10AF700080912A0C882309F34FCF8091280C1092DE
:10AF8000280C882399F00F94054580912A0C88237A
:10AF900069F042CFC33009F4A6CFC43051F2C530B6
:10AFA00009F027CF80912F0C853039F380917A02F8
:10AFB000882309F41ECFFF92EF92DF92CF92DF93A6
:10AFC00081E090912F0C953009F04DCF75CF809195
:10AFD000450C803210F40F94C2360E944D8C0C94B4
:10AFE000B48D80E090E0A0E8B0E480937B0D909376
:10AFF0007C0DA0937D0DB0937E0D80EB92E00F94BD
:10B000005707809133070F943841109231070C9401
:10B01000B48D80E090E0A0E8B0E480937B0D909345
:10B020007C0DA0937D0DB0937E0D80EB92E00F948C
:10B030005707E091320780E090E0A6E1B3E4E43006
:10B0400009F44AC080E090E0A0EBB1E48093730D76
:10B050009093740DA093750DB093760D8093770D3A
:10B060009093780DA093790DB0937A0DEE0FFF0BAE
:10B07000E057FD4F808191818330910549F1843003
:10B080009105D9F1029761F480E090E0ABE8B3E478
:10B090008093730D9093740DA093750DB093760DFE
:10B0A00088E992E00F94570710927B0D10927C0D67
:10B0B00010927D0D10927E0D80EB92E00F94570759
:10B0C000809132078F5F8530ECF4809332070895CA
:10B0D00080E090E0ABE8B3E48093730D9093740D3F
:10B0E000A093750DB093760D8093770D9093780DA6
:10B0F000A093790DB0937A0DD3CF80E090E0ABE8C8
:10B10000B3E4F2CF10923207089580917A02882337
:10B1100041F030E020E041E06DEF73E182E00E9419
:10B12000BF98809112098770873079F410923207A6
:10B1300020E040E070E060E08DE99CE40E94CC8C6F
:10B1400081E0809324070C9409580895CF93DF93EE
:10B1500000D01F92CDB7DEB70F94A0C30F9440BBB1
:10B1600069837A838B839C83CE0101960F94F015BB
:10B170000F900F900F900F90DF91CF9108950F9443
:10B1800042BB2AE037ED43E25DE30F9427C320E0A2
:10B1900030E0A9010F942DC20C94A658CF92DF92F3
:10B1A000EF92FF92CF93DF9300D01F92CDB7DEB71F
:10B1B0006B017C0120E030E0A9010F943BBB87FDCF
:10B1C0001BC06DEB77E386E095E3A70196010F9432
:10B1D0002DC269837A838B839C83CE0101960F9461
:10B1E000F0150F900F900F900F90DF91CF91FF907F
:10B1F000EF90DF90CF9008956DEB77E386E095EBCD
:10B20000E4CF0F9442BB2AE037ED43E25DE30F94B5
:10B2100027C320E030E0A9010F942DC20C94CE5832
:10B220000F9442BB20E030E0A9010F942DC20C9492
:10B23000CE58CF92DF92EF92FF92CF93DF9300D060
:10B240001F92CDB7DEB70F9442BB20E030E048EC50
:10B2500052E40F9427C320E030E0A9010F942DC2DF
:10B260006B017C0120E030E0A9010F943BBB2DEB8A
:10B2700037E346E055E387FF04C02DEB37E346E0B4
:10B2800055EBC701B6010F942DC269837A838B8376
:10B290009C83CE0101960F9492170F900F900F9000
:10B2A0000F90DF91CF91FF90EF90DF90CF900895B6
:10B2B0007F928F929F92AF92BF92CF92DF92EF9246
:10B2C000FF920F931F93CF93DF9361E081E00E9481
:10B2D0006E8CC091300C65E0862E8C0ED6E0DC1BA7
:10B2E00085E0D82EDC1A84E0C82ECC1A83E0B82E74
:10B2F000BC1A82E0A82EAC1A81E0982E9C1A7C2EF3
:10B300007194C11134C080912F0C8823B1F08091C9
:10B310007A02882359F081E090912F0C911180E0FE
:10B3200024E043E958E0672D0F943297CF5FC811AE
:10B33000E8CF87E08093290C0CC08091280C1092F4
:10B34000280C882321F30E94B48D80912A0C882335
:10B35000F1F2DF91CF911F910F91FF90EF90DF906D
:10B36000CF90BF90AF909F908F907F900895C13005
:10B37000E9F580912F0C8130E9F080917A028823E1
:10B38000A9F211E080912F0C813009F010E060915A
:10B39000E5137091E6138091E7139091E8130E94F2
:10B3A000CE5800E09C014EED57E0692D812F0E94A0
:10B3B000F49ABCCF8091280C1092280C8823E9F2D3
:10B3C0000F948D98E12C1CE3F12E0CE116E420E0A3
:10B3D00030E040E85FE365EE73E18EED97E00F94B7
:10B3E000999880912A0C882341F2B3CFC23009F09A
:10B3F00006C180912F0C8230D9F080917A02882387
:10B4000009F494CF11E080912F0C823009F010E004
:10B410006091E9137091EA138091EB139091EC1312
:10B420000E94CE5800E09C0147ED57E06A2DBECF48
:10B430008091280C1092280C8823F9F20F948D9893
:10B44000E12C1CE3F12E0CE116E420E030E040E8B2
:10B450005FE369EE73E187ED97E00F94999880912F
:10B460002A0C882351F275CF80912F0C8330D9F0AC
:10B4700080917A02882309F459CF11E080912F0C32
:10B48000833009F010E06091ED137091EE1380911C
:10B49000EF139091F0130E94CE5800E09C0140ED14
:10B4A00057E06B2D83CF8091280C1092280C8823B5
:10B4B000F9F20F948D98E12C1CE3F12E0CE116E4C7
:10B4C00020E030E040E85FE36DEE73E180ED97E06F
:10B4D0000F94999880912A0C882351F23ACF809149
:10B4E0002F0C8430D9F080917A02882309F41ECF82
:10B4F00011E080912F0C843009F010E06091F1137D
:10B500007091F2138091F3139091F4130E94CE582E
:10B5100000E09C0149EC57E06C2D48CF8091280C4D
:10B520001092280C8823F9F20F948D98E12C1CE3DB
:10B53000F12E0CE116E420E030E040E85FE361EF3B
:10B5400073E189EC97E00F94999880912A0C8823F5
:10B5500051F2FFCE80912F0C8530D9F080917A0284
:10B56000882309F4E3CE11E080912F0C853009F097
:10B5700010E0609101147091021480910314909175
:10B5800004140E94CE5800E09C0144EC57E06D2D5D
:10B590000DCF8091280C1092280C8823F9F20F947B
:10B5A0008D98E12C1CE3F12E0CE116E420E030E054
:10B5B000A90161E074E184EC97E00F94999880917F
:10B5C0002A0C882359F2C5CE8091280C1092280CA1
:10B5D000882329F10F948D98E12C1CE3F12E0CE1C6
:10B5E00016E420E030E0A90165E074E18AEB97E021
:10B5F0000F94999880912A0C882389F0AACEC330A1
:10B6000009F432CFC43009F46ACFC53009F4A2CFAF
:10B61000C63009F08BCE80912F0C8630A9F2809134
:10B620007A02882309F482CE11E080912F0C8630B3
:10B6300009F010E0609105147091061480910714D0
:10B64000909108140E94CE5800E09C014AEB57E00C
:10B650006D2FACCE2F923F924F925F926F927F925E
:10B660008F929F92AF92BF92CF92DF92EF92FF9212
:10B670000F931F93CF93DF93CDB7DEB72C970FB601
:10B68000F894DEBF0FBECDBFC090C513D090C613D7
:10B69000E090C713F090C8138091C9139091CA131A
:10B6A000A091CB13B091CC138C159D05AE05BF05B1
:10B6B00010F4D701C601C090C113D090C213E0901E
:10B6C000C313F090C413BC01CD016C157D058E052C
:10B6D0009F0510F4C701B6010F9440BB2B013C013C
:10B6E00061E081E00E946E8C2091300C2B872E83CC
:10B6F000822F8B5F8D8387E0922F821B8F8386E062
:10B70000821B888785E0821B898784E0821B8A8769
:10B7100083E0282E221A82E0382E321A91959C87D7
:10B720002B85211142C080912F0C8823C9F0809174
:10B730007A02882359F081E090912F0C911180E0DA
:10B7400024E043E958E06C850F9432978B858F5F36
:10B750008B879D819813E4CF88E08093290C0CC0DF
:10B760008091280C1092280C882309F30E94B48D34
:10B7700080912A0C8823D9F22C960FB6F894DEBF5C
:10B780000FBECDBFDF91CF911F910F91FF90EF9032
:10B79000DF90CF90BF90AF909F908F907F906F90F1
:10B7A0005F904F903F902F9008958B85813009F0E6
:10B7B0008BC080912F0C8130F9F080917A02882320
:10B7C00029F211E080912F0C813009F010E0609196
:10B7D000F5137091F6138091F7139091F8130E946E
:10B7E000CE5861E02E81621B00E09C0144E158E0EC
:10B7F000812F0E94F49AAACF8091280C1092280CD5
:10B800008823D9F20F948D982AE037ED43E25DE367
:10B81000C301B2010F94A1BB20E030E0A9010F9455
:10B820002DC24B015C0120E030E040E05FE40F946A
:10B830003BBB87FD05C0812C912CA12C3FE4B32E8E
:10B840002AE037ED43E25DE36091F5137091F61362
:10B850008091F7139091F8130F94A1BB20E030E092
:10B86000A9010F942DC220E030E040E85FE30F947F
:10B870002CC20F94A0C369837A838B839C83C501F8
:10B88000B4010F9499C37B018C0121E0E21AF10805
:10B89000010911091F92912C812C21E4A22E20E490
:10B8A000B22EC980DA8021E030E040E050E065EF60
:10B8B00073E184E198E00E94F28D0F9080912A0C50
:10B8C000882309F47ACF58CF8B85823009F090C154
:10B8D00080912F0C8230D9F080917A02882309F46C
:10B8E00035CF11E080912F0C823009F010E060918B
:10B8F000F9137091FA138091FB139091FC130E943D
:10B90000CE5800E09C014AE058E0632D71CF809151
:10B91000280C1092280C8823F9F20F948D986091CE
:10B92000CD137091CE138091CF139091D0130F94BB
:10B9300040BB7B018C0120E030E048EC52E469EF31
:10B9400073E18AE098E00F94999880912A0C8823FB
:10B9500019F212CF80912F0C8330D9F080917A02A6
:10B96000882309F4F3CE11E080912F0C833009F085
:10B9700010E06091FD137091FE138091FF13909180
:10B9800000140E94CE5800E09C0141E058E0622D76
:10B990002FCF8091280C1092280C8823F9F20F9455
:10B9A0008D982AE037ED43E25DE3C301B2010F94C5
:10B9B000A1BB20E030E0A9010F942DC24B015C0136
:10B9C00020E030E040E05FE40F943BBB87FD05C022
:10B9D000812C912CA12C9FE4B92E2AE037ED43E273
:10B9E0005DE36091FD137091FE138091FF139091C0
:10B9F00000140F94A1BB20E030E0A9010F942DC2E8
:10BA000020E030E040E85FE30F942CC20F94A0C325
:10BA100069837A838B839C83C501B4010F9499C396
:10BA20007B018C0121E0E21AF108010911091F9242
:10BA3000912C812C81E4A82E80E4B82EC980DA8074
:10BA400021E030E040E050E06DEF73E181E098E00C
:10BA50000E94F28D0F9080912A0C882309F47ECFEA
:10BA60008BCE80912F0C8430E9F080917A0288236C
:10BA700009F46CCE11E080912F0C843009F010E0B5
:10BA80006091C1137091C2138091C3139091C4133C
:10BA90000F9440BB0E94A65800E09C014AEF57E07B
:10BAA0006A85A6CE8091280C1092280C8823E9F292
:10BAB0000F948D980CEE13E624E630E040E050E061
:10BAC00061EC73E18AEF97E00F94379980912A0C2B
:10BAD000882359F251CE80912F0C8530E9F0809166
:10BAE0007A02882309F432CE11E080912F0C853040
:10BAF00009F010E06091C5137091C6138091C713CF
:10BB00009091C8130F9440BB0E94A65800E09C017E
:10BB100043EF57E069856CCE8091280C1092280C79
:10BB20008823E9F20F948D980AEE13E624E630E0BC
:10BB300040E050E065EC73E183EF97E00F943799B4
:10BB400080912A0C882359F217CE80912F0C8630D1
:10BB5000E9F080917A02882309F4F8CD11E0809110
:10BB60002F0C863009F010E06091C9137091CA1350
:10BB70008091CB139091CC130F9440BB0E94A65898
:10BB800000E09C014CEE57E0688532CE8091280C95
:10BB90001092280C8823E9F20F948D9808EE13E692
:10BBA0002AE030E040E050E069EC73E18CEE97E091
:10BBB0000F94379980912A0C882359F2DDCD80911A
:10BBC000280C1092280C882339F10F948D9806EEDA
:10BBD00013E624E630E040E050E06DEC73E185EEE2
:10BBE00097E00F94379980912A0C8823A9F0C4CD4F
:10BBF0002B85233009F4AECE243009F432CF253022
:10BC000009F469CF263009F4A0CF273009F09ECD82
:10BC100080912F0C873099F280917A02882309F461
:10BC200095CD11E080912F0C873009F010E06091E4
:10BC3000CD137091CE138091CF139091D0130F94A8
:10BC400040BB0E94A65800E09C0145EE57E06F8182
:10BC5000CFCDBF92CF92DF92EF92FF920F931F93BF
:10BC6000CF93DF9361E081E00E946E8CC091300C35
:10BC700085E0C82ECC0ED4E0DC1B13E01C1B82E058
:10BC8000F82EFC1A81E0E82EEC1ABC2EB194C111FA
:10BC900030C080912F0C8823B1F080917A028823E4
:10BCA00059F081E090912F0C911180E024E043E95C
:10BCB00058E06B2D0F943297CF5FCC11E8CF85E021
:10BCC0008093290C0CC08091280C1092280C88239A
:10BCD00021F30E94B48D80912A0C8823F1F2DF9128
:10BCE000CF911F910F91FF90EF90DF90CF90BF9079
:10BCF0000895C130B9F580912F0C8130F1F0809119
:10BD00007A028823C9F2DD24D39480912F0C8130EC
:10BD100009F0D12C6091D5137091D6138091D7136F
:10BD20009091D8130E94733900E09C0148E858E0D4
:10BD30006E2D8D2D0E94F49ABFCF8091280C109209
:10BD4000280C8823E1F20F948D9844EE53E665EDBC
:10BD500073E188E898E00F94B99980912A0C8823C0
:10BD600071F2BDCFC23009F07FC080912F0C8230BC
:10BD7000E1F080917A02882309F49ECFDD24D394E8
:10BD800080912F0C823009F0D12C6091D9137091E1
:10BD9000DA138091DB139091DC130E94733900E079
:10BDA0009C014DE758E06F2DC4CF8091280C109274
:10BDB000280C8823F1F20F948D9842EE53E669ED3A
:10BDC00073E18DE798E00F94B99980912A0C88234C
:10BDD00081F285CF80912F0C8330E1F080917A023F
:10BDE000882309F469CFDD24D39480912F0C83300C
:10BDF00009F0D12C6091DD137091DE138091DF1377
:10BE00009091E0130E94733900E09C0142E758E0F2
:10BE1000612F8FCF8091280C1092280C8823F1F28B
:10BE20000F948D9840EE53E66DED73E182E798E054
:10BE30000F94B99980912A0C882381F250CF809178
:10BE4000280C1092280C8823C9F00F948D984EED81
:10BE500053E661EE73E187E698E00F94B99980911B
:10BE60002A0C882359F03BCFC33009F4B3CFC43038
:10BE700009F022CF80912F0C843009F380917A024F
:10BE8000882309F419CFDD24D39480912F0C8430BA
:10BE900009F0D12C6091E1137091E2138091E313CA
:10BEA0009091E4130E94733900E09C0147E658E04A
:10BEB0006D2F3FCF2F923F924F925F926F927F9262
:10BEC0008F929F92AF92BF92CF92DF92EF92FF92AA
:10BED0000F931F93CF93DF9300D000D0CDB7DEB781
:10BEE00061E081E00E946E8C7090300C672C85E0E0
:10BEF000870D8D838CE087198E8388E0582E571824
:10BF00008BE0482E47188AE0382E371889E0282E13
:10BF100027187110EAC080912F0C882309F4BEC045
:10BF200080917A02882361F0662D619581E090917D
:10BF30002F0C911180E024E043E958E00F943297F0
:10BF40002CEA35EC47E25EE360913A1970913B19B7
:10BF500080913C1990913D190F9427C3609320075D
:10BF60007093210780932207909323072CEA35ECE6
:10BF700047E25EE360913E1970913F19809140194C
:10BF8000909141190F94A1BB60931C0770931D07FA
:10BF900080931E0790931F0785E07812E5C11092E9
:10BFA000450C80912F0C853009F4C7C180917A022D
:10BFB0008823C9F011E080912F0C853009F010E042
:10BFC000609136197091371980913819909139190B
:10BFD0000E94334F65E0661900E09C014CE857E091
:10BFE000812F0E94F49A2CEA35EC47E25EE36091DF
:10BFF000900C7091910C8091920C9091930C0F94F5
:10C0000027C36093200770932107809322079093A2
:10C0100023072CEA35EC47E25EE36091940C7091C3
:10C02000950C8091960C9091970C0F94A1BB609306
:10C030001C0770931D0780931E0790931F0789E0CC
:10C040007812B8C28FEF8093450C80912F0C893005
:10C0500009F499C280917A028823C1F011E080919D
:10C060002F0C893009F010E060918C0C70918D0CD0
:10C0700080918E0C90918F0C0E94334F00E09C01B8
:10C080004CE857E0622D812F0E94F49A73948D81C1
:10C0900078123FCF8DE08093290C0EC08091280C40
:10C0A0001092280C882309F43BCF0E94B48D809114
:10C0B0002A0C882309F434CF26960FB6F894DEBFF5
:10C0C0000FBECDBFDF91CF911F910F91FF90EF90E9
:10C0D000DF90CF90BF90AF909F908F907F906F90A8
:10C0E0005F904F903F902F90089581E0781230C07C
:10C0F00090912F0C9130C9F080917A02882309F435
:10C100001FCF61E0661981E0913009F080E09091E5
:10C11000D4092EEA37E0911102C02AEA37E001E0A3
:10C1200041EB57E00E94F49A0BCF8091280C1092BB
:10C13000280C882309F38091D40987258093D4099A
:10C1400083E080937A0280912A0C8823A9F2B4CFED
:10C1500082E07812EDC280912F0C823009F466C023
:10C1600080917A028823A9F011E080912F0C82300F
:10C1700009F010E080913702909138020F9407196E
:10C1800062E0661900E09C0143EA57E0812F0E94BB
:10C19000F49A2CEA35EC47E25EE360913A1970912B
:10C1A0003B1980913C1990913D190F9427C36093DE
:10C1B00020077093210780932207909323072CEA8E
:10C1C00035EC47E25EE360913E1970913F19809132
:10C1D0004019909141190F94A1BB60931C07709373
:10C1E0001D0780931E0790931F0788E07812FBCEEF
:10C1F0001092450C80912F0C883009F4A9C18091D0
:10C200007A02882309F4D7C011E080912F0C88307E
:10C2100009F010E080910202909103020F94071937
:10C2200000E09C014DE657E0652DDACE8091280CA8
:10C230001092280C882309F493CF10E000E02CE240
:10C2400031E050E040E067E372E083EA97E00F946A
:10C25000059A80912A0C882309F482CF2DCF8091F2
:10C260002F0C8330C9F080917A02882309F491CF92
:10C2700011E080912F0C833009F010E0809135029D
:10C28000909136020F94071963E0661900E09C0153
:10C290004CE957E0812F46CF8091280C1092280C52
:10C2A000882309F310E000E02CE231E050E040E0A8
:10C2B00065E372E08CE997E00F94059A80912A0C6F
:10C2C000882389F2F9CE8091280C1092280C8823BB
:10C2D00009F43AC220E030E048EC52E460913102C7
:10C2E0007091320280913302909134020F94A1BB7D
:10C2F00020E030E0A9010F942DC20F94A0C31F923B
:10C30000912C812CE9E5AE2EE0E4BE2E6B0118EEF7
:10C31000E12E13E0F12E00E010E020E030E0A90172
:10C3200061E372E084E997E00E94F28D0F908091C2
:10C330002A0C882309F408C2BFCE8091280C1092E1
:10C34000280C882309F432CE0F948D9850E040E0F9
:10C3500066E379E18CE897E00F94B29A80912A0C19
:10C36000882309F423CEA8CE86E07812B7C01092B5
:10C37000450C80912F0C863009F46BC080917A02B5
:10C380008823C9F011E080912F0C863009F010E06D
:10C3900060912007709121078091220790912307D7
:10C3A0000E943C3866E0661900E09C0144E857E0D2
:10C3B000812F0E94F49A2CEA35EC47E25EE360910B
:10C3C000900C7091910C8091920C9091930C0F9421
:10C3D00027C36093200770932107809322079093CF
:10C3E00023072CEA35EC47E25EE36091940C7091F0
:10C3F000950C8091960C9091970C0F94A1BB609333
:10C400001C0770931D0780931E0790931F078CE0F5
:10C4100078123CCE8FEF8093450C80912F0C8C309E
:10C4200009F46BC180917A02882309F42FCE11E0C0
:10C4300080912F0C8C3009F010E0809100029091D7
:10C4400001020F94071900E09C014DE657E06E8150
:10C450001ACE8091280C1092280C882309F48ECFD4
:10C460000F948D9820E030E048EC52E46091200772
:10C470007091210780912207909123070F94A1BB0F
:10C4800020E030E0A9010F942DC220E030E040E828
:10C490005FE30F942CC20F94A0C31F923BEC832E3A
:10C4A00034E8932E4DE4A42E40E4B42E6B0117E53E
:10C4B000E12E1EE3F12E0FE010E021E030E040E03D
:10C4C00050E060E277E084E897E00E94F28D0F9000
:10C4D00080912A0C882309F451CFEECD87E07812A1
:10C4E00084CE1092450C80912F0C8730E1F0809122
:10C4F0007A02882309F45FCF11E080912F0C8730F6
:10C5000009F010E060911C0770911D0780911E07D3
:10C5100090911F070E94334F67E0661900E09C016D
:10C520004CE757E05DCD8091280C1092280C8823B1
:10C53000F1F20F948D9844EB54E86CE177E08CE7CE
:10C5400097E00F94B29A80912A0C882381F2B4CD9F
:10C550008091280C1092280C882309F450CE0F9457
:10C560008D9801EF13E62CE231E046E950E062E0FD
:10C5700072E08DE697E00F94059A80912A0C88234B
:10C5800009F43DCE99CD8091280C1092280C882377
:10C5900009F460CD0F948D9850E040E06CE87CE0A9
:10C5A0008CE897E00F94B29A80912A0C882309F4C2
:10C5B00051CD82CD8AE0781266C08FEF8093450C12
:10C5C00080912F0C8A30D9F080917A02882309F467
:10C5D0005DCD11E080912F0C8A3009F010E0609160
:10C5E00020077091210780912207909123070E94D4
:10C5F0003C3800E09C0144E857E0632D44CD809135
:10C60000280C1092280C8823F9F20F948D9820E0C2
:10C6100030E048EC52E4609120077091210780914E
:10C620002207909123070F94A1BB20E030E0A901DD
:10C630000F942DC220E030E040E85FE30F942CC25D
:10C640000F94A0C31F9285E9882E8BE3982E9DE45A
:10C65000A92E90E4B92E6B0117E5E12E1EE3F12E11
:10C660000FE010E021E030E040E050E060E277E0F1
:10C6700084E897E00E94F28D0F9080912A0C882325
:10C6800009F4A2CF19CD8BE07812C1CE8FEF809341
:10C69000450C80912F0C8B30D9F080917A02882341
:10C6A00009F4F4CC11E080912F0C8B3009F010E0EC
:10C6B00060911C0770911D0780911E0790911F07C4
:10C6C0000E94334F00E09C014CE757E0642DDBCC27
:10C6D0008091280C1092280C8823F9F20F948D98E1
:10C6E0004EE75BE36CE177E08CE797E00F94B29A5A
:10C6F00080912A0C882389F2DFCC8091280C10923B
:10C70000280C882309F48ECE0F948D980EEE13E634
:10C710002CE830E046E450E060E072E08DE697E01F
:10C720000F94059A80912A0C882309F47BCEC4CCFF
:10C7300083E0781609F493CD84E0781201CC8091DF
:10C740002F0C843009F4BFCD80917A02882309F43C
:10C7500020CD14E01619FF24F39480912F0C84301F
:10C7600009F0F12C8090310290903202A0903302B7
:10C77000B090340220E030E0A901C501B4010F946B
:10C780003BBB2DEB37E346E055EB87FD04C02DEBBB
:10C7900037E346E055E3C501B4010F942DC2698328
:10C7A0007A838B839C83CE0101960F94921700E0CD
:10C7B0009C0144E957E0612F8F2DB4CC0C9419EB08
:10C7C0000C9419EB0C9419EB0C9419EB0C94CBEA28
:10C7D0000C94CBEA0C94CBEA0C94CBEA8FEF0C943C
:10C7E000578D8091450C0C94578DEF92FF920F93CB
:10C7F0001F93CF93DF9300D000D000D01F921F92E1
:10C80000CDB7DEB77C012091310C422F022E000CF7
:10C81000550B8091320C833079F1843031F180E511
:10C820009AE05F932F939F938F938E010F5F1F4F1B
:10C830001F930F930F94D2BAC7010E94BFEAC80199
:10C840000E94468C0F900F900F900F900F900F90BA
:10C850002B960FB6F894DEBF0FBECDBFDF91CF9100
:10C860001F910F91FF90EF9008958CE59AE027FDBE
:10C87000D8CF87E49AE0D5CF85E69AE0D2CFE09191
:10C88000450C85E1E802F0011124E35DF64E868156
:10C8900097810C94F563E091450C86E0E802F00185
:10C8A0001124EA5EF34F808191810C94F5630F931C
:10C8B0001F93CF93DF938C01EB019091E5192091A9
:10C8C000E619921305C00F94E01B0F94AF09F5CF42
:10C8D0008091E41934E0839FF0011124E951F64E70
:10C8E00011830083D383C2839F5F9093E5198F5F89
:10C8F000281739F08093E419DF91CF911F910F91A0
:10C9000008951092E419F8CFCF92DF92EF92FF9240
:10C910006B017C0120E030E0A9010F943BBB87FD57
:10C9200026C06DEB77E386E095E3A70196010F94AF
:10C930002DC26B017C0120E030E0A9010F943BBBCC
:10C9400020E030E040E05FE387FF04C020E030E01B
:10C9500040E05FEBC701B6010F942DC20F9499C35D
:10C96000CB01FF90EF90DF90CF900D9407196DEB06
:10C9700077E386E095EBD9CF0F9442BB20E030E01F
:10C98000A9010F942DC20C9484643F924F925F9240
:10C990006F927F928F929F92AF92BF92CF92DF92CF
:10C9A000EF92FF920F931F93CF93DF9361E081E0AB
:10C9B0000E946E8CC091300CA5E04A2E4C0ED4E043
:10C9C000DC1B83E0782E7C1A82E0682E6C1A81E0F2
:10C9D000582E5C1A3C2E3194C11138C080912F0C16
:10C9E0008823B1F080917A02882359F081E09091F8
:10C9F0002F0C911180E024E043E958E0632D0F945F
:10CA00003297CF5FC411E8CF85E08093290C0CC02A
:10CA10008091280C1092280C882321F30E94B48D59
:10CA200080912A0C8823F1F2DF91CF911F910F9111
:10CA3000FF90EF90DF90CF90BF90AF909F908F903E
:10CA40007F906F905F904F903F900895C13009F0B4
:10CA50005DC080912F0C8130E9F080917A028823AB
:10CA600081F211E080912F0C813009F010E060918B
:10CA7000840D7091850D8091860D9091870D0E9497
:10CA8000846400E09C0142E358E0652D812F0E9400
:10CA9000F49AB7CF8091280C1092280C8823E9F2E1
:10CAA0000F948D9820E030E0A9016091840D709181
:10CAB000850D8091860D9091870D0F942DC220E0F9
:10CAC00030E040E85FE30F942CC20F94A0C31F92A4
:10CAD000912C812CE3E2AE2EE0E4BE2E6B011DED25
:10CAE000E12E13E0F12E00E010E021E030E040E024
:10CAF00050E064E87DE082E398E00E94F28D0F90C0
:10CB000080912A0C882309F4A8CF8ECFC23009F077
:10CB1000FEC080912F0C8230D9F080917A02882358
:10CB200009F46FCF11E080912F0C823009F010E0F2
:10CB30006091880D7091890D80918A0D90918B0D77
:10CB40000E94846400E09C014AE258E0662D9ECF7A
:10CB50008091280C1092280C8823F9F20F948D985C
:10CB600020E030E0A9016091880D7091890D8091DD
:10CB70008A0D90918B0D0F942DC220E030E040E89B
:10CB80005FE30F942CC20F94A0C31F92912C812CB1
:10CB900043E2A42E40E4B42E6B011DEDE12E13E020
:10CBA000F12E00E010E021E030E040E050E068E8E5
:10CBB0007DE08AE298E00E94F28D0F9080912A0C2D
:10CBC000882309F4AACF30CF80912F0C8330D9F07D
:10CBD00080917A02882309F414CF11E080912F0C00
:10CBE000833009F010E060918C0D70918D0D809173
:10CBF0008E0D90918F0D0E943C3800E09C0142E226
:10CC000058E0672D43CF8091280C1092280C882380
:10CC1000F9F20F948D9820E030E048EC52E46091F6
:10CC20008C0D70918D0D80918E0D90918F0D0F94C4
:10CC3000A1BB20E030E0A9010F942DC220E030E03C
:10CC400040E251E40F942CC20F94A0C31F92912C88
:10CC5000812C2DE4A22E20E4B22E6B011EEAE12EDF
:10CC600012E8F12E01E010E02AE030E040E050E070
:10CC70006CE87DE082E298E00E94F28D0F90809156
:10CC80002A0C882309F4A4CFCFCE8091280C1092CF
:10CC9000280C882309F446C00F948D9820E030E0DA
:10CCA00048EC52E46091900D7091910D8091920D3D
:10CCB0009091930D0F94A1BB20E030E0A9010F9457
:10CCC0002DC220E030E040E251E40F942CC20F94DA
:10CCD000A0C31F92912C812C8DE4A82E80E4B82E45
:10CCE0006B011EEAE12E12E8F12E01E010E02AE0CD
:10CCF00030E040E050E060E97DE08AE198E00E94A9
:10CD0000F28D0F9080912A0C882361F08DCEC33074
:10CD100009F45ACFC43009F074CE80912F0C8430BE
:10CD200009F4B3CF80917A02882309F46ACE11E026
:10CD300080912F0C843009F010E06091900D70917B
:10CD4000910D8091920D9091930D0E943C3800E0DE
:10CD50009C014AE158E06D2F99CECF93DF93EC010F
:10CD60000E94CB8D20E040E070E060E0CE01DF91DA
:10CD7000CF910C94CC8C2F923F924F925F926F92F6
:10CD80007F928F929F92AF92BF92CF92DF92EF925B
:10CD9000FF920F931F93CF93DF9300D01F92CDB7D5
:10CDA000DEB761E081E00E946E8C8091300C8B8355
:10CDB000282E8B5F8983922D91959A8388E0782E17
:10CDC000721887E0682E621886E0582E521885E0A7
:10CDD000482E421882E0382E321881E082198C8366
:10CDE0009B81911113C080912F0C882361F1809158
:10CDF0007A02882359F081E090912F0C911180E004
:10CE000024E043EE55E16A810F9432978091820CC1
:10CE1000882309F44DC08B81813009F06EC0909158
:10CE20002F0C913099F180917A02882309F4B2C0D5
:10CE300081E0913009F080E020E24FEC55E16C8117
:10CE40000F943297A7C08091280C1092280C882349
:10CE500071F20E94B48D80912A0C882341F20F90C8
:10CE60000F900F900F90DF91CF911F910F91FF9036
:10CE7000EF90DF90CF90BF90AF909F908F907F907A
:10CE80006F905F904F903F902F9008958091280C65
:10CE90001092280C882339F22EED35E13093D30B14
:10CEA0002093D20B80912A0C882309F4BCCFD7CFD2
:10CEB0009B81913011F590912F0C913069F0809108
:10CEC0007A02882309F466C081E0913009F080E09D
:10CED00020E24DEB55E1B3CF8091280C1092280C45
:10CEE000882369F32AEC35E13093D30B2093D20BDE
:10CEF00080912A0C882319F3B2CF8B81823019F5E7
:10CF000080912F0C823081F080917A02882309F47D
:10CF100041C081E090912F0C923009F080E023E035
:10CF20004CEA55E1632D8CCF8091280C1092280C8F
:10CF3000882351F38BEF98E60E94AD6680912A0C0E
:10CF4000882311F38CCF9B81933009F034C18091F9
:10CF50002F0C833009F45CC080917A028823D1F0D1
:10CF600088EB9BE39F938F9382EA95E19F938F9346
:10CF700083E082198F9381E090912F0C933009F018
:10CF800080E08F930E94388C0F900F900F900F903D
:10CF90000F900F9080917E0C90917F0CA091800C4F
:10CFA000B091810C8093330C9093340CA093350C8A
:10CFB000B093360C8B81883009F580912F0C883026
:10CFC00009F4C2C080917A028823C1F011E08091F7
:10CFD0002F0C883009F010E06091330C7091340C04
:10CFE0008091350C9091360C0E94846400E09C0185
:10CFF0004AE555E1672D812F0E94F49A9B819F5F3E
:10D000009B8389819813ECCE89E08093290C27CFEC
:10D010008091280C1092280C882309F49DCF0E943F
:10D02000B83B80912A0C882309F496CF18CF8091C1
:10D030002F0C843089F080917A02882309F4AACFDA
:10D0400064E0621981E090912F0C943009F080E047
:10D0500023E045E955E1F4CE8091280C1092280C8C
:10D06000882349F38DEF96E40E94AD6680912A0CE7
:10D07000882309F3F4CE80912F0C853009F180913B
:10D080007A02882361F081E090912F0C953009F0AD
:10D0900080E023E045E855E1642D0F9432978091BC
:10D0A0007E0C90917F0CA091800CB091810C8093AC
:10D0B000330C9093340CA093350CB093360C9ECF68
:10D0C0008091280C1092280C8823C9F282E89CE3F6
:10D0D0000E94AD6680912A0C882389F2C0CE80918F
:10D0E0002F0C863079F080917A028823C1F281E09A
:10D0F00090912F0C963009F080E023E04BE755E14A
:10D10000652D9ECE8091280C1092280C882359F30F
:10D110008AE69AE60E94AD6680912A0C882319F36C
:10D120009ECE8091280C1092280C882309F455C0BB
:10D1300026E735E13093D30B2093D20B80912A0C54
:10D14000882309F44AC08BCE8091280C1092280CB9
:10D15000882309F437CF0F948D9820E030E0A9019F
:10D160006091330C7091340C8091350C9091360C99
:10D170000F942DC20F94A0C31F9281E7882E80E4E4
:10D18000982E93E2A92E90E4B92E6B0114E6E12EBD
:10D19000F12C00E010E020E030E0A90163E37CE046
:10D1A0008AE595E10E94F28D0F9080912A0C8823E8
:10D1B00009F408CF54CE9B81943009F438CF9530D0
:10D1C00009F459CF963009F48ACF973009F0E2CEAE
:10D1D00090912F0C973009F4A4CF80917A02882384
:10D1E00009F45DCF81E0973009F080E020E246E667
:10D1F00055E1662D25CE9F92AF92BF92CF92DF92DE
:10D20000EF92FF920F931F93CF93DF9361E081E042
:10D210000E946E8CC091300CCC2E85E0982E9C0E16
:10D2200093EFA92E96E4B92ED7E0DC1B16E01C1B69
:10D2300005E00C1B84E0F82EFC1A82E0E82EEC1AC4
:10D2400081E0D82EDC1AC11133C080912F0C8823C5
:10D25000B9F080917A02882361F06C2D619581E0AC
:10D2600090912F0C911180E024E045E455E10F945A
:10D270003297CF5FC911E7CF88E08093290C0CC0AB
:10D280008091280C1092280C882319F30E94B48DE9
:10D2900080912A0C8823E9F2DF91CF911F910F91A1
:10D2A000FF90EF90DF90CF90BF90AF909F90089548
:10D2B000C13011F590912F0C913069F080917A0274
:10D2C0008823B9F281E0913009F080E020E24BE25E
:10D2D00055E16D2DCCCF8091280C1092280C88231D
:10D2E00069F32EE335E13093D30B2093D20B809179
:10D2F0002A0C882319F3D0CFC23009F0BDC0909119
:10D300002F0C923071F080917A02882309F4B1CF0A
:10D3100081E0923009F080E020E242E155E16E2D9B
:10D32000A6CF8091280C1092280C882361F323E269
:10D3300035E13093D30B2093D20B80912A0C8823B4
:10D3400011F3AACF80912F0C833089F080917A025B
:10D35000882309F48ECF63E06C1981E090912F0C43
:10D36000933009F080E023E041E055E180CF8091E7
:10D37000280C1092280C882349F384E594E40E9439
:10D38000AD6680912A0C882309F386CF90912F0CEB
:10D39000943071F080917A02882309F46ACF81E099
:10D3A000943009F080E020E245EE54E16F2D5FCF2C
:10D3B0008091280C1092280C882361F326EF34E129
:10D3C0003093D30B2093D20B80912A0C882311F336
:10D3D00063CF80912F0C853081F080917A02882371
:10D3E00009F447CF81E090912F0C953009F080E04F
:10D3F00023E044ED54E1602F3ACF8091280C109245
:10D40000280C882351F384E594E40E94AD66809152
:10D410002A0C882311F340CF90912F0C963071F095
:10D4200080917A02882309F424CF81E0963009F0B4
:10D4300080E020E248EB54E1612F19CF8091280C65
:10D440001092280C882361F329EC34E13093D30B3C
:10D450002093D20B80912A0C882311F31DCF809149
:10D46000280C1092280C8823C9F00E94F346809162
:10D470002A0C882399F010CFC33009F463CFC4304D
:10D4800009F484CFC53009F4A4CFC63029F2C730DF
:10D4900009F0EFCE80912F0C873009F380917A024A
:10D4A000882309F4E6CEBF92AF9287EA94E19F9376
:10D4B0008F93DF9381E090912F0C973009F080E0FB
:10D4C0008F930E94388C0F900F900F900F900F90B9
:10D4D0000F90CFCEAF92BF92CF92DF92EF92FF929A
:10D4E0000F931F93CF93DF9361E081E00E946E8CD6
:10D4F000C091300C85E0B82EBC0ED5E0DC1B14E0EA
:10D500001C1B03E00C1B9BE8C92E94E1D92E82E082
:10D51000F82EFC1A81E0E82EEC1AAC2EA194C11171
:10D5200031C080912F0C8823B1F080917A0288233A
:10D5300059F081E090912F0C911180E024E045E4B6
:10D5400055E16A2D0F943297CF5FCB11E8CF86E07B
:10D550008093290C0CC08091280C1092280C8823F1
:10D5600021F30E94B48D80912A0C8823F1F2DF917F
:10D57000CF911F910F91FF90EF90DF90CF90BF90D0
:10D58000AF900895C13011F580912F0C813079F062
:10D5900080917A028823C1F281E090912F0C913022
:10D5A00009F080E023E04CE954E16E2DCBCF80916F
:10D5B000280C1092280C882359F38BE79BE60E94D5
:10D5C000AD6680912A0C882319F3D1CFC23009F0BF
:10D5D00076C090912F0C923071F080917A0288235E
:10D5E00009F4B2CF81E0923009F080E020E247E711
:10D5F00054E16F2DA7CF8091280C1092280C88231E
:10D6000061F3D092D30BC092D20B80912A0C882365
:10D6100021F3ADCF80912F0C833081F080917A027D
:10D62000882309F491CF81E090912F0C933009F079
:10D6300080E023E049E654E1602F84CF8091280CFC
:10D640001092280C882351F384E594E40E94AD667F
:10D6500080912A0C882311F38ACF80912F0C84307B
:10D6600081F080917A02882309F46ECF81E0909155
:10D670002F0C943009F080E023E04FE554E1612F56
:10D6800061CF8091280C1092280C882351F38AE4F2
:10D690009DE60E94AD6680912A0C882311F367CF26
:10D6A0008091280C1092280C8823A9F08EE49EE625
:10D6B0000E94AD6680912A0C882369F058CFC33050
:10D6C00009F4A8CFC43049F2C53009F03DCF8091AC
:10D6D0002F0C853029F380917A02882309F434CF06
:10D6E00081E090912F0C953009F080E023E041E536
:10D6F00054E16D2F27CF9F92AF92BF92CF92DF92CE
:10D70000EF92FF920F931F93CF93DF9361E081E03D
:10D710000E946E8CC091300CDC2F85E0982E9C0E00
:10D720009FE4A92E9DE8B92E19E01C1B08E00C1BF4
:10D7300087E0F82EFC1A86E0E82EEC1A85E0D82E59
:10D74000DC1A84E0C82ECC1AC11133C080912F0C92
:10D750008823B9F080917A02882361F06D2F61955A
:10D7600081E090912F0C911180E024E04BE755E18E
:10D770000F943297CF5FC911E7CF8AE08093290CCD
:10D780000CC08091280C1092280C882319F30E9459
:10D79000B48D80912A0C8823E9F2DF91CF911F91FB
:10D7A0000F91FF90EF90DF90CF90BF90AF909F9040
:10D7B0000895C13041F5EBECFCE68591949190938E
:10D7C000470C8093460C90912F0C913059F080912A
:10D7D0007A02882379F261E06D1B81E0913061F17A
:10D7E00080E02AC08091280C1092280C882379F3BD
:10D7F0002DE533E13093D30B2093D20B80912A0C8B
:10D80000882329F3CACFC23009F00FC1EDECFCE642
:10D81000859194919093470C8093460C90912F0C96
:10D82000923071F080917A02882309F4A3CF62E0EC
:10D830006D1B81E09230A1F620E24EE453E198CFD7
:10D840008091280C1092280C882361F328E233E1A0
:10D850003093D30B2093D20B80912A0C882311F3A1
:10D860009CCF80912F0C833089F080917A0288239D
:10D8700009F480CF63E06D1B81E090912F0C933011
:10D8800009F080E023E046E153E172CF8091280C5B
:10D890001092280C882349F380EB95E40E94AD6632
:10D8A00080912A0C882309F378CF90912F0C943023
:10D8B00071F080917A02882309F45CCF81E0943082
:10D8C00009F080E020E24FEF52E16C2D51CF8091C2
:10D8D000280C1092280C882361F32FE033E1309359
:10D8E000D30B2093D20B80912A0C882311F355CFB0
:10D8F00080912F0C853081F080917A02882309F481
:10D9000039CF81E090912F0C953009F080E023E031
:10D9100042EF52E16D2D2CCF8091280C1092280CF3
:10D92000882351F389E49DE30E94AD6680912A0C1F
:10D93000882311F332CF90912F0C963071F08091A3
:10D940007A02882309F416CF81E0963009F080E04E
:10D9500020E249ED52E16E2D0BCF8091280C109200
:10D96000280C882361F32BEE32E13093D30B209304
:10D97000D20B80912A0C882311F30FCF80912F0CAA
:10D980008730B1F080917A02882309F4F3CE87E4DE
:10D9900098E49F938F938AEC92E19F938F93FF92E9
:10D9A00081E090912F0C973009F46AC080E068C044
:10D9B0008091280C1092280C882321F30E9447485C
:10D9C00080912A0C8823F1F2E8CE90912F0C9830A8
:10D9D00071F080917A02882309F4CCCE81E09830EE
:10D9E00009F080E020E242EB52E1602FC1CE80914D
:10D9F000280C1092280C882361F325EC32E1309337
:10DA0000D30B2093D20B80912A0C882311F3C5CE1F
:10DA10008091280C1092280C882301F10E944F8DD0
:10DA200080912A0C8823D1F0B8CEC33009F419CFE5
:10DA3000C43009F43ACFC53009F45ACFC63009F4DE
:10DA40007ACFC73009F49ACFC83009F4BECFC930B5
:10DA500009F090CE80912F0C8930D1F280917A021A
:10DA6000882309F487CEBF92AF9286EA92E19F9312
:10DA70008F931F9381E090912F0C993009F096CFEE
:10DA80008F930E94388C0F900F900F900F900F90F3
:10DA90000F9070CE5F926F927F928F929F92AF9213
:10DAA000BF92CF92DF92EF92FF920F931F93CF938B
:10DAB000DF9361E081E00E946E8CC091300C85E0C4
:10DAC000682E6C0E9FE4E92E9DE8F92E26EAC22E00
:10DAD00022E1D22ED4E0DC1B13E01C1B34E9A32E80
:10DAE00031E1B32E02E00C1B49EA842E41E1942E71
:10DAF00081E0782E7C1A5C2E5194C11136C0809141
:10DB00002F0C8823B1F080917A02882359F081E0AC
:10DB100090912F0C911180E024E04BE755E1652DA9
:10DB20000F943297CF5FC611E8CF85E08093290C20
:10DB30000CC08091280C1092280C882321F30E949D
:10DB4000B48D80912A0C8823F1F2DF91CF911F913F
:10DB50000F91FF90EF90DF90CF90BF90AF909F908C
:10DB60008F907F906F905F900895C13001F59091F4
:10DB70002F0C913069F080917A02882399F281E02C
:10DB8000913009F080E020E24BE951E1672DC8CFE8
:10DB90008091280C1092280C882369F39092D30B63
:10DBA0008092D20B80912A0C882329F3CECFC230E9
:10DBB00009F051C090912F0C923071F080917A024F
:10DBC000882309F4AFCF81E0923009F080E020E2B1
:10DBD00042E851E1602FA4CF8091280C1092280CCC
:10DBE000882361F3B092D30BA092D20B80912A0CC0
:10DBF000882321F3AACF80912F0C833081F080916C
:10DC00007A02882309F48ECF81E090912F0C933013
:10DC100009F080E023E04FE651E1612F81CF809150
:10DC2000280C1092280C882351F385E69EE30E946D
:10DC3000AD6680912A0C882311F387CF8091280C40
:10DC40001092280C882381F00E944F8D80912A0C1D
:10DC5000882351F07ACFC33071F2C43009F062CF1B
:10DC600080912F0C843051F380917A02882309F43B
:10DC700059CFFF92EF92DF92CF92DF9381E09091A4
:10DC80002F0C943009F080E08F930E94388C0F9015
:10DC90000F900F900F900F900F9044CF8F929F9204
:10DCA000AF92BF92CF92DF92EF92FF920F931F93AA
:10DCB000CF93DF9361E081E00E946E8CC091300CC5
:10DCC00085E0982E9C0E9FE4E92E9DE8F92E26EA29
:10DCD000C22E22E1D22ED3E0DC1B12E01C1B35E465
:10DCE000A32E32E1B32E01E00C1B8C2E8194C111C6
:10DCF00033C080912F0C8823B1F080917A02882361
:10DD000059F081E090912F0C911180E024E04BE7D5
:10DD100055E1682D0F943297CF5FC911E8CF84E0A9
:10DD20008093290C0CC08091280C1092280C882319
:10DD300021F30E94B48D80912A0C8823F1F2DF91A7
:10DD4000CF911F910F91FF90EF90DF90CF90BF90F8
:10DD5000AF909F908F900895C13001F590912F0C56
:10DD6000913069F080917A028823B1F281E091309C
:10DD700009F080E020E244E352E1602FCBCF8091B4
:10DD8000280C1092280C882369F3B092D30BA09230
:10DD9000D20B80912A0C882329F3D1CFC23081F590
:10DDA00080912F0C823081F080917A02882309F4CF
:10DDB000B3CF81E090912F0C923009F080E023E006
:10DDC00041E252E1612FA6CF8091280C1092280CDD
:10DDD000882351F387E393E40E94AD6680912A0C77
:10DDE000882311F3ACCF8091280C1092280C882343
:10DDF00071F00E944F8D80912A0C882341F09FCFB3
:10DE0000C33009F089CF80912F0C833061F380916A
:10DE10007A02882309F480CFFF92EF92DF92CF92AB
:10DE2000DF9381E090912F0C933009F080E08F9385
:10DE30000E94388C0F900F900F900F900F900F90C2
:10DE40006BCF7F928F929F92AF92BF92CF92DF92D1
:10DE5000EF92FF920F931F93CF93DF9361E081E0E6
:10DE60000E946E8CC091300C9C2E85E0A82EAC0ECA
:10DE7000D7E0DC1BBB24B39486E0F82EFC1A85E0C7
:10DE8000E82EEC1A84E0D82EDC1A82E0C82ECC1AD8
:10DE90008B2C8C1A7C2E7194C11150C080912F0C48
:10DEA000882391F180917A02882359F081E0909142
:10DEB0002F0C911180E024E046E151E1672D0F9491
:10DEC00032978091AC0D8093330CC43009F056C06A
:10DED0001092450C80912F0C843009F4E8C0809199
:10DEE0007A02882309F489C111E080912F0C8430D3
:10DEF00009F010E08091330C0F943C1900E09C0174
:10DF000049EF50E16D2D37C08091280C1092280CFC
:10DF1000882341F20E94B48D80912A0C882311F24B
:10DF2000DF91CF911F910F91FF90EF90DF90CF90F5
:10DF3000BF90AF909F908F907F900895C13009F06F
:10DF400061C080912F0C813009F443C080917A0226
:10DF50008823A1F011E080912F0C813009F010E0AE
:10DF600080917C0290917D020F94071900E09C0142
:10DF700040E151E1682D812F0E94F49A8091AD0D0E
:10DF80008093330CC53009F0BCC0B092450C809131
:10DF90002F0C853009F4A0C080917A02882391F07B
:10DFA00011E080912F0C853009F010E08091330C46
:10DFB0000F943C1900E09C0149EF50E16E2D812F38
:10DFC0000E94F49ACF5FAC1267CF88E08093290C4F
:10DFD000A7CF8091280C1092280C882309F4B6CF83
:10DFE00010E000E027EE33E04AE050E06CE772E03A
:10DFF00080E191E10F94059A80912A0C882309F41D
:10E00000A5CF8ECFC23009F0D8C080912F0C8230BE
:10E01000D1F080917A02882309F4B0CF11E0809189
:10E020002F0C823009F010E080913319909134194F
:10E030000F94071900E09C0149E051E16C2D812FFC
:10E040000E94F49A3ECF8091280C1092280C8823CD
:10E0500001F30F948D9801ED1AE42CE231E050E0C9
:10E0600040E063E379E189E091E10F94059A8091C2
:10E070002A0C882371F254CF8091280C1092280C1E
:10E08000882309F4A2C00F948D980DEC14ED2CE8B0
:10E0900030E050E040E069E87CE085E091E10F94F9
:10E0A000059A80912A0C882309F48FC039CF80917A
:10E0B000280C1092280C882309F411CF0F948D9806
:10E0C00062EC77E389EF90E10F94FE9A80912A0C3D
:10E0D000882309F404CF24CF8091280C1092280CB7
:10E0E000882309F459CF0F948D9862EC77E389EF78
:10E0F00090E10F94FE9A80912A0C882309F44CCF6A
:10E100000FCFC63091F580912F0C8630B9F08091F9
:10E110007A02882309F456CF11E080912F0C8630C3
:10E1200009F010E08091390290913A020F9407199A
:10E1300000E09C0144EF50E16F2D41CF8091280C0D
:10E140001092280C882319F30FE917E327EE33E028
:10E150004AE050E069E372E084EF90E10F94059AA1
:10E1600080912A0C882399F2DBCEC73009F02ACFA0
:10E1700080912F0C873091F080917A02882309F4E6
:10E1800021CF81E090912F0C973009F080E023E0BF
:10E1900045EE50E16D2F0F94329714CF8091280CEB
:10E1A0001092280C882341F389EC99E90E94AD660E
:10E1B00080912A0C882301F3B3CEC33009F081CEBD
:10E1C00080912F0C833009F457CF80917A028823F5
:10E1D00009F4D4CE11E080912F0C833009F010E0C7
:10E1E0008091890C90918A0C0F94071963E069194A
:10E1F00000E09C0145E051E122CF8091AD0D80937C
:10E20000330CE0CE5F926F927F928F929F92AF928B
:10E21000BF92CF92DF92EF92FF920F931F93CF9313
:10E22000DF93FF24F3948091331990913419892B53
:10E2300009F4F12C61E081E00E946E8CC091300CF9
:10E240008C2E95E0992E9C0EAA24A39484E0E82EAF
:10E25000EC1A83E0D82EDC1A82E0C82ECC1A7A2C75
:10E260007C1A6C2E619487E0B82EBC1AC111B8C01C
:10E2700080912F0C882309F495C080917A0288231D
:10E2800059F081E090912F0C911180E024E040EE54
:10E2900050E1662D0F9432978091AD0D8093330C31
:10E2A000C430E9F4A092450C80912F0C843009F41D
:10E2B00045C180917A02882391F0D1E080912F0CA2
:10E2C000843009F0D0E08091330C0F943C1900E0C9
:10E2D0009C0149EC50E16E2D8D2F0E94F49A10E0C4
:10E2E00000E0D5E05C2E58180093330CCD131FC00E
:10E2F000F801EE0FFF1FE553F34985919491909338
:10E30000470C8093460C80912F0C8C1709F42BC17D
:10E3100080917A02882359F081E090912F0C9D130F
:10E3200080E023E04FEB50E1652D0F9432978D2F65
:10E330000F5F1F4FD6E08630B9F68091890C90911F
:10E340008A0C892B19F4FF2009F42DC1C73009F577
:10E3500080912F0C873009F417C180917A028823AD
:10E36000C1F083ED9AE49F938F9386EB90E19F93A6
:10E370008F93BF9281E090912F0C973009F080E04D
:10E380008F930E94388C0F900F900F900F900F90EA
:10E390000F9088E0FF24F394CF5FC91167CF80937B
:10E3A000290C0EC08091280C1092280C882309F4A7
:10E3B00064CF0E94B48D80912A0C882309F45DCF2C
:10E3C000DF91CF911F910F91FF90EF90DF90CF9051
:10E3D000BF90AF909F908F907F906F905F900895C7
:10E3E000C13009F05FC080912F0C813009F43FC02B
:10E3F00080917A02882309F44FCFD1E080912F0CCD
:10E40000813009F0D0E080913319909134190F9444
:10E41000071900E09C0149ED50E1672D8D2F0E9406
:10E42000F49A8091AC0D8093330CC33009F034CF53
:10E430001092450C80912F0C833009F46AC08091B2
:10E440007A02882309F44BCFD1E080912F0C8330DE
:10E4500009F0D0E08091330C0F943C1900E09C014E
:10E4600049EC50E16D2D8D2F0E94F49A15CF8091CB
:10E47000280C1092280C882309F4BACF0F948D9899
:10E480000FEC1AE42CE231E050E040E063E379E184
:10E4900089ED90E10F94059A80912A0C882309F464
:10E4A000A7CF8ECFC23009F0BCCF80912F0C823025
:10E4B000B9F080917A02882309F4EECED1E0809100
:10E4C0002F0C823009F0D0E08091890C90918A0C59
:10E4D0000F94071900E09C0145ED50E16C2D9ECF93
:10E4E0008091280C1092280C882319F30F948D9892
:10E4F0000DEC14ED2CE830E050E040E069E87CE001
:10E5000085ED90E10F94059A80912A0C882389F279
:10E5100057CF8091280C1092280C882309F48FCFB4
:10E520000F948D9862EC77E389EC90E10F94FE9A5A
:10E5300080912A0C882309F482CF42CF8091280C45
:10E540001092280C882309F4B4CE0F948D9862ECB5
:10E5500077E389EC90E10F94FE9A80912A0C88234E
:10E5600009F4A7CE2DCF8091280C1092280C882377
:10E5700009F4CECE8EED9AE40E94AD6680912A0C0D
:10E58000882309F4C5CE1CCF8091280C1092280C4A
:10E59000882309F4E2CE0E94D34A80912A0C882372
:10E5A00009F4DBCE0DCF87E0F7CE9F92AF92BF92FA
:10E5B000CF92DF92EF92FF920F931F93CF93DF934F
:10E5C00061E081E00E946E8CC091300CDC2F85E010
:10E5D000982E9C0E98E1A92E90E1B92E19E01C1BF3
:10E5E00008E00C1B87E0F82EFC1A86E0E82EEC1AF7
:10E5F00085E0D82EDC1A84E0C82ECC1AC11133C0B5
:10E6000080912F0C8823B9F080917A02882361F0E1
:10E610006D2F619581E090912F0C911180E024E0A5
:10E6200049E850E10F943297CF5FC911E7CF8AE0F4
:10E630008093290C0CC08091280C1092280C882300
:10E6400019F30E94B48D80912A0C8823E9F2DF919E
:10E65000CF911F910F91FF90EF90DF90CF90BF90DF
:10E66000AF909F900895C13019F580912F0C8130A3
:10E6700081F080917A028823B9F261E06D1B81E01C
:10E6800090912F0C913009F080E023E043EA5CE6A2
:10E69000C9CF8091280C1092280C882351F388E868
:10E6A00094E70E94AD6680912A0C882311F3CFCFA6
:10E6B000C23009F006C190912F0C923079F0809110
:10E6C0007A02882309F4B0CF62E06D1B81E09230BA
:10E6D00009F080E020E24FE750E1A4CF8091280CC0
:10E6E0001092280C882359F328E034E13093D30B9F
:10E6F0002093D20B80912A0C882309F3A8CF909104
:10E700002F0C933079F080917A02882309F48CCF12
:10E7100063E06D1B81E0933009F080E020E243E785
:10E7200050E180CF8091280C1092280C882359F357
:10E730002AE730E13093D30B2093D20B80912A0C3F
:10E74000882309F384CF90912F0C943071F080913D
:10E750007A02882309F468CF81E0943009F080E0E0
:10E7600020E247E650E16C2D5DCF8091280C10929D
:10E77000280C882361F32EE630E13093D30B2093ED
:10E78000D20B80912A0C882311F361CF90912F0C2A
:10E79000953071F080917A02882309F445CF81E0A9
:10E7A000953009F080E020E24BE550E16D2D3ACF45
:10E7B0008091280C1092280C882361F322E630E126
:10E7C0003093D30B2093D20B80912A0C882311F322
:10E7D0003ECF80912F0C863081F080917A02882381
:10E7E00009F422CF81E090912F0C963009F080E05F
:10E7F00023E046E450E16E2D15CF8091280C109255
:10E80000280C882351F38BEB96E60E94AD6680912D
:10E810002A0C882311F31BCF80912F0C873081F0B5
:10E8200080917A02882309F4FFCE81E090912F0C29
:10E83000973009F080E023E048E350E16F2DF2CEFD
:10E840008091280C1092280C882351F389EE9BE4C8
:10E850000E94AD6680912A0C882311F3F8CE909126
:10E860002F0C983071F080917A02882309F4DCCE65
:10E8700081E0983009F080E020E24CE150E1602F27
:10E88000D1CE8091280C1092280C882361F32BE2C2
:10E8900030E13093D30B2093D20B80912A0C882344
:10E8A00011F3D5CE8091280C1092280C882311F1F9
:10E8B000B092D30BA092D20B80912A0C8823D1F076
:10E8C000C6CEC33009F41BCFC43009F43CCFC530E9
:10E8D00009F45CCFC63009F47CCFC73009F49CCF73
:10E8E000C83009F4BCCFC93009F09ECE90912F0CEE
:10E8F0009930C1F280917A02882309F495CE81E0A3
:10E90000993009F080E020E247E050E1612F8ACEA3
:10E91000AF92BF92CF92DF92EF92FF920F931F932D
:10E92000CF93DF9361E081E00E946E8CC091300C48
:10E9300085E0C82ECC0ED5E0DC1B93E0D92E14E088
:10E940001C1BBD2CBC1A82E0F82EFC1A81E0E82EBC
:10E95000EC1AAC2EA194C1112BC080912F0C8823EE
:10E9600081F080917A02882369F181E090912F0CE7
:10E97000911180E024E040E050E16A2D0F9432973D
:10E9800021C08091280C1092280C882351F30E94FA
:10E99000B48D80912A0C882321F3DF91CF911F91B0
:10E9A0000F91FF90EF90DF90CF90BF90AF900895C0
:10E9B000C130A1F590912F0C913059F080917A02DD
:10E9C000811119C0CF5FCC11C6CF86E08093290C8E
:10E9D000E4CF8091280C1092280C882379F3809141
:10E9E0003B028C2780933B02D0927A0280912A0CC2
:10E9F000882321F3D2CF81E0913009F080E090911B
:10EA00003B022FEE3FE0911102C02BEE3FE001E010
:10EA100042EF5FE06E2D0E94F49AD4CFC23009F02D
:10EA200077C080912F0C823079F080917A02882310
:10EA300049F281E090912F0C923009F080E023E0C0
:10EA400044EC5CE66F2D9ACF8091280C1092280C34
:10EA5000882359F384E19CE40E94AD6680912A0CDE
:10EA6000882319F39ACF80912F0C833081F0809105
:10EA70007A02882309F4A6CF81E090912F0C93307D
:10EA800009F080E023E04DEB5CE66B2D77CF8091C1
:10EA9000280C1092280C882351F38FE09CE40E94EC
:10EAA000AD6680912A0C882311F377CF80912F0CCB
:10EAB000843081F080917A02882309F483CF81E049
:10EAC00090912F0C943009F080E023E046EB5CE657
:10EAD000612F54CF8091280C1092280C882351F379
:10EAE0008AE09CE40E94AD6680912A0C882311F391
:10EAF00054CF8091280C1092280C8823A9F08FED18
:10EB00009BE30E94AD6680912A0C882369F045CF73
:10EB1000C33009F4A8CFC43049F2C53009F052CF50
:10EB200080912F0C853029F380917A02882309F493
:10EB300049CF81E090912F0C953009F080E023E0DF
:10EB40004DEA5CE66D2F1ACF3F924F925F926F9223
:10EB50007F928F929F92AF92BF92CF92DF92EF926D
:10EB6000FF920F931F93CF93DF93CDB7DEB7EB9751
:10EB70000FB6F894DEBF0FBECDBF80912F0788235C
:10EB800069F18091431A00E010E083FF23C08FE712
:10EB90009AE10E94C9E08BE1EFE7FAE1DE0191968C
:10EBA00001900D928A95E1F710E000E0BE016F5FE1
:10EBB0007F4FCE0181960F942D8518163CF4CE011F
:10EBC00001960E9405D9080F111DF0CFCE01819644
:10EBD0000F944736009334071093350761E081E0C6
:10EBE0000E946E8C1091300C412E85E0582E510EF3
:10EBF000312E31949DECA92E97E3B92E23EC822E71
:10EC00002FE0922E81E0682E611A111113C08091BD
:10EC10002F0C882339F180917A02882359F081E002
:10EC200090912F0C911180E024E047EC5FE0632D80
:10EC30000F9432978091431A85FD5BC083FF59C0C2
:10EC4000113009F054C080912F0C813079F18091FE
:10EC50007A02811138C082E01F5F5112D6CF8093B3
:10EC6000290C0CC08091280C1092280C882399F252
:10EC70000E94B48D80912A0C882369F2EB960FB61E
:10EC8000F894DEBF0FBECDBFDF91CF911F910F91E2
:10EC9000FF90EF90DF90CF90BF90AF909F908F90BC
:10ECA0007F906F905F904F903F9008958091280CD7
:10ECB0001092280C882359F20E94CD3780912A0C9B
:10ECC000882329F2DBCFBF92AF929F928F926F92EF
:10ECD00081E090912F0C913009F080E08F930E9499
:10ECE000388C0F900F900F900F900F900F9082E044
:10ECF00001C081E090917A02992309F4ADCF082FE9
:10ED0000D12CC12C712E7418802FE0903407F09014
:10ED10003507CE14DF0408F09FCF0113ACC081E0AB
:10ED2000E81AF108EC18FD088FE79AE10E94C9E0A3
:10ED30008BE1EFE7FAE1DE01919601900D928A9561
:10ED4000E1F7F12CBE016F5F7F4FCE0181960F94EA
:10ED50002D8518167CF4CE0101960E9405D98823D2
:10ED600089F3EF106BC0BE016F5F7F4F8AE49CE0B8
:10ED70000E9420D9CE0181960F9447369091431A74
:10ED800080912F0C94FF7CC0811366C09091280C59
:10ED90001092280C992309F45FC019821C8280917B
:10EDA000821A64E67AE1882311F06FE77AE121E0C4
:10EDB0004AE45CE0CE0101960F94781F882309F4A1
:10EDC0003FC08BE1FE013196AFE7BAE101900D92B1
:10EDD0008A95E1F78091431A8F7D8093431AA09121
:10EDE000381AAA3080F481E08A0F8093381A8BE1B8
:10EDF0008A9FD0011124A656B54EEFE7FAE10190A3
:10EE00000D928A95E1F7CE0101960F944736109244
:10EE1000300C82E090E0A0E0B0E080932B0C909367
:10EE20002C0CA0932D0CB0932E0C81E080932A0C17
:10EE300010922C0783E080937A0220CFF39482CF44
:10EE40000F9458596AE47CE08DEA9FE00F94435197
:10EE50008AE00F949745D7CF90917A02992359F081
:10EE6000FF24F3948113F12C6F2D872D0E94EF91D5
:10EE700041E0811118C08FEFC81AD80A0F5F44CF44
:10EE80008117B1F080917A028823A9F3FF24F394CB
:10EE900080912F0C8113F12C6F2D872D0E94EF9103
:10EEA000882349F340E0672D8F2D0F94D296E3CF4E
:10EEB0008091280C1092280C882321F385E79FE489
:10EEC0000E94AD6680912A0C8823E1F2D7CE2F9262
:10EED0003F924F925F926F927F928F929F92AF92EA
:10EEE000BF92CF92DF92EF92FF920F931F93CF9337
:10EEF000DF9300D000D0CDB7DEB70F94EC42582E90
:10EF00008091431A83FB222720F92983212C83FF38
:10EF100003C00F941943282E61E081E00E946E8C9B
:10EF20008091300C8D83782E8B5F8A8305E711E00A
:10EF30009BE3E92E9FE0F92E25E4C22E2FE8D22E86
:10EF40003FE4A32E3FE0B32E81E0482E471884E033
:10EF500087198B8383E087198C8382E0382E3718DA
:10EF600044EC842E4EE8942E9D81911143C18091F2
:10EF70002F0C882309F417C180917A02882361F04D
:10EF8000672D619581E090912F0C911180E024E034
:10EF900046E85FE00F943297511050C10F94274319
:10EFA000882309F4E5C18D81813009F007C2809181
:10EFB0002F0C813009F4B6C180917A028111C1C150
:10EFC00092E09E838E818F5F9D81891316C0809110
:10EFD0002F0C891709F402C280917A02882369F004
:10EFE0006D81671981E090912F0C2D81921380E043
:10EFF00023E044E35FE00F9432978E818E5F8E832F
:10F000009E812D81921316C080912F0C891709F4CF
:10F01000F6C180917A02882369F06D81671981E0D9
:10F0200090912F0C2D81921380E023E048E25FE065
:10F030000F9432978E818F5F9D81891316C08091C6
:10F040002F0C891709F4ECC180917A02882369F0AA
:10F050006D81671981E090912F0C2D81921380E0D2
:10F0600023E04AE15FE00F9432976E8063946394EB
:10F0700051101EC08D81681217C080912F0C9D8188
:10F08000891709F4DEC180917A02882369F06D81C5
:10F09000671981E090912F0C2D81921380E023E07D
:10F0A0004BE05FE00F94329783E0682E8E81680E0C
:10F0B0009D81691216C080912F0C861509F4D2C16A
:10F0C00080917A02882369F06D81671981E09091BF
:10F0D0002F0C2D81921380E023E04BEF5EE00F9424
:10F0E000329781E0860D9D81891316C080912F0C87
:10F0F000891709F4C8C180917A02882369F06D816B
:10F10000671981E090912F0C2D81921380E023E00C
:10F110004DEE5EE00F94329782E0860D51103AC0BA
:10F120009981992309F4E4C1211034C02D818213FF
:10F1300014C090912F0C921709F4B6C180917A02F5
:10F14000882359F06D81671981E02D81921380E049
:10F1500020E24CED5EE00F94329783E0860D9D81B6
:10F16000891316C080912F0C891709F4B0C18091C2
:10F170007A02882369F06D81671981E090912F0CE4
:10F180002D81921380E023E04BEC5EE00F943297E8
:10F1900084E0860D9D819F5F9D832A819213E4CE3A
:10F1A0008093290C0EC08091280C1092280C882383
:10F1B00009F4E2CE0E94B48D80912A0C882309F4D0
:10F1C000DBCE26960FB6F894DEBF0FBECDBFDF9123
:10F1D000CF911F910F91FF90EF90DF90CF90BF9054
:10F1E000AF909F908F907F906F905F904F903F90E7
:10F1F0002F900895552009F4D1CE2D81213071F53D
:10F2000080912F0C8130E9F080917A028823B1F04F
:10F210009F928F928AE79FE09F938F934F9281E016
:10F2200090912F0C913009F080E08F930E94388CE0
:10F230000F900F900F900F900F900F9095E09E837E
:10F24000DFCE8091280C1092280C8823E9F20E94CE
:10F25000C48E80912A0C8823B9F2B3CF8D8182307D
:10F2600031F580912F0C823099F080917A028823B9
:10F2700061F081E090912F0C923009F080E023E062
:10F280004FE65FE0632D0F94329725E02E83D2CEB8
:10F290008091280C1092280C882339F38DE39CE48C
:10F2A0000E94AD6680912A0C8823F9F28ACF9D8155
:10F2B000933009F043C180912F0C833099F08091F5
:10F2C0007A02882361F081E090912F0C933009F04D
:10F2D00080E023E04AE65FE06C810F94329785E09E
:10F2E0008E83C3CE8091280C1092280C882339F38A
:10F2F00081E29FE60E94AD6680912A0C8823F9F294
:10F3000060CF8091280C1092280C882309F41FC12B
:10F3100087E79CE30E94AD6680912A0C882309F45C
:10F3200016C14FCF8091280C1092280C882309F425
:10F3300043CE0E94458F80912A0C882309F43CCE4D
:10F3400040CFDF92CF92BF92AF924F9281E09091E7
:10F350002F0C913009F080E08F930E94388C0F9031
:10F360000F900F900F900F900F9022E02E832ACED7
:10F3700081E08E832E818D81281324CE80912F0CE5
:10F380008217F9F080917A02882309F41BCE1F932B
:10F390000F93FF92EF928D8187198F9381E0909167
:10F3A0002F0C2D81921380E08F930E94388C0F9048
:10F3B0000F900F900F900F900F9004CE92E09E83CD
:10F3C000D9CF8091280C1092280C8823D9F20F9461
:10F3D000BB4680912A0C8823A9F2F3CE8091280C99
:10F3E0001092280C882309F4F7CD85ED92E70E944E
:10F3F000AD6680912A0C882309F4EECDE2CE80918F
:10F40000280C1092280C882309F403CE82E091E79F
:10F410000E94AD6680912A0C882309F4FACDD1CEE2
:10F420008091280C1092280C882309F40DCE81E2DB
:10F430009DE70E94AD6680912A0C882309F404CED2
:10F44000C0CE8091280C1092280C882309F41BCE82
:10F4500081ED9FE40E94AD6680912A0C882309F417
:10F4600012CEAFCE8091280C1092280C882309F47C
:10F4700027CE87E99BE70E94AD6680912A0C8823FE
:10F4800009F41ECE9ECE8091280C1092280C882361
:10F4900009F431CE87EB9AE70E94AD6680912A0C81
:10F4A000882309F428CE8DCE8091280C1092280C48
:10F4B000882309F443CE29EE3EE03093D30B20930A
:10F4C000D20B80912A0C882309F438CE7ACE809111
:10F4D000280C1092280C882309F449CE84EA95E779
:10F4E0000E94AD6680912A0C882309F440CE69CE33
:10F4F0009D81891321C090912F0C2D81921302C000
:10F500001092280C80917A028823B1F01F921F92EA
:10F5100026E43FE03F932F938D8187198F9381E0FD
:10F520002D81921380E08F930E94388C0F900F9062
:10F530000F900F900F900F9083E02BCE8D81843031
:10F5400009F07CCE80912F0C843009F4DACE8091C2
:10F550007A02882309F4C3CE81E090912F0C943075
:10F5600009F080E023E04CE55FE06B818CCEDF9218
:10F57000EF92FF920F931F93CF93DF9361E081E0AF
:10F580000E946E8CC091300C85E0E82EEC0ED4E029
:10F59000DC1B13E01C1B02E00C1B81E0F82EFC1AA4
:10F5A000DC2ED194C1112EC080912F0C8823B1F094
:10F5B00080917A02882359F081E090912F0C91116B
:10F5C00080E024E048E65DE06D2D0F943297CF5F38
:10F5D000CE11E8CF85E08093290C0CC08091280CD7
:10F5E0001092280C882321F30E94B48D80912A0C5C
:10F5F0008823F1F2DF91CF911F910F91FF90EF904F
:10F60000DF900895C13011F580912F0C813079F091
:10F6100080917A028823D9F281E090912F0C913069
:10F6200009F080E023E04BE55DE06F2DCECF8091C7
:10F63000280C1092280C882359F380EC91E50E9445
:10F64000AD6680912A0C882319F3D4CFC23009F01B
:10F6500055C080912F0C823081F080917A028823EE
:10F6600009F4B5CF81E090912F0C923009F080E041
:10F6700023E040E55DE0602FA8CF8091280C109238
:10F68000280C882351F38FE592E50E94AD668091A6
:10F690002A0C882311F3AECF80912F0C833081F098
:10F6A00080917A02882309F492CF81E090912F0C07
:10F6B000933009F080E023E044E45DE0612F85CFE2
:10F6C0008091280C1092280C882351F388EF92E542
:10F6D0000E94AD6680912A0C882311F38BCF809114
:10F6E000280C1092280C882391F085ED93E50E9458
:10F6F000AD6680912A0C882351F07CCFC33061F233
:10F70000C43009F064CF80912F0C843041F3809194
:10F710007A02882309F45BCF81E090912F0C94301A
:10F7200009F080E023E046E35DE06D2F4ECF7F924D
:10F730008F929F92AF92BF92CF92DF92EF92FF9201
:10F740000F931F93CF93DF930F942743882309F4DC
:10F750006CC081E08093330C0E94A98D982E61E0EB
:10F7600081E00E946E8CC091300C85E0882E8C0E5A
:10F770007C2E71949EE6E92E9AE0F92ED3E0DC1BF4
:10F7800023E7C22E2AE0D22E12E01C1B38E7A32E5C
:10F790003AE0B32E01E00C1BC11114C080912F0C74
:10F7A000882309F444C080917A02882359F081E0CB
:10F7B00090912F0C911180E024E040E85AE0672DF1
:10F7C0000F9432978091BE0D81115DC080913319E5
:10F7D0009091341920918A0230918B022150310985
:10F7E000821793070CF04FC0C13009F0FCC0809124
:10F7F0002F0C8130C1F180917A02882361F081E081
:10F8000090912F0C913009F080E023E04FEC5CE602
:10F81000602F0F943297992009F455C082E0CF5F92
:10F820008C12BACF8093290C10C082E093CF8091C4
:10F83000280C1092280C882309F4B5CF0E94B48DAF
:10F8400080912A0C882309F4AECFDF91CF911F91CC
:10F850000F91FF90EF90DF90CF90BF90AF909F906F
:10F860008F907F9008958091280C1092280C882307
:10F8700011F285E996E50E94AD6680912A0C8823F5
:10F8800009F4B9CFE2CFC13031F690912F0C91300D
:10F8900059F080917A02882309F4BDCF81E091303C
:10F8A00009F080E020E2B2CF8091280C1092280C61
:10F8B000882379F3B092D30BA092D20B80912A0CBB
:10F8C000882339F3C2CF8091BE0D8111A6C08091EB
:10F8D00033199091341920918A0230918B02215072
:10F8E0003109821793070CF081C0C230A1F48091D6
:10F8F0002F0C823029F180917A02882361F081E017
:10F9000090912F0C923009F080E023E04FEE5CE6FE
:10F91000612F0F94329720913319309134198091CF
:10F92000BE0D81117CC080918A0290918B0201975B
:10F93000281739070CF073C0C33011F184E06FCF82
:10F940008091280C1092280C8823A9F282E996E570
:10F950000E94AD6680912A0C882369F276CF80914F
:10F96000280C1092280C882309F44CC0D092D30B99
:10F97000C092D20B80912A0C882309F443C065CF32
:10F9800080912F0C833089F080917A028823B1F224
:10F9900081E090912F0C933009F080E023E04FED4F
:10F9A0005CE66D2F0F943297C9CF8091280C10928E
:10F9B000280C882349F38FE896E50E94AD66809174
:10F9C0002A0C882309F341CF8091280C1092280C2F
:10F9D000882361F1F092D30BE092D20B80912A0C34
:10F9E000882321F132CF911019CF75CF209133198F
:10F9F00030913419C23009F096CF90912F0C92308B
:10FA000009F4ADCF80917A02882309F484CF81E094
:10FA1000923009F080E020E279CFC23071F3C33038
:10FA200009F08CCF90912F0C933071F280917A0273
:10FA3000882309F483CF81E0933009F080E020E24D
:10FA4000AECF2F923F924F925F926F927F928F92A2
:10FA50009F92AF92BF92CF92DF92EF92FF920F935D
:10FA60001F93CF93DF9300D01F92CDB7DEB70E94D4
:10FA7000A98DE82E61E081E00E946E8C2091300C0F
:10FA80002B8363E0F62EE11002C054E0F52E1B81BB
:10FA9000812F8B5F898323E0722E972D911B9A8390
:10FAA0006624639435EEC32E30E0D32E82E0582EC8
:10FAB000511A462C411A312E319441E0A42E43E0D4
:10FAC000B42E8B81811111C180912F0C882309F4F0
:10FAD000E7C080917A02882359F081E090912F0C41
:10FAE000911180E024E042E45AE0632D0F943297B4
:10FAF000E11013C18B81833009F00FC180912F0C6D
:10FB0000833009F44EC180917A0281115BC194E087
:10FB10009C838C818F5F9B81891309C080912F0CFE
:10FB2000891709F48DC180917A028111A2C18C815B
:10FB30008E5F8C83912C812C2B80211A9B812C81B0
:10FB4000921323C0F401EE0FFF1FE553F349859193
:10FB500094918092450C9093470C8093460C809131
:10FB60002F0C9B81891709F49EC180917A0288230A
:10FB700061F081E090912F0C2C81921380E023E0C2
:10FB800048EE59E0622D0F9432970C8181E0800F8E
:10FB90008C838A94892809F082C12B81821323C027
:10FBA00080912F0C821709F48FC180917A028823EB
:10FBB000D1F082E69CE89F938F9389ED99E09F9323
:10FBC0008F938B81811B8F9381E090912F0C2B81E0
:10FBD000921380E08F930E94388C0F900F900F90BB
:10FBE0000F900F900F9082E0800FE11050C09B812A
:10FBF000891323C080912F0C891709F474C1809157
:10FC00007A028823D1F086E69CE89F938F938BEC51
:10FC100099E09F938F938B81811B8F9381E09091CB
:10FC20002F0C2B81921380E08F930E94388C0F90C1
:10FC30000F900F900F900F900F9083E0800F9B819B
:10FC4000891323C080912F0C891709F45BC180911F
:10FC50007A028823D1F08AE69CE89F938F938AEBFF
:10FC600099E09F938F938B81811B8F9381E090917B
:10FC70002F0C2B81921380E08F930E94388C0F9071
:10FC80000F900F900F900F900F9084E0800F9B814A
:10FC90009F5F9B832981921314CF8093290C0EC000
:10FCA0008091280C1092280C882309F412CF0E940E
:10FCB000B48D80912A0C882309F40BCF0F900F90FC
:10FCC0000F900F90DF91CF911F910F91FF90EF90C8
:10FCD000DF90CF90BF90AF909F908F907F906F906C
:10FCE0005F904F903F902F9008959B81913091F5B8
:10FCF00080912F0C8130F9F080917A02882309F4E9
:10FD0000F7CE81E090912F0C913009F080E023E054
:10FD100040E35AE0642D0F9432978B81F81209C0AA
:10FD200080912F0C8F1509F45CC080917A028111AB
:10FD300071C0FC82EECE8091280C1092280C882392
:10FD4000D9F287E290E80E94AD6680912A0C882360
:10FD500099F2B4CF2B81223009F0CACE80912F0CBA
:10FD6000823081F080917A02882309F4C1CE81E04B
:10FD700090912F0C923009F080E023E041E25AE0AC
:10FD8000652DC9CF8091280C1092280C882351F33F
:10FD900089EC99E90E94AD6680912A0C882311F3C1
:10FDA0008DCF8091280C1092280C882309F4ABCEBB
:10FDB00083EB96E50E94AD6680912A0C882309F4B6
:10FDC000A2CE7CCF81E090912F0C933009F080E09F
:10FDD00023E049E15AE06A810F94329724E02C83B2
:10FDE00098CE8091280C1092280C882309F49DCF7E
:10FDF0008091590286258093590270927A02C1142B
:10FE0000D10411F00F94523180912A0C882309F407
:10FE10008CCF54CF6B81611B81E090912F0C2B8193
:10FE2000921380E09091590228E03AE0911102C0CB
:10FE300024E03AE001E04BE05AE00E94F49A79CFE6
:10FE40008091280C1092280C882309F46CCE8091A4
:10FE5000B80986258093B80970927A02A114B1047A
:10FE600011F00F94273680912A0C882309F45BCE79
:10FE700025CF6B81611B81E090912F0C2B81921318
:10FE800080E09091B80928E03AE0911102C024E0A6
:10FE90003AE001E047EF59E00E94F49A48CE882406
:10FEA0008394912C4BCE8091280C1092280C88239F
:10FEB00009F45BCE8EE299E40E94AD6680912A0C33
:10FEC000882309F452CEFACE8091280C1092280C87
:10FED000882309F46ACE0E94628C80912A0C8823C0
:10FEE00009F463CEEBCE8091280C1092280C882365
:10FEF00009F485CE0E94668C80912A0C882309F42F
:10FF00007ECEDCCE8091280C1092280C882309F438
:10FF10009ECE0E946A8C80912A0C882309F497CE89
:10FF2000CDCECF92DF92EF92FF920F931F93CF939C
:10FF3000DF930091040261E081E00E946E8CC09129
:10FF4000300CEC2E85E0F82EFC0EDC2ED194C11185
:10FF500014C080912F0C882309F44BC080917A0241
:10FF6000882359F081E090912F0C911180E024E0DA
:10FF70004EE659E06D2D0F9432971FEFD1E0CC2E55
:10FF8000CE188091290718170CF05BC0011779F182
:10FF9000812F17FD802F40912507509126076091F2
:10FFA000270770912807082E04C076956795579506
:10FFB00047950A94D2F740FD1AC0DC1315C0809310
:10FFC000450C80912F0C8D1759F180917A0288236E
:10FFD00059F081E090912F0C9D1380E023E04EE5D5
:10FFE00059E06C2D0F94329717FD29C0DF5F1F5F1A
:10FFF000C8CF8091280C1092280C882309F4AECF2A
:020000021000EC
:100000000E94B48D80912A0C882309F4A7CFDF9138
:10001000CF911F910F91FF90EF90DF90CF900895B7
:100020008091280C1092280C882379F28CE59CE4AE
:100030000E94AD6680912A0C882339F2E8CFDE5FFA
:10004000D6CFCF5FFC1283CFD093290CE0CF7F9225
:100050008F929F92AF92BF92CF92DF92EF92FF92D8
:100060000F931F93CF93DF930E94A98D182F61E008
:1000700081E00E946E8CC091300C0C2F85E0782EB0
:100080007C0E85E0F82EFC1A86E0E82EEC1A84E05F
:10009000D82EDC1A83E0C82ECC1A82E0982E9C1A47
:1000A00093EBA92E98E0B92E81E0882E8C1AC1110D
:1000B0004AC080912F0C882361F180917A028823B5
:1000C00061F0602F619581E090912F0C911180E09B
:1000D00024E042E259E00F943297111193C1C530E8
:1000E00009F022C180912F0C853009F4BBC08091AA
:1000F0007A02882361F081E090912F0C953009F00D
:1001000080E023E048EE58E06F2D0F943297D7E05F
:100110007AC18091280C1092280C882371F20E94D9
:10012000B48D80912A0C882341F2DF91CF911F91E9
:100130000F91FF90EF90DF90CF90BF90AF909F9086
:100140008F907F900895C13079F580912F0C813088
:10015000D1F080917A02882309F4BFCF1F9281E108
:1001600099E09F938F938F9281E090912F0C913023
:1001700009F080E08F930E94388C0F900F900F90C1
:100180000F900F90AACF8091280C1092280C8823F2
:1001900001F3B092D30BA092D20B0E944F8D8091AD
:1001A0002A0C8823B1F2C1CFC23009F00EC1809170
:1001B0002F0C8230A1F080917A02882361F081E0D7
:1001C00090912F0C923009F080E023E048E059E054
:1001D000692D0F943297112309F499CF13C180919F
:1001E000280C1092280C882331F388E599E50E94A9
:1001F000AD6680912A0C8823F1F297CF80912F0C65
:10020000833081F080917A02882309F4F8C081E07C
:1002100090912F0C933009F080E023E04BEF58E0F1
:100220006C2DD7CF8091280C1092280C882351F385
:100230008AE29BE50E94AD6680912A0C882311F327
:1002400074CF8091280C1092280C882309F4C8C020
:1002500085EC94E60E94AD6680912A0C882309F40F
:10026000BFC063CF8091280C1092280C882309F41A
:100270003ECF8FE293E80E94AD6680912A0C8823DE
:1002800009F435CF52CF8091280C1092280C882386
:1002900009F452C089E29EE50E94AD6680912A0C65
:1002A000882309F449C041CF8091280C1092280C72
:1002B000882309F4AFC08AE59FE50E94AD6680916E
:1002C0002A0C882309F4A6C030CF8091280C109204
:1002D000280C882309F44BC080EB9BE90E94AD6693
:1002E00080912A0C882309F442C01FCF8091280CEA
:1002F0001092280C882309F453C00E94CB8D20E073
:1003000040E070E060E08CEB9CE4DF91CF911F91C6
:100310000F91FF90EF90DF90CF90BF90AF909F90A4
:100320008F907F900C94CC8CC63009F0F0CE8091E9
:100330002F0C863009F4A7CF80917A02882309F424
:10034000E6CE81E090912F0C963009F080E023E01A
:100350004FED58E06E2D0F943297D7E081E08D0F6E
:100360008C1315C080912F0C8C1709F4AECF80919F
:100370007A02882361F06C2F601B81E090912F0C32
:100380009C1380E023E04AEC58E00F94329782E01F
:100390008D0F8C1313C090912F0C9C1709F4A6CFCE
:1003A00080917A02882351F06C2F601B81E09C13AE
:1003B00080E023E048EB58E00F943297CF5FC711FD
:1003C00076CEDD5FD093290CB0CEC33009F416CFC2
:1003D000C43009F082CE80912F0C843009F431CFE3
:1003E00080917A02882359F081E090912F0C94300B
:1003F00009F080E023E046EF58E06D2DEACE1123AE
:1004000009F492CFD5E0DC13A9CF80912F0C8D1782
:1004100009F44ACF80917A02882309F49FCF6C2F88
:10042000601B81E090912F0C9C1380E023E043ED52
:1004300058E00F94329792CFCF92DF92EF92FF92D3
:1004400020E030E04AE754E46091360770913707C6
:1004500080913807909139070F94A1BB0F9499C3ED
:100460006B017C0125E030E040E050E00F94A1C139
:10047000A7019601261B370B480B590BCA01B9017E
:100480000F9442BB20E030E04AE754E40F9427C3C6
:10049000FF90EF90DF90CF900895FC0180819181D3
:1004A000A281B3818093360790933707A0933807D2
:1004B000B093390720E040E070E060E088E998E41C
:1004C0000C94CC8C61116093050240932B078C3007
:1004D00008F03AC0E82F880FFF0B8827ED58FD473A
:1004E0008F4F0D9424C2A6827F828A82A9828D8238
:1004F000908293829F829682A48299829C828BE6CC
:1005000096E521E02093310720E040E070E060E0D4
:100510000C94CC8C83E796E5F4CF87E796E5F1CF92
:100520008BE796E5EECF8FE796E5EBCF83E896E590
:10053000E8CF87E896E5E5CF8BE896E5E2CF109225
:100540006F0C80E29FE3DDCF0C944F8D87E696E53C
:10055000D8CF8FE696E5D5CFCF92DF92EF92FF927C
:100560006B017C0120E030E0A9010F943BBB87FDCB
:1005700026C06DEB77E386E095E3A70196010F9423
:100580002DC26B017C0120E030E0A9010F943BBB40
:1005900020E030E040E05FE387FF04C020E030E08F
:1005A00040E05FEBC701B6010F942DC20F9499C3D1
:1005B000CB01FF90EF90DF90CF900D945D186DEB25
:1005C00077E386E095EBD9CF0F9442BB20E030E093
:1005D000A9010F942DC20C94AC82CF92DF92EF92BE
:1005E000FF92CF93DF9300D01F92CDB7DEB76B01A0
:1005F0007C0120E030E0A9010F943BBB87FD1BC0CC
:100600006DEB77E386E095E3A70196010F942DC289
:1006100069837A838B839C83CE0101960F947397B1
:100620000F900F900F900F90DF91CF91FF90EF9070
:10063000DF90CF9008956DEB77E386E095EBE4CF04
:100640000F9442BB20E030E04AE754E40F9427C304
:1006500020E030E0A9010F942DC20C94ED824F925E
:100660005F926F927F928F929F92AF92BF92CF9242
:10067000DF92EF92FF920F931F93CF93DF9361E08E
:1006800081E00E946E8CC091300C65E0562E5C0EAD
:10069000D3E0DC1B82E0782E7C1A81E0682E6C1A95
:1006A0004C2E4194C11137C080912F0C8823B1F09A
:1006B00080917A02882359F081E090912F0C91115A
:1006C00080E024E043E958E0642D0F943297CF5F37
:1006D000C511E8CF84E08093290C0CC08091280CD0
:1006E0001092280C882321F30E94B48D80912A0C4B
:1006F0008823F1F2DF91CF911F910F91FF90EF903E
:10070000DF90CF90BF90AF909F908F907F906F9031
:100710005F904F900895C13009F061C080912F0C17
:100720008130E9F080917A02882389F211E080918A
:100730002F0C813009F010E06091C0197091C1193F
:100740008091C2199091C3190E94F23800E09C0177
:1007500048E558E0662D812F0E94F49AB8CF809129
:10076000280C1092280C8823E9F220E030E040E2C7
:1007700051E46091C0197091C1198091C219909192
:10078000C3190F94A1BB20E030E0A9010F942DC242
:1007900020E030E84BE355E40F942DC20F94A0C342
:1007A0001F92912C812C45E3A42E40E4B42E6B01C2
:1007B00010E7E12E17E1F12E00E010E028E434EF1D
:1007C0004FEF5FEF60EC79E188E598E00E94F28DF1
:1007D0000F9080912A0C882309F4A4CF8BCFC230CC
:1007E00009F09FC080912F0C8230D9F080917A025D
:1007F000882309F46CCF11E080912F0C823009F02E
:1008000010E06091C4197091C5198091C61990913A
:10081000C7190E94F23800E09C0149E458E0672DB6
:100820009ACF8091280C1092280C8823F9F220E0AE
:1008300030E040E251E46091C4197091C519809193
:10084000C6199091C7190F94A1BB20E030E0A9010F
:100850000F942DC220E030E84BE355E40F942DC2F5
:100860000F94A0C31F92912C812C25E3A22E20E48B
:10087000B22E6B0110E7E12E17E1F12E00E010E03F
:1008800028E434EF4FEF5FEF64EC79E189E498E01E
:100890000E94F28D0F9080912A0C882309F4A6CF34
:1008A00029CF8091280C1092280C882309F441C08C
:1008B00020E030E04AE754E46091C8197091C9190A
:1008C0008091CA199091CB190F94A1BB20E030E020
:1008D000A9010F942DC220E030EA4CE056E40F94B9
:1008E0002DC20F94A0C31F92912C812C8BE6A82EB1
:1008F00080E4B82E6B0110E5E12E16E4F12E00E045
:1009000010E028ED3CED4FEF5FEF68EC79E18AE312
:1009100098E00E94F28D0F9080912A0C882349F074
:10092000E9CEC33009F0D3CE80912F0C833009F487
:10093000B8CF80917A02882309F4C9CE11E0809162
:100940002F0C833009F010E06091C8197091C9191B
:100950008091CA199091CB190E94ED8200E09C0110
:100960004AE358E06D2FF7CE2CEA35EC47E25EE320
:1009700060911C0770911D0780911E0790911F07C1
:100980000F9427C360933E1970933F1980934019C9
:100990009093411908952CEA35EC47E25EE36091AB
:1009A00020077091210780912207909123070F94CF
:1009B000A1BB60933A1970933B1980933C199093B3
:1009C0003D1908958091330C9091340CA091350C11
:1009D000B091360C8093550290935602A093570223
:1009E000B09358020895FC0184910895FC01808120
:1009F0000895FC01A081B1811C92A281B3818C91E8
:100A00008F5F8C930280F381E02D90818CE0989F22
:100A1000800D1124E9EFF9E113AE84AF0895119828
:100A2000000000009091020187FD909591709093D5
:100A30000001119A00000000000000001198000061
:100A400000009091020186FD9095917090930001B5
:100A5000119A000000000000000011980000000042
:100A60009091020185FD9095917090930001119AEB
:100A700000000000000000001198000000009091AC
:100A8000020184FD9095917090930001119A0000ED
:100A90000000000000001198000000009091020189
:100AA00083FD9095917090930001119A00000000D1
:100AB000000000001198000000009091020182FDEA
:100AC0009095917090930001119A00000000000031
:100AD00000001198000000009091020181FD9095A6
:100AE000917090930001119A000000000000000036
:100AF0001198000000008091020181708093000134
:100B0000119A0000000000000000089590E080E0CD
:100B1000089590E080E00895282F90917D0C833017
:100B200021F495FD0FC094FD0FC0892F90E0B0E037
:100B3000A0E004C0B695A795979587952A95D2F71A
:100B40008170089581E0089580E008950F931F93C8
:100B5000CF938C01C62F87EB9CE10F942246C801EE
:100B60000F9422468AE30F94974580E38C0F0F94ED
:100B700097458AE0CF911F910F910D9497458AE395
:100B80009EE10F94224660E08AE29EE10E94A685E3
:100B900060E085E19EE10E94A68561E08EE09EE135
:100BA0000E94A68561E083E09EE10E94A68561E047
:100BB00083EF9DE10E94A68560E08AEE9DE10E94A0
:100BC000A68561E080EE9DE10E94A68561E086ED4C
:100BD0009DE10E94A68561E08FEC9DE10E94A685C3
:100BE00061E087EC9DE10E94A68561E089EB9DE1D3
:100BF0000E94A68561E08BEA9DE10E94A68560E0E7
:100C00008CE99DE10E94A68560E08EE89DE10E944E
:100C1000A68560E088E79DE10E94A68561E087E601
:100C20009DE10E94A68561E088E59DE10E94A68580
:100C300061E081E59DE10E94A68560E08AE49DE196
:100C40000E94A68561E081E49DE10E94A68561E0A5
:100C50008CE29DE10E94A68561E08EE19DE10E940B
:100C6000A68561E08BE09DE10E94A68560E08EEFA5
:100C70009CE10E94A68561E089EF9CE10E94A68527
:100C800061E08CEE9CE10E94A68560E088ED9CE12D
:100C90000E94A68560E085EC9CE10E94A68560E04C
:100CA00087E49AE10E948985682F61708CEB9CE152
:100CB0000C94A685AF92BF92CF92DF92EF92FF92F3
:100CC0000F931F93CF93DF936B01E9014A3009F42F
:100CD000C1C0453109F073C0DB011296ED91FC9162
:100CE000F280C681D78180910201809582708093C5
:100CF000000188E28A950000E9F7BF2CB29420EF4A
:100D0000B22230E1A32EAF0C48E2E42E88EF0E941D
:100D10000F858E2D8A950000E9F7BFE1BF1508F415
:100D200085C08F2D807780680E940F858B2D0E9453
:100D30000F858E2D8A950000E9F780E80E940F85C7
:100D400080E00E940F858E2D8A950000E9F78AEFDA
:100D50000E940F858E2D8A950000E9F78E01005FB5
:100D60001F4F8881807F0E940F8589918295807FA7
:100D70000E940F85C017D107A1F78E2D8A9500001C
:100D8000E9F7F394E0E1BE0EFA10C0CF80910201C2
:100D9000827080930001D6011296CD91DC91CE0134
:100DA0000F94F9A3811147C2DF91CF911F910F9149
:100DB000FF90EF90DF90CF90BF90AF900895FB0130
:100DC00002811381423309F4F1C108F4F5C14634BC
:100DD00009F4E2C1473409F4E5C14B3329F58981AF
:100DE0002B81D80112966C91129713964C91213059
:100DF00009F438C2233009F002C238EF380F582FF7
:100E000091E0431708F490E041E0531708F040E008
:100E100031E0561708F430E0592F542B352309F0F0
:100E200016C2942309F013C281E0BECF80EE8F0D6D
:100E30008068807F0E940F858F2D8295807F0E9421
:100E40000F858E2D8A950000E9F780E80E940F85B6
:100E500080E877CF809101018260809301018091C9
:100E60000201827080930001809101018160809372
:100E7000010180910201817080930001099A119A09
:100E800080910201809582708093000188E28A95AA
:100E90000000E9F788E790E0CEE9DFE0FE01319756
:100EA000F1F70197D9F788EF0E940F8518E2812F9B
:100EB0008A950000E9F780E20E940F8580E00E9499
:100EC0000F85812F8A950000E9F780E00E940F8549
:100ED00080E80E940F85812F8A950000E9F780E065
:100EE0000E940F8580E10E940F85812F8A95000066
:100EF000E9F7CE010197F1F7CE010197F1F7CE01A5
:100F00000197F1F7CE010197F1F7CE010197F1F7C3
:100F1000CE010197F1F7CE010197F1F7CE010197CC
:100F2000F1F7CE010197F1F7CE010197F1F7CE016C
:100F30000197F1F7CE010197F1F7CE010197F1F793
:100F4000CE010197F1F72197F1F780E20E940F851A
:100F500080E40E940F85812F8A950000E9F780E2E6
:100F60000E940F8580E60E940F851A950000E9F720
:100F700010E0D0E0C8E28D2F807780680E940F8556
:100F8000812F0E940F858C2F8A950000E9F780E859
:100F90000E940F8580E00E940F858C2F8A950000AB
:100FA000E9F78AEF0E940F858C2F8A950000E9F7F8
:100FB00090E21198000000008091020181708093FE
:100FC0000001119A000000000000000011980000CC
:100FD000000080910201817080930001119A00004D
:100FE0000000000000001198000000008091020144
:100FF000817080930001119A000000000000000041
:10100000119800000000809102018170809300011E
:10101000119A00000000000000001198000000007C
:1010200080910201817080930001119A00000000FC
:101030000000000011980000000080910201817002
:1010400080930001119A0000000000000000119838
:101050000000000080910201817080930001119ACC
:1010600000000000000000001198000000008091C6
:101070000201817080930001119A000000000000BD
:10108000000011980000000080910201817080939F
:101090000001119A000000000000000011980000FB
:1010A000000080910201817080930001119A00007C
:1010B0000000000000001198000000008091020173
:1010C000817080930001119A000000000000000070
:1010D000119800000000809102018170809300014E
:1010E000119A0000000000000000119800000000AC
:1010F00080910201817080930001119A000000002C
:101100000000000011980000000080910201817031
:1011100080930001119A0000000000000000119867
:101120000000000080910201817080930001119AFB
:1011300000000000000000001198000000008091F5
:101140000201817080930001119A000000000000EC
:1011500000008C2F8A950000E9F7915009F029CF03
:1011600088EF0E940F858C2F8A950000E9F7DF5FDA
:10117000105FD03209F0FFCE80E00E940F8580EC36
:101180000E940F85CA950000E9F7809102018270E4
:101190008093000181E008CED80115968C91888358
:1011A00081E002CEF80181818883FACFB901C801BC
:1011B0000F9416A481E0F8CD443171F0473109F065
:1011C00033CE1882F80182818983858181508A8398
:1011D00083818B8381E0E8CDD80115964C911597DA
:1011E00050E0440F551F70E060E016968D919C9181
:1011F0000F94B0C6C8010F940FA481E0D5CD481755
:1012000008F412CE861708F40FCEFA80E12CD12C08
:10121000243070F41DC0BE01C8010F9416A489814A
:1012200098819D0D98838E0D8983FF0C09F4FCCD68
:10123000F7FEF6CFF0CF4D8150E0440F551F70E020
:1012400060E08E819F810F94B0C681E0ADCDFA80C1
:1012500030E0F901E251FD4FD08026513D4FF901B8
:10126000E080E6CF58E0580F382FCACDEF92FF92BA
:101270000F931F93CF93DF93EC018B017A018A8543
:101280009B858617970731F0888199810F94EFA588
:101290001B870A87B701888199810F9459982E81FD
:1012A0003F81820F932F911D9F838E8390E080E07A
:1012B000DF91CF911F910F91FF90EF9008959F9232
:1012C000AF92BF92CF92DF92EF92FF920F931F9354
:1012D000CF93DF93EC018B01942EA52E8A859B85FD
:1012E0008617970731F0888199810F94EFA51B87A6
:1012F0000A8788859985019649F5BC800A818E8187
:10130000080FC880D980D6015596ED91FC91C60191
:101310001995B80EE92CFA2C10E0F70121917F0104
:10132000211127C08E819F81810F911D9F838E8304
:1013300090E080E0DF91CF911F910F91FF90EF90AF
:10134000DF90CF90BF90AF909F9008950E811F8146
:10135000692D7A2D888199810F945998800F912F4A
:10136000911D288539852817390738F681E090E0E6
:10137000E1CF4B2D602FC6010F9447A6080F180F21
:10138000CCCFDF92EF92FF920F931F93CF93DF9317
:10139000EC01D62E1CAD0BAD7C0184E0E80EF11CF7
:1013A000E98DFA8DC7011995412F480F2D2D602F1A
:1013B000C7010F9447A69BAD890F8BAF81E090E0EA
:1013C000DF91CF911F910F91FF90EF90DF900895E3
:1013D000CF92DF92EF92FF920F931F93CF93DF9301
:1013E000CDB7DEB72C970FB6F894DEBF0FBECDBFDA
:1013F000F090341AE090351A20917B0821111DC01D
:1014000046EB51E26E2D8F2D0F94B3A690E080E055
:10141000F80EF092341AE092351A99272C960FB6EE
:10142000F894DEBF0FBECDBFDF91CF911F910F911A
:10143000FF90EF90DF90CF900895C090011AD09068
:10144000021A2DEF39E13A8329832F2D30E03C83B6
:101450002B832E2D30E03E832D8318861F827A87C2
:1014600069871C861B860FE519E89E012F5F3F4F99
:1014700043EF54E8BC01C6010F94FE81B6018DEF25
:1014800099E10F94EFA58F819885C2CFCF93C62F96
:101490000F940739882319F0CF910D9461388C2F60
:1014A000CF910895CF93DF93EB010F9407398823F1
:1014B00019F00F945138EB01CE01DF91CF910895CF
:1014C0000F931F93CF93DF9300D01F92CDB7DEB75A
:1014D0009C0107E51CE090E1E3E7FDE0D801019005
:1014E0000D929A95E1F7F901208131814281538172
:1014F000F80160857185828593850F942DC2F8016E
:10150000608771878287938780E090E0A0EAB0E4EB
:1015100089839A83AB83BC83CE0101960F94F00636
:101520000F900F900F900F90DF91CF911F910F911F
:101530000895CF9384E50F940739C0E08823D9F04C
:101540000F946138C82F1816B4F40F9458598DE4CD
:101550000F94974580917408909175080F94EEA7A9
:101560006C2FCC0F770B8EE699E10F9417498AE028
:101570000F949745CFEF8C2FCF91089583E50F946B
:1015800007398823E9F00F94489E6093670C7093A5
:10159000680C8093690C90936A0C0F94893820E052
:1015A00030E04AE754E40F94A1BB0F94A0C36093CA
:1015B0001D0270931E0280931F02909320020895D3
:1015C0008091690784FD13C080916B0787FD0FC070
:1015D00080916C07837059F40E944EEB8091300724
:1015E000882321F0109230071092310708950E944D
:1015F0003DEB88E50F94B938882331F05F9A8091EC
:10160000CF0B8E7F8093CF0B89E50F94B938882359
:1016100031F08A9A8091CF0B8D7F8093CF0B8AE532
:101620000F94B938882359F0809108018095817012
:10163000809306018091CF0B8B7F8093CF0B85E445
:101640000F94B938882351F20F94FE42C7CF80918E
:101650003E0790913F07009731F04AE050E070E07C
:1016600060E00D9419B960E070E0CB0108958091BD
:101670006907827149F480916B078C7829F4809115
:101680006C07837009F475C082E40F94B93888231D
:1016900051F00E94278B6093D1137093D2138093E3
:1016A000D3139093D41383E50F94B938882351F062
:1016B0000F9489386093011470930214809303147B
:1016C0009093041484E50F94B938882351F00F9453
:1016D00089386093051470930614809307149093CF
:1016E000081488E50F94B938882351F00F9489388D
:1016F0006093840D7093850D8093860D9093870D74
:1017000089E50F94B938882351F00F948938609394
:10171000880D7093890D80938A0D90938B0D8AE5C7
:101720000F94B9388823B1F00F94893860938C0DE9
:1017300070938D0D80938E0D90938F0D2DEC3CEC5E
:101740004CEC5DE30F943BBB181624F084E798E162
:101750000F94224685E40F94B938882351F00F94F2
:1017600089386093900D7093910D8093920D9093B2
:10177000930D0895AF92BF92CF92DF92EF920F93A5
:101780001F93CF93DF935B01EA016901882309F47A
:1017900063C08DE698E10F942246F5016081718166
:1017A0008281938146E00F945721E1100BC084E6BB
:1017B00098E10F942246688179818A819B8146E075
:1017C0000F9457218DE598E10F942246F601608130
:1017D00071818281938143E00F94572186E598E1DE
:1017E0000F942246F801608171818281938143E0E8
:1017F0000F9457218DE498E10F942246F601208141
:10180000318142815381F8016081718182819381AC
:101810000F942CC243E00F945721EE20F9F08AE098
:101820000F94974588E398E10F9422466881798167
:101830008A819B8146E00F9457218AE00F94974557
:101840008AE0DF91CF911F910F91EF90DF90CF90C1
:10185000BF90AF900D949745E110E4CFDF91CF9109
:101860001F910F91EF90DF90CF90BF90AF900895B0
:10187000CF93DF93CDB7DEB720E2488559856F81DE
:101880008E810F943297DF91CF9108954FE350E00E
:10189000BC0184ED9BE00D94F5C663E972E084E63B
:1018A00090E00E9457646AEB72E084E690E00C944A
:1018B000576481110C944D8C68EB71E084E190E0E9
:1018C0000C9457640E94F9E60C94598C0F94D32C15
:1018D0000C94598C0F94500F0C944D8C282F10920F
:1018E0003B0C80912B0C90912C0CA0912D0CB09165
:1018F0002E0CB7FF08C010922B0C10922C0C1092DB
:101900002D0C10922E0C80912F07882331F080919E
:101910002B0C80932F0C10922A0C8091290C1816F6
:10192000FCF4082E000C990B821B910920912F0CBE
:10193000022E000C330B2817390794F097FF02C0D2
:1019400090E080E080932F0C092E000CAA0BBB0BBB
:1019500080932B0C90932C0CA0932D0CB0932E0CF9
:1019600080912F0C6623A9F09091300C891714F404
:101970008093300C2091300C022E000C330B2C5F26
:101980003F4F482F082E000C550B241735071CF429
:1019900084508093300C08958F929F92AF92BF92A3
:1019A000EF92FF920F931F93CF93DF93EC018B0184
:1019B000E42EF22E8091F7199091F8198C179D075B
:1019C00009F440C020910A0927FD10920A0927E76F
:1019D000C736D20709F041C080519E4971F40F9477
:1019E000489E6E517B4F8F4F9F4F60930C097093B1
:1019F0000D0980930E0990930F09D093F819C093A5
:101A0000F71930E020E000932B0C10932C0C20935E
:101A10002D0C30932E0CE092300CF092290CC0511A
:101A2000DE4931F41092310710920B091092300701
:101A300082E080937A0281E080932A0C10922C0736
:101A400010922407DF91CF911F910F91FF90EF909B
:101A5000BF90AF909F908F9008952EE9C031D2072C
:101A600061F68756974719F0C0E1DEE9C6CF0F94BB
:101A7000489E80900C0990900D09A0900E09B0909E
:101A80000F09681979098A099B0997FFEDCF8091A1
:101A9000CF0B8770873041F7C9ECD9E9AECF20E092
:101AA00040E070E060E080E19EE90C94CC8C0F9304
:101AB0001F93CF93DF93CDB7DEB76E970FB6F89431
:101AC000DEBF0FBECDBF282F082E000C330B909128
:101AD0000002409101028F3F39F0F901EE0FFF1F24
:101AE000EE5FFD4F908141814F939F933F938F9382
:101AF0008BEA94E29F938F938E010F5F1F4F1F938A
:101B00000F930F94D2BAC8010E94468C0E944F8D49
:101B10000FB6F894DEBF0FBECDBF6E960FB6F89429
:101B2000DEBF0FBECDBFDF91CF911F910F91089502
:101B3000CF930F94500F0E94F9E6C82F882319F015
:101B400080E00F9485258C2F0E94598CCF910C94A6
:101B50004F8D8091D1199091D219891B8F7011F4FA
:101B60000D94EC4281E00895E0910B09EE2389F099
:101B7000E150E0930B0988E0E89FF0011124E55360
:101B8000F74F6281738127814681808191810C9416
:101B9000CC8C0C944F8DE0910B09E63010F581E070
:101BA0008E0F80930B0940912B0C50912C0C60915F
:101BB0002D0C70912E0C9091300C8091290C28E006
:101BC000E29FF0011124E553F74F2091F71930916E
:101BD000F81931832083428353836483758396830A
:101BE000878308952F923F924F925F926F927F92D8
:101BF0008F929F92AF92BF92CF92DF92EF92FF921D
:101C00000F931F93CF93DF9300D000D0CDB7DEB7F3
